 libGLES_CM

 Timestamp is 4be8cfbf (Tue May 11 12:32:15 2010)

 Preferred load address is 10000000

 Start         Length     Name                   Class
 0001:00000000 00000004H .CRT$XCA                CODE
 0001:00000004 00000004H .CRT$XCZ                CODE
 0001:00000008 00000004H .CRT$XIA                CODE
 0001:0000000c 00000004H .CRT$XIZ                CODE
 0001:00000010 00000004H .CRT$XPA                CODE
 0001:00000014 00000004H .CRT$XPZ                CODE
 0001:00000018 00000004H .CRT$XTA                CODE
 0001:0000001c 00000004H .CRT$XTZ                CODE
 0001:00000020 00012d43H .rdata                  CODE
 0001:00012d64 00000027H .rdata$debug            CODE
 0001:00012d8c 000605f8H .text                   CODE
 0001:00073384 00000024H .xdata                  CODE
 0001:000733a8 0000003cH .idata$2                CODE
 0001:000733e4 00000014H .idata$3                CODE
 0001:000733f8 000001e0H .idata$4                CODE
 0001:000735d8 0000015aH .idata$6                CODE
 0001:00073740 000010a7H .edata                  CODE
 0002:00000000 000001e0H .idata$5                DATA
 0002:000001e0 0000000cH .data                   DATA
 0002:000001ec 00000010H .bss                    DATA
 0003:00000000 00001f70H .pdata                  DATA

  Address         Publics by Value              Rva+Base       Lib:Object

 0000:00000000       ___safe_se_handler_count   00000000     <absolute>
 0000:00000000       ___safe_se_handler_table   00000000     <absolute>
 0001:00000000       __xc_a                     10001000     corelib0:crt0init.obj
 0001:00000004       __xc_z                     10001004     corelib0:crt0init.obj
 0001:00000008       __xi_a                     10001008     corelib0:crt0init.obj
 0001:0000000c       __xi_z                     1000100c     corelib0:crt0init.obj
 0001:00000010       __xp_a                     10001010     corelib0:crt0init.obj
 0001:00000014       __xp_z                     10001014     corelib0:crt0init.obj
 0001:00000018       __xt_a                     10001018     corelib0:crt0init.obj
 0001:0000001c       __xt_z                     1000101c     corelib0:crt0init.obj
 0001:00000994       sGLES1FunctionTable        10001994     eglglue.obj
 0001:000009c0       ??_C@_0CH@JLEJGINJ@glEGLImageTargetRenderbufferStor@ 100019c0     eglglue.obj
 0001:000009e8       ??_C@_0BN@FPPCHDBA@glEGLImageTargetTexture2DOES?$AA@ 100019e8     eglglue.obj
 0001:00000a08       ??_C@_0BE@MPDFJJLL@glMultiDrawElements?$AA@ 10001a08     eglglue.obj
 0001:00000a1c       ??_C@_0BC@IBABPJFA@glMultiDrawArrays?$AA@ 10001a1c     eglglue.obj
 0001:00000a30       ??_C@_0BB@CEFEJGJJ@glUnmapBufferOES?$AA@ 10001a30     eglglue.obj
 0001:00000a44       ??_C@_0P@MBENIONB@glMapBufferOES?$AA@ 10001a44     eglglue.obj
 0001:00000a54       ??_C@_0BH@HANHAAH@glGetBufferPointervOES?$AA@ 10001a54     eglglue.obj
 0001:00000a6c       ??_C@_0BD@PIBFHNP@glTexBindStreamIMG?$AA@ 10001a6c     eglglue.obj
 0001:00000a80       ??_C@_0BM@MBNDOCOP@glGetTexStreamDeviceNameIMG?$AA@ 10001a80     eglglue.obj
 0001:00000a9c       ??_C@_0CD@OCNNIBKN@glGetTexStreamDeviceAttributeivI@ 10001a9c     eglglue.obj
 0001:00000ac0       ??_C@_0BB@JDDNIFAN@glGenProgramsARB?$AA@ 10001ac0     eglglue.obj
 0001:00000ad4       ??_C@_0BE@EJCMOJPP@glDeleteProgramsARB?$AA@ 10001ad4     eglglue.obj
 0001:00000ae8       ??_C@_0BB@OAGHGJAC@glBindProgramARB?$AA@ 10001ae8     eglglue.obj
 0001:00000afc       ??_C@_0BD@HIBLHAHB@glProgramStringARB?$AA@ 10001afc     eglglue.obj
 0001:00000b10       ??_C@_0BO@HGKLJN@glDisableVertexAttribArrayARB?$AA@ 10001b10     eglglue.obj
 0001:00000b30       ??_C@_0BN@FKABDPBF@glEnableVertexAttribArrayARB?$AA@ 10001b30     eglglue.obj
 0001:00000b50       ??_C@_0BJ@KNOILOPF@glVertexAttribPointerARB?$AA@ 10001b50     eglglue.obj
 0001:00000b6c       ??_C@_0BM@DIEJBCK@glProgramEnvParameter4xvIMG?$AA@ 10001b6c     eglglue.obj
 0001:00000b88       ??_C@_0BL@IPGFFKBA@glProgramEnvParameter4xIMG?$AA@ 10001b88     eglglue.obj
 0001:00000ba4       ??_C@_0BO@HBENEBND@glProgramLocalParameter4xvIMG?$AA@ 10001ba4     eglglue.obj
 0001:00000bc4       ??_C@_0BN@EBNCCGNG@glProgramLocalParameter4xIMG?$AA@ 10001bc4     eglglue.obj
 0001:00000be4       ??_C@_0BE@PEDBDIJA@glVertexAttrib4xIMG?$AA@ 10001be4     eglglue.obj
 0001:00000bf8       ??_C@_0BO@OHCIBKNP@glProgramLocalParameter4fvARB?$AA@ 10001bf8     eglglue.obj
 0001:00000c18       ??_C@_0BN@DBLLDHNC@glProgramLocalParameter4fARB?$AA@ 10001c18     eglglue.obj
 0001:00000c38       ??_C@_0BM@JFOBMKCG@glProgramEnvParameter4fvARB?$AA@ 10001c38     eglglue.obj
 0001:00000c54       ??_C@_0BL@PPAMELBE@glProgramEnvParameter4fARB?$AA@ 10001c54     eglglue.obj
 0001:00000c70       ??_C@_0BE@IEFICJJE@glVertexAttrib4fARB?$AA@ 10001c70     eglglue.obj
 0001:00000c84       ??_C@_0BE@BMGJDPBK@glGenerateMipmapOES?$AA@ 10001c84     eglglue.obj
 0001:00000c98       ??_C@_0CJ@FPBNJAAI@glGetFramebufferAttachmentParame@ 10001c98     eglglue.obj
 0001:00000cc4       ??_C@_0BN@CEGIKEBP@glFramebufferRenderbufferOES?$AA@ 10001cc4     eglglue.obj
 0001:00000ce4       ??_C@_0BK@IBODAJKF@glFramebufferTexture2DOES?$AA@ 10001ce4     eglglue.obj
 0001:00000d00       ??_C@_0BM@FKHNDAOE@glCheckFramebufferStatusOES?$AA@ 10001d00     eglglue.obj
 0001:00000d1c       ??_C@_0BF@GBILCPIM@glGenFramebuffersOES?$AA@ 10001d1c     eglglue.obj
 0001:00000d34       ??_C@_0BI@DJPGNLDO@glDeleteFramebuffersOES?$AA@ 10001d34     eglglue.obj
 0001:00000d4c       ??_C@_0BF@HIIGGHIK@glBindFramebufferOES?$AA@ 10001d4c     eglglue.obj
 0001:00000d64       ??_C@_0BD@PMGNFKPK@glIsFramebufferOES?$AA@ 10001d64     eglglue.obj
 0001:00000d78       ??_C@_0CA@ODMPPHIE@glGetRenderbufferParameterivOES?$AA@ 10001d78     eglglue.obj
 0001:00000d98       ??_C@_0BJ@OLDCKGHK@glRenderbufferStorageOES?$AA@ 10001d98     eglglue.obj
 0001:00000db4       ??_C@_0BG@EDIBBEEP@glGenRenderbuffersOES?$AA@ 10001db4     eglglue.obj
 0001:00000dcc       ??_C@_0BJ@GGLGLLBL@glDeleteRenderbuffersOES?$AA@ 10001dcc     eglglue.obj
 0001:00000de8       ??_C@_0BG@FPKCPFFN@glBindRenderbufferOES?$AA@ 10001de8     eglglue.obj
 0001:00000e00       ??_C@_0BE@PCDGPFM@glIsRenderbufferOES?$AA@ 10001e00     eglglue.obj
 0001:00000e14       ??_C@_0BB@GPIPACKB@glGetTexGenxvOES?$AA@ 10001e14     eglglue.obj
 0001:00000e28       ??_C@_0BB@FGFDGBEK@glGetTexGenfvOES?$AA@ 10001e28     eglglue.obj
 0001:00000e3c       ??_C@_0BB@KHAFNDJP@glGetTexGenivOES?$AA@ 10001e3c     eglglue.obj
 0001:00000e50       ??_C@_0O@OEFPDKKM@glTexGenxvOES?$AA@ 10001e50     eglglue.obj
 0001:00000e60       ??_C@_0N@DPLLCAOI@glTexGenxOES?$AA@ 10001e60     eglglue.obj
 0001:00000e70       ??_C@_0O@NNIDFJEH@glTexGenfvOES?$AA@ 10001e70     eglglue.obj
 0001:00000e80       ??_C@_0N@OAGLAJAL@glTexGenfOES?$AA@ 10001e80     eglglue.obj
 0001:00000e90       ??_C@_0O@CMNFOLJC@glTexGenivOES?$AA@ 10001e90     eglglue.obj
 0001:00000ea0       ??_C@_0N@GCDLJONK@glTexGeniOES?$AA@ 10001ea0     eglglue.obj
 0001:00000eb0       ??_C@_0BH@FBPJDECF@glBlendFuncSeparateOES?$AA@ 10001eb0     eglglue.obj
 0001:00000ec8       ??_C@_0BL@LJMLCLCI@glBlendEquationSeparateOES?$AA@ 10001ec8     eglglue.obj
 0001:00000ee4       ??_C@_0BD@BBOLNBAI@glBlendEquationOES?$AA@ 10001ee4     eglglue.obj
 0001:00000ef8       ??_C@_0BC@DEKNHIDE@glQueryMatrixxOES?$AA@ 10001ef8     eglglue.obj
 0001:00000f0c       ??_C@_0P@LKNACIFH@glDrawTexxvOES?$AA@ 10001f0c     eglglue.obj
 0001:00000f1c       ??_C@_0P@IDAMELLM@glDrawTexfvOES?$AA@ 10001f1c     eglglue.obj
 0001:00000f2c       ??_C@_0P@HCFKPJGJ@glDrawTexivOES?$AA@ 10001f2c     eglglue.obj
 0001:00000f3c       ??_C@_0P@NABHNIJE@glDrawTexsvOES?$AA@ 10001f3c     eglglue.obj
 0001:00000f4c       ??_C@_0O@GOFANFJA@glDrawTexxOES?$AA@ 10001f4c     eglglue.obj
 0001:00000f5c       ??_C@_0O@LBIAPMHD@glDrawTexfOES?$AA@ 10001f5c     eglglue.obj
 0001:00000f6c       ??_C@_0O@DDNAGLKC@glDrawTexiOES?$AA@ 10001f6c     eglglue.obj
 0001:00000f7c       ??_C@_0O@BJIAOEIB@glDrawTexsOES?$AA@ 10001f7c     eglglue.obj
 0001:00000f8c       ??_C@_0BD@PCEFFFDF@glWeightPointerOES?$AA@ 10001f8c     eglglue.obj
 0001:00000fa0       ??_C@_0BI@BEEEECPN@glMatrixIndexPointerOES?$AA@ 10001fa0     eglglue.obj
 0001:00000fb8       ??_C@_0CE@HEFPEHID@glLoadPaletteFromModelViewMatrix@ 10001fb8     eglglue.obj
 0001:00000fdc       ??_C@_0BK@NDELAMFO@glCurrentPaletteMatrixOES?$AA@ 10001fdc     eglglue.obj
 0001:00000ff8       ??_C@_0BG@PIPFALFL@glPointSizePointerOES?$AA@ 10001ff8     eglglue.obj
 0001:000016dc       ui32NumCombineOpSources    100026dc     fftex.obj
 0001:00001a88       ??_C@_0BA@JNOOKNAN@fftnlshader?4txt?$AA@ 10002a88     fftnlgles.obj
 0001:00001a98       ??_C@_0BB@NNIEEEPA@OpenGL?5ES?9CM?51?41?$AA@ 10002a98     get.obj
 0001:00001aac       ??_C@_0BP@MJBNMJBG@PowerVR?5SGX?5with?5VGP?5emulation?$AA@ 10002aac     get.obj
 0001:00001acc       ??_C@_0BA@HGHHDPMC@PowerVR?5SGX?5540?$AA@ 10002acc     get.obj
 0001:00001adc       ??_C@_0BJ@FGEHHHOH@Imagination?5Technologies?$AA@ 10002adc     get.obj
 0001:00001c64       pszRenderer                10002c64     get.obj
 0001:00002544       ??_C@_0L@CDGAGNFA@KickTAMode?$AA@ 10003544     misc.obj
 0001:00002550       ??_C@_0BA@FMCJLEC@KickTAThreshold?$AA@ 10003550     misc.obj
 0001:00002560       ??_C@_0L@OHKGCBME@EmulateVGP?$AA@ 10003560     misc.obj
 0001:0000256c       ??_C@_0BH@NAIKDGLA@ForceNoExternalZBuffer?$AA@ 1000356c     misc.obj
 0001:00002584       ??_C@_0BE@CONEIBKK@OptimisedValidation?$AA@ 10003584     misc.obj
 0001:00002598       ??_C@_0BE@MLGMBNML@DisableHWNormalBlit?$AA@ 10003598     misc.obj
 0001:000025ac       ??_C@_0BH@EMEDPOLF@DisableHWTextureUpload?$AA@ 100035ac     misc.obj
 0001:000025c4       ??_C@_0BA@ELLICOAA@DisableHWMipGen?$AA@ 100035c4     misc.obj
 0001:000025d4       ??_C@_0P@LPEGOECO@FlushBehaviour?$AA@ 100035d4     misc.obj
 0001:000025e4       ??_C@_0BG@CHMKCCI@EnableStaticPDSVertex?$AA@ 100035e4     misc.obj
 0001:000025fc       ??_C@_0BE@CJIJABHD@EnableStaticMTECopy?$AA@ 100035fc     misc.obj
 0001:00002610       ??_C@_0BP@JBLIJOPK@DisableStaticPDSPixelSAProgram?$AA@ 10003610     misc.obj
 0001:00002630       ??_C@_0BB@FEGFPPJN@DisableUSEASMOPT?$AA@ 10003630     misc.obj
 0001:00002644       ??_C@_0M@HPPFGNFE@DumpShaders?$AA@ 10003644     misc.obj
 0001:00002650       ??_C@_0BI@GMOOJAHB@DefaultVertexBufferSize?$AA@ 10003650     misc.obj
 0001:00002668       ??_C@_0BH@EMCDMDFL@DefaultIndexBufferSize?$AA@ 10003668     misc.obj
 0001:00002680       ??_C@_0BJ@FDELEOJK@DefaultPDSVertBufferSize?$AA@ 10003680     misc.obj
 0001:0000269c       ??_C@_0BP@CGBHEOOJ@DefaultPregenPDSVertBufferSize?$AA@ 1000369c     misc.obj
 0001:000026bc       ??_C@_0BP@CNJFMOH@DefaultPregenMTECopyBufferSize?$AA@ 100036bc     misc.obj
 0001:000026dc       ??_C@_0BF@GMGALNEL@DefaultVDMBufferSize?$AA@ 100036dc     misc.obj
 0001:0000394c       TexFormatABGR8888          1000494c     texformat.obj
 0001:00003958       TexFormatARGB8888          10004958     texformat.obj
 0001:00003964       TexFormatARGB1555          10004964     texformat.obj
 0001:00003970       TexFormatARGB4444          10004970     texformat.obj
 0001:0000397c       TexFormatXBGR8888          1000497c     texformat.obj
 0001:00003988       TexFormatRGB565            10004988     texformat.obj
 0001:00003994       TexFormatAlpha             10004994     texformat.obj
 0001:000039a0       TexFormatLuminance         100049a0     texformat.obj
 0001:000039ac       TexFormatLuminanceAlpha    100049ac     texformat.obj
 0001:000039b8       TexFormatPVRTC2RGB         100049b8     texformat.obj
 0001:000039c4       TexFormatPVRTC4RGB         100049c4     texformat.obj
 0001:000039d0       TexFormatPVRTC2RGBA        100049d0     texformat.obj
 0001:000039dc       TexFormatPVRTC4RGBA        100049dc     texformat.obj
 0001:000039e8       TexFormatPVRTCII2RGB       100049e8     texformat.obj
 0001:000039f4       TexFormatPVRTCII4RGB       100049f4     texformat.obj
 0001:00003a00       TexFormatPVRTCII2RGBA      10004a00     texformat.obj
 0001:00003a0c       TexFormatPVRTCII4RGBA      10004a0c     texformat.obj
 0001:00003a18       TexFormatETC1RGB8          10004a18     texformat.obj
 0001:00003a24       TexFormatUYVY              10004a24     texformat.obj
 0001:00003a30       TexFormatYUYV              10004a30     texformat.obj
 0001:00003a3c       TexFormatYUV420            10004a3c     texformat.obj
 0001:00003e80       ??_C@_0BA@ELCMJBIB@BufferDevice?$CFd?6?$AA@ 10004e80     texstream.obj
 0001:00004410       ??_C@_0BD@MFPFLDAC@Assember?5Error?3?$CFs?6?$AA@ 10005410     useasmgles.obj
 0001:00004990       CopyData                   10005990     vertex.obj
 0001:00004a00       MemCopyData                10005a00     vertex.obj
 0001:00004a70       CopyDataShortAligned       10005a70     vertex.obj
 0001:00004ae0       CopyDataByteAligned        10005ae0     vertex.obj
 0001:000052d0       ??_C@_0FJ@EGGFMBDH@H?3?2WINCE600?2PLATFORM?2SMDKV210?2SR@ 100062d0     vpreg.obj
 0001:0000532c       ??_C@_0BI@ONMJPNJJ@Load?5the?5?$CFs?5from?5memory?$AA@ 1000632c     vpreg.obj
 0001:000054b0       ??_C@_0FA@KPBPOIEA@Instruction?5below?5can?8t?5have?5exi@ 100064b0     vpinst.obj
 0001:00005500       ??_C@_0FK@LAKHAAEK@H?3?2WINCE600?2PLATFORM?2SMDKV210?2SR@ 10006500     vpinst.obj
 0001:0000555c       ??_C@_0DP@JOJOOGOB@Possible?5optimisation?$DP?5?9?5Switch?5@ 1000655c     vpinst.obj
 0001:00005890       ??_C@_0FN@ICNMGIJF@H?3?2WINCE600?2PLATFORM?2SMDKV210?2SR@ 10006890     vpcodegen.obj
 0001:000058f0       ??_C@_0BH@JPOGKGMJ@VGP?5Binary?5instruction?$AA@ 100068f0     vpcodegen.obj
 0001:00005908       ??_C@_08EOPPEGAM@HACK?9MOV?$AA@ 10006908     vpcodegen.obj
 0001:00005914       ??_C@_0L@JPHNAFAM@TEX?9INIT?9z?$AA@ 10006914     vpcodegen.obj
 0001:00005920       ??_C@_0L@CKNDHLEB@TEX?9INIT?9w?$AA@ 10006920     vpcodegen.obj
 0001:0000592c       ??_C@_03MLIHNEFJ@LOG?$AA@  1000692c     vpcodegen.obj
 0001:00005930       ??_C@_03KKGFKKLA@EXP?$AA@  10006930     vpcodegen.obj
 0001:00005934       ??_C@_0BA@IAHNLBID@AMV?9MAD?3?5n?$CK4?5?$CL0?$AA@ 10006934     vpcodegen.obj
 0001:00005944       ??_C@_0BD@JGCFGINK@convert?5to?5integer?$AA@ 10006944     vpcodegen.obj
 0001:00005958       ??_C@_03NEKIMBBK@FRC?$AA@  10006958     vpcodegen.obj
 0001:0000595c       ??_C@_0P@POCLEHCC@DST?3?5dst?4x?5?$DN?51?$AA@ 1000695c     vpcodegen.obj
 0001:0000596c       ??_C@_0P@BEMMGAML@DST?3?5dst?4y?5?$DN?5x?$AA@ 1000696c     vpcodegen.obj
 0001:0000597c       ??_C@_0BB@GAGBCLDJ@DST?3?5dst?4z?5?$DN?5x?$FO2?$AA@ 1000697c     vpcodegen.obj
 0001:00005990       ??_C@_0BB@ECNNIMLH@DST?3?5dst?4w?5?$DN?51?1x?$AA@ 10006990     vpcodegen.obj
 0001:000059a4       ??_C@_0BF@BFDNMAON@SMOA?3?5disable?5mirror?$AA@ 100069a4     vpcodegen.obj
 0001:000059bc       ??_C@_0DK@JELNICIB@LIT?3?5dst?4z?5?$DN?5?$CItemp?4x?5?$DO?50?$CJ?5?$DP?5exp?5@ 100069bc     vpcodegen.obj
 0001:000059f8       ??_C@_0BG@MMEAPGLC@SMRI?3?5set?5clamp?5range?$AA@ 100069f8     vpcodegen.obj
 0001:00005a10       ??_C@_0BH@FCNFMMCM@temp?4w?5?5?$CK?5?$CIlog?5temp?4y?$CJ?$AA@ 10006a10     vpcodegen.obj
 0001:00005a28       ??_C@_0BE@FBKDKAGD@SMOA?3?5enable?5mirror?$AA@ 10006a28     vpcodegen.obj
 0001:00005a3c       ??_C@_0BD@OBPKCBJJ@copy?5?5src1?5to?5temp?$AA@ 10006a3c     vpcodegen.obj
 0001:00005a50       ??_C@_0BN@IPMLOEJE@LIT?3?5temp?4x?5?$DM?50?5?$DP?50?5?3?5temp?4x?$AA@ 10006a50     vpcodegen.obj
 0001:00005a70       ??_C@_0BN@EBDCFFIN@LIT?3?5temp?4y?5?$DM?50?5?$DP?50?5?3?5temp?4y?$AA@ 10006a70     vpcodegen.obj
 0001:00005a90       ??_C@_0P@IFCHGNFC@LIT?3?5dst?4x?5?$DN?51?$AA@ 10006a90     vpcodegen.obj
 0001:00005aa0       ??_C@_0BE@KAEFBPJN@LIT?3?5dst?4y?5?$DN?5temp?4x?$AA@ 10006aa0     vpcodegen.obj
 0001:00005ab4       ??_C@_0P@HEHBNPIH@LIT?3?5dst?4w?5?$DN?51?$AA@ 10006ab4     vpcodegen.obj
 0001:00005ac3       ??_C@_00CNPNBAHC@?$AA@     10006ac3     vpcodegen.obj
 0001:00005ac4       ??_C@_0L@KJIDELMO@log?5temp?4y?$AA@ 10006ac4     vpcodegen.obj
 0001:00005ad0       ??_C@_0CI@DHCLHGJ@Test?5if?5src1?4x?5?$DO?$DN?5src2?4x?5per?5com@ 10006ad0     vpcodegen.obj
 0001:00005af8       ??_C@_0BO@HHMDBPCO@SGE?3?5src1?4x?5?$DO?$DN?5src2?4x?5?$DP?51?5?3?50?$AA@ 10006af8     vpcodegen.obj
 0001:00005b18       ??_C@_0CI@OKFIGHGL@Test?5if?5src1?4y?5?$DO?$DN?5src2?4y?5per?5com@ 10006b18     vpcodegen.obj
 0001:00005b40       ??_C@_0BO@PNGGEPFG@SGE?3?5src1?4y?5?$DO?$DN?5src2?4y?5?$DP?51?5?3?50?$AA@ 10006b40     vpcodegen.obj
 0001:00005b60       ??_C@_0CI@KFGBBCM@Test?5if?5src1?4z?5?$DO?$DN?5src2?4z?5per?5com@ 10006b60     vpcodegen.obj
 0001:00005b88       ??_C@_0BO@LJPILJJP@SGE?3?5src1?4z?5?$DO?$DN?5src2?4z?5?$DP?51?5?3?50?$AA@ 10006b88     vpcodegen.obj
 0001:00005ba8       ??_C@_0CI@NFKHBELA@Test?5if?5src1?4w?5?$DO?$DN?5src2?4w?5per?5com@ 10006ba8     vpcodegen.obj
 0001:00005bd0       ??_C@_0BO@PKFHDEIC@SGE?3?5src1?4w?5?$DO?$DN?5src2?4w?5?$DP?51?5?3?50?$AA@ 10006bd0     vpcodegen.obj
 0001:00005bf0       ??_C@_0BB@PHLKCDKB@Set?5?5dst?5to?5zero?$AA@ 10006bf0     vpcodegen.obj
 0001:00005c04       ??_C@_0CH@GFMEMLCG@Test?5if?5src1?4x?5?$DM?5src2?4x?5per?5comp@ 10006c04     vpcodegen.obj
 0001:00005c2c       ??_C@_0BN@DGDGFNLK@SLT?3?5src1?4x?5?$DM?5src2?4x?5?$DP?51?5?3?50?$AA@ 10006c2c     vpcodegen.obj
 0001:00005c4c       ??_C@_0CH@FHPKGPC@Test?5if?5src1?4y?5?$DM?5src2?4y?5per?5comp@ 10006c4c     vpcodegen.obj
 0001:00005c74       ??_C@_0BN@OBGLGNM@SLT?3?5src1?4y?5?$DM?5src2?4y?5?$DP?51?5?3?50?$AA@ 10006c74     vpcodegen.obj
 0001:00005c94       ??_C@_0CH@KELCBAIO@Test?5if?5src1?4z?5?$DM?5src2?4z?5per?5comp@ 10006c94     vpcodegen.obj
 0001:00005cbc       ??_C@_0BN@EGHHILHG@SLT?3?5src1?4z?5?$DM?5src2?4z?5?$DP?51?5?3?50?$AA@ 10006cbc     vpcodegen.obj
 0001:00005cdc       ??_C@_0CH@COKMKOGJ@Test?5if?5src1?4w?5?$DM?5src2?4w?5per?5comp@ 10006cdc     vpcodegen.obj
 0001:00005d04       ??_C@_0BN@IEKCJAPJ@SLT?3?5src1?4w?5?$DM?5src2?4w?5?$DP?51?5?3?50?$AA@ 10006d04     vpcodegen.obj
 0001:00005d24       ??_C@_03LEPPJAKI@MAX?$AA@  10006d24     vpcodegen.obj
 0001:00005d28       ??_C@_03KGHEHEMH@MIN?$AA@  10006d28     vpcodegen.obj
 0001:00005d2c       ??_C@_03BNFLDCMO@DP4?$AA@  10006d2c     vpcodegen.obj
 0001:00005d30       ??_C@_03FCBKKEAJ@DP3?$AA@  10006d30     vpcodegen.obj
 0001:00005d34       ??_C@_0N@LKMHMKM@RSQ?5of?5src?4w?$AA@ 10006d34     vpcodegen.obj
 0001:00005d44       ??_C@_0N@MGDKEOJA@RCP?5of?5src?4w?$AA@ 10006d44     vpcodegen.obj
 0001:00005d54       ??_C@_03IBHOEMFB@MUL?$AA@  10006d54     vpcodegen.obj
 0001:00005d58       ??_C@_03FCIIMNPF@MAD?$AA@  10006d58     vpcodegen.obj
 0001:00005d5c       ??_C@_03BOJFLAKG@ADD?$AA@  10006d5c     vpcodegen.obj
 0001:00005d60       ??_C@_03CAOCJACM@MOV?$AA@  10006d60     vpcodegen.obj
 0001:00005d64       ??_C@_07KNMMKPGG@SWIZZLE?$AA@ 10006d64     vpcodegen.obj
 0001:00005d6c       ??_C@_0BB@MPFGHBLJ@SWIZZLE?5DISABLED?$AA@ 10006d6c     vpcodegen.obj
 0001:00005d80       ??_C@_0BI@KIEKJNPB@VP?3?5Emit?5Vertex?5and?5End?$AA@ 10006d80     vpcodegen.obj
 0001:00005f00       ??_C@_0N@GAOADMDM@vpshader?4txt?$AA@ 10006f00     vpgles.obj
 0001:00006f48       ??_C@_0EL@CEJMDIFD@Branch?5destination?5is?5out?5of?5ran@ 10007f48     useasm:useasm.obj
 0001:00006f98       ??_C@_0EM@IGAKCAGC@Branch?5destination?5is?5out?5of?5ran@ 10007f98     useasm:useasm.obj
 0001:00006fe8       ??_C@_0JC@CGJAIGHK@The?5destination?5label?5for?5a?5bran@ 10007fe8     useasm:useasm.obj
 0001:0000707c       ??_C@_0DK@NIFCHDCD@A?5swizzle?5is?5invalid?5for?5argumen@ 1000807c     useasm:useasm.obj
 0001:000070b8       ??_C@_0EC@FENPMIAM@The?5modifiers?5?4flt32?0?5?4flt16?0?5?4c@ 100080b8     useasm:useasm.obj
 0001:000070fc       ??_C@_0DE@EJENDBGB@?4u8?5is?5invalid?5for?5argument?5?$CFd?5f@ 100080fc     useasm:useasm.obj
 0001:00007130       ??_C@_0DF@KNCENLBB@?4c10?5is?5invalid?5for?5argument?5?$CFd?5@ 10008130     useasm:useasm.obj
 0001:00007168       ??_C@_0DH@LCLAOIMP@?4flt16?5is?5invalid?5for?5argument?5?$CF@ 10008168     useasm:useasm.obj
 0001:000071a0       ??_C@_0DH@IAOLGEKP@?4flt32?5is?5invalid?5for?5argument?5?$CF@ 100081a0     useasm:useasm.obj
 0001:000071d8       ??_C@_0EC@LIBCAICE@Disable?5writeback?5is?5invalid?5for@ 100081d8     useasm:useasm.obj
 0001:0000721c       ??_C@_0DG@MICEFMNE@?4comp?5is?5invalid?5for?5argument?5?$CFd@ 1000821c     useasm:useasm.obj
 0001:00007254       ??_C@_0DH@BJDJAOJN@?4alpha?5is?5invalid?5for?5argument?5?$CF@ 10008254     useasm:useasm.obj
 0001:0000728c       ??_C@_0DG@NIHNAGBL@?4high?5is?5invalid?5for?5argument?5?$CFd@ 1000828c     useasm:useasm.obj
 0001:000072c4       ??_C@_0DF@HFACOLNL@?4low?5is?5invalid?5for?5argument?5?$CFd?5@ 100082c4     useasm:useasm.obj
 0001:000072fc       ??_C@_0DI@BMAPILCJ@?4invert?5is?5invalid?5for?5argument?5@ 100082fc     useasm:useasm.obj
 0001:00007334       ??_C@_0DK@PJAHFLKI@A?5bytemask?5is?5invalid?5for?5argume@ 10008334     useasm:useasm.obj
 0001:00007370       ??_C@_0EC@IJJBJBBP@A?5component?5select?5is?5invalid?5fo@ 10008370     useasm:useasm.obj
 0001:000073b4       ??_C@_0DE@NBGIMLFH@?4abs?5is?5invalid?5for?5argument?5?$CFd?5@ 100083b4     useasm:useasm.obj
 0001:000073e8       ??_C@_0DE@MPDILDBH@?4neg?5is?5invalid?5for?5argument?5?$CFd?5@ 100083e8     useasm:useasm.obj
 0001:0000741c       ??_C@_0CG@HDBABLGF@?4minp?5is?5invalid?5for?5this?5instru@ 1000841c     useasm:useasm.obj
 0001:00007444       ??_C@_0CG@JNEGBJAJ@?4irsd?5is?5invalid?5for?5this?5instru@ 10008444     useasm:useasm.obj
 0001:0000746c       ??_C@_0CH@MOFKMNFF@?4pwait?5is?5invalid?5for?5this?5instr@ 1000846c     useasm:useasm.obj
 0001:00007494       ??_C@_0CI@FJKAAMII@?4noread?5is?5invalid?5for?5this?5inst@ 10008494     useasm:useasm.obj
 0001:000074bc       ??_C@_0CM@BKAEHGEJ@?4dm_nomatch?5is?5invalid?5for?5this?5@ 100084bc     useasm:useasm.obj
 0001:000074e8       ??_C@_0CI@LAPAEMDG@?4global?5is?5invalid?5for?5this?5inst@ 100084e8     useasm:useasm.obj
 0001:00007510       ??_C@_0CI@JBBFIBPL@?4gpiext?5is?5invalid?5for?5this?5inst@ 10008510     useasm:useasm.obj
 0001:00007538       ??_C@_0CK@DEEAJLON@?4bypassl1?5is?5invalid?5for?5this?5in@ 10008538     useasm:useasm.obj
 0001:00007564       ??_C@_0CF@EHCJCPGO@?4cut?5is?5invalid?5for?5this?5instruc@ 10008564     useasm:useasm.obj
 0001:0000758c       ??_C@_0CL@OGDOHFNH@?4threepart?5is?5invalid?5for?5this?5i@ 1000858c     useasm:useasm.obj
 0001:000075b8       ??_C@_0CJ@FCBBHHDD@?4twopart?5is?5invalid?5for?5this?5ins@ 100085b8     useasm:useasm.obj
 0001:000075e4       ??_C@_0CJ@GOGNFJGL@?4trigger?5is?5invalid?5for?5this?5ins@ 100085e4     useasm:useasm.obj
 0001:00007610       ??_C@_0CJ@GIKGIFLP@?4syncend?5is?5invalid?5for?5this?5ins@ 10008610     useasm:useasm.obj
 0001:0000763c       ??_C@_0CG@IHPDGLHB@?4sinf?5is?5invalid?5for?5this?5instru@ 1000863c     useasm:useasm.obj
 0001:00007664       ??_C@_0CF@NKHJPKHH@?4rsd?5is?5invalid?5for?5this?5instruc@ 10008664     useasm:useasm.obj
 0001:0000768c       ??_C@_0CI@NKNMDDOG@?4pcff16?5is?5invalid?5for?5this?5inst@ 1000868c     useasm:useasm.obj
 0001:000076b4       ??_C@_0CF@CNBHLDDL@?4pcf?5is?5invalid?5for?5this?5instruc@ 100086b4     useasm:useasm.obj
 0001:000076dc       ??_C@_0CG@KBDEHIIG@?4incs?5is?5invalid?5for?5this?5instru@ 100086dc     useasm:useasm.obj
 0001:00007704       ??_C@_0CF@HDBKEIDN@?4tog?5is?5invalid?5for?5this?5instruc@ 10008704     useasm:useasm.obj
 0001:0000772c       ??_C@_0CF@CPPKEJPF@?4c10?5is?5invalid?5for?5this?5instruc@ 1000872c     useasm:useasm.obj
 0001:00007754       ??_C@_0CH@JJCJAFEG@?4tpres?5is?5invalid?5for?5this?5instr@ 10008754     useasm:useasm.obj
 0001:0000777c       ??_C@_0CF@KOMKFHLA@?4i10?5is?5invalid?5for?5this?5instruc@ 1000877c     useasm:useasm.obj
 0001:000077a4       ??_C@_0CF@KACIFBOK@?4flt?5is?5invalid?5for?5this?5instruc@ 100087a4     useasm:useasm.obj
 0001:000077cc       ??_C@_0CF@KDIDNMAN@?4i32?5is?5invalid?5for?5this?5instruc@ 100087cc     useasm:useasm.obj
 0001:000077f4       ??_C@_0CF@HFMHLBAE@?4i16?5is?5invalid?5for?5this?5instruc@ 100087f4     useasm:useasm.obj
 0001:0000781c       ??_C@_0CF@GBAIFKNL@?4sat?5is?5invalid?5for?5this?5instruc@ 1000881c     useasm:useasm.obj
 0001:00007844       ??_C@_0DE@KONNOGII@pre?9?1post?9increment?5is?5invalid?5f@ 10008844     useasm:useasm.obj
 0001:00007878       ??_C@_0CH@MJONMLMP@?4scale?5is?5invalid?5for?5this?5instr@ 10008878     useasm:useasm.obj
 0001:000078a0       ??_C@_0CH@BGLMLOBA@?4taske?5is?5invalid?5for?5this?5instr@ 100088a0     useasm:useasm.obj
 0001:000078c8       ??_C@_0CH@OIAHEBAH@?4tasks?5is?5invalid?5for?5this?5instr@ 100088c8     useasm:useasm.obj
 0001:000078f0       ??_C@_0CI@JKBHNFPL@?4fcfill?5is?5invalid?5for?5this?5inst@ 100088f0     useasm:useasm.obj
 0001:00007918       ??_C@_0CJ@POAKEGNN@?4bpcache?5is?5invalid?5for?5this?5ins@ 10008918     useasm:useasm.obj
 0001:00007944       ??_C@_0CK@NHGHHGDI@?4onceonly?5is?5invalid?5for?5this?5in@ 10008944     useasm:useasm.obj
 0001:00007970       ??_C@_0CH@OGBNJBLO@?4freep?5is?5invalid?5for?5this?5instr@ 10008970     useasm:useasm.obj
 0001:00007998       ??_C@_0CH@NCCAPODE@?4fetch?5is?5invalid?5for?5this?5instr@ 10008998     useasm:useasm.obj
 0001:000079c0       ??_C@_0CL@BFLFDPDE@testenable?5is?5invalid?5for?5this?5i@ 100089c0     useasm:useasm.obj
 0001:000079ec       ??_C@_0CM@GBLJGDF@rangeneable?5is?5invalid?5for?5this?5@ 100089ec     useasm:useasm.obj
 0001:00007a18       ??_C@_0CO@LDDPCEIK@postincrement?5is?5invalid?5for?5thi@ 10008a18     useasm:useasm.obj
 0001:00007a48       ??_C@_0CN@ILKEEOL@preincrement?5is?5invalid?5for?5this@ 10008a48     useasm:useasm.obj
 0001:00007a78       ??_C@_0CH@PGFJCIMI@?4flt16?5is?5invalid?5for?5this?5instr@ 10008a78     useasm:useasm.obj
 0001:00007aa0       ??_C@_0DD@MCGMIGNN@This?5instruction?5can?8t?5be?5part?5o@ 10008aa0     useasm:useasm.obj
 0001:00007ad4       ??_C@_0CJ@OKDELEHB@?4renable?5is?5invalid?5for?5this?5ins@ 10008ad4     useasm:useasm.obj
 0001:00007b00       ??_C@_0CF@FIFBOHH@?4abs?5is?5invalid?5for?5this?5instruc@ 10008b00     useasm:useasm.obj
 0001:00007b28       ??_C@_0CF@KMGKJBBN@?4mon?5is?5invalid?5for?5this?5instruc@ 10008b28     useasm:useasm.obj
 0001:00007b50       ??_C@_0CG@HGFIGOGH@?4mask?5is?5invalid?5for?5this?5instru@ 10008b50     useasm:useasm.obj
 0001:00007b78       ??_C@_0CJ@BJIFKGIO@?4partial?5is?5invalid?5for?5this?5ins@ 10008b78     useasm:useasm.obj
 0001:00007ba4       ??_C@_0CK@IEFIOMMP@?4savelink?5is?5invalid?5for?5this?5in@ 10008ba4     useasm:useasm.obj
 0001:00007bd0       ??_C@_0CH@EIPKEMIK@?4synce?5is?5invalid?5for?5this?5instr@ 10008bd0     useasm:useasm.obj
 0001:00007bf8       ??_C@_0CF@KFDDBKGG@?4end?5is?5invalid?5for?5this?5instruc@ 10008bf8     useasm:useasm.obj
 0001:00007c20       ??_C@_0CM@ONJAAFFM@A?5predicate?5is?5invalid?5for?5this?5@ 10008c20     useasm:useasm.obj
 0001:00007c4c       ??_C@_0CO@HKFMBEAO@A?5repeat?5mask?5is?5invalid?5for?5thi@ 10008c4c     useasm:useasm.obj
 0001:00007c7c       ??_C@_0CI@BKLOOKDP@?4repeat?5is?5invalid?5for?5this?5inst@ 10008c7c     useasm:useasm.obj
 0001:00007ca4       ??_C@_0CJ@JOPLONOF@?4nosched?5is?5invalid?5for?5this?5ins@ 10008ca4     useasm:useasm.obj
 0001:00007cd0       ??_C@_0CH@LGEBLDJN@?4syncs?5is?5invalid?5for?5this?5instr@ 10008cd0     useasm:useasm.obj
 0001:00007cf8       ??_C@_0CE@LNKCCLIM@?4i8?5is?5invalid?5for?5this?5instruct@ 10008cf8     useasm:useasm.obj
 0001:00007d1c       ??_C@_0CJ@MMEFPBHM@?4skipinv?5is?5invalid?5for?5this?5ins@ 10008d1c     useasm:useasm.obj
 0001:00007d48       ??_C@_07MALOAKCI@invalid?$AA@ 10008d48     useasm:useasm.obj
 0001:00007d50       ??_C@_0DP@KIFGKPIF@Offset?5into?5indexed?5register?5ban@ 10008d50     useasm:useasm.obj
 0001:00007d90       ??_C@_0CC@LJGIDMA@Register?5type?5?$CFs?5is?5not?5indexabl@ 10008d90     useasm:useasm.obj
 0001:00007db4       ??_C@_0BO@NAKOKMPE@?$CFs?5is?5not?5a?5valid?5destination?$AA@ 10008db4     useasm:useasm.obj
 0001:00007dd4       ??_C@_0CK@FBILJLCJ@Destination?5must?5be?5a?5modifiable@ 10008dd4     useasm:useasm.obj
 0001:00007e00       ??_C@_0CK@JGFFOFI@Invalid?5internal?5register?5specif@ 10008e00     useasm:useasm.obj
 0001:00007e2c       ??_C@_0CO@LBPJMKJE@Invalid?5fp?5internal?5register?5spe@ 10008e2c     useasm:useasm.obj
 0001:00007e5c       ??_C@_0CI@BLCMIAIL@Invalid?5global?5register?5specifie@ 10008e5c     useasm:useasm.obj
 0001:00007e84       ??_C@_0CH@OHEKEBML@Invalid?5index?5mask?5specified?5?$CIwa@ 10008e84     useasm:useasm.obj
 0001:00007eac       ??_C@_0DG@PBPNOJGF@Invalid?5secondary?5attribute?5regi@ 10008eac     useasm:useasm.obj
 0001:00007ee4       ??_C@_0DB@FPFAHPGJ@Destination?5type?5is?5invalid?5for?5@ 10008ee4     useasm:useasm.obj
 0001:00007f18       ??_C@_0DE@LFLBECCD@Invalid?5primary?5attribute?5regist@ 10008f18     useasm:useasm.obj
 0001:00007f4c       ??_C@_0CI@JCGMLMHK@Invalid?5output?5register?5specifie@ 10008f4c     useasm:useasm.obj
 0001:00007f74       ??_C@_0CL@BINLLFEH@Invalid?5temporary?5register?5speci@ 10008f74     useasm:useasm.obj
 0001:00007fa0       ??_C@_0CP@DIKNGJCD@Source?50?5type?5can?8t?5be?5?$CFs?5for?5th@ 10008fa0     useasm:useasm.obj
 0001:00007fd0       ??_C@_0BK@EAPIEFOL@Source?50?5type?5can?8t?5be?5?$CFs?$AA@ 10008fd0     useasm:useasm.obj
 0001:00007fec       ??_C@_0BK@DOBHJKGK@Source?50?5can?8t?5be?5indexed?$AA@ 10008fec     useasm:useasm.obj
 0001:00008008       ??_C@_0DG@NFHFDDMG@?$CFs?5immediate?5value?5is?5too?5small?5@ 10009008     useasm:useasm.obj
 0001:00008040       ??_C@_0DF@HLDFHJJG@?$CFs?5immediate?5value?5is?5too?5large?5@ 10009040     useasm:useasm.obj
 0001:00008078       ??_C@_0DI@KIGIDHNA@Indexed?5sources?5are?5not?5availabl@ 10009078     useasm:useasm.obj
 0001:000080b0       ??_C@_0BK@JHBKMFLD@Source?51?5type?5can?8t?5be?5?$CFs?$AA@ 100090b0     useasm:useasm.obj
 0001:000080cc       ??_C@_0DL@PKMEEOIP@Source?51?5immediate?5value?5is?5too?5@ 100090cc     useasm:useasm.obj
 0001:00008108       ??_C@_08IPCCDMEN@Source?51?$AA@ 10009108     useasm:useasm.obj
 0001:00008114       ??_C@_0CK@INEOLDIC@Invalid?5constant?5register?5specif@ 10009114     useasm:useasm.obj
 0001:00008140       ??_C@_0HF@OJAOJKHK@Sequence?5number?5?$CIg?$CFd?$CJ?0?5edge?5mask@ 10009140     useasm:useasm.obj
 0001:000081b8       ??_C@_0DK@LCPGEMNK@Task?5queue?5data?5?$CIg?$CFd?5to?5g?$CFd?$CJ?5can@ 100091b8     useasm:useasm.obj
 0001:000081f4       ??_C@_0CP@JHOJPLGE@Source?51?5type?5can?8t?5be?5?$CFs?5for?5th@ 100091f4     useasm:useasm.obj
 0001:00008224       ??_C@_0BK@DEEMEDBK@Source?52?5type?5can?8t?5be?5?$CFs?$AA@ 10009224     useasm:useasm.obj
 0001:00008240       ??_C@_0DL@EAJBEKJI@Source?52?5immediate?5value?5is?5too?5@ 10009240     useasm:useasm.obj
 0001:0000827c       ??_C@_08KEAPGPIO@Source?52?$AA@ 1000927c     useasm:useasm.obj
 0001:00008288       ??_C@_0CP@LNFFELOM@Source?52?5type?5can?8t?5be?5?$CFs?5for?5th@ 10009288     useasm:useasm.obj
 0001:000082b8       ??_C@_0CM@IBHBOODC@Invalid?5predicate?5type?5for?5this?5@ 100092b8     useasm:useasm.obj
 0001:000082e4       ??_C@_0DN@GHBJDHKE@The?5third?5argument?5to?5dot3?1dot4?5@ 100092e4     useasm:useasm.obj
 0001:00008324       ??_C@_0DH@BBGJEJBC@No?5flags?5are?5valid?5for?5the?5third@ 10009324     useasm:useasm.obj
 0001:00008360       ??_C@_0EE@JPJEDBPB@The?5third?5argument?5to?5dot3?1dot4?5@ 10009360     useasm:useasm.obj
 0001:000083a4       ??_C@_0DP@MPNPCIOH@The?5second?5argument?5to?5dot3?1dot4@ 100093a4     useasm:useasm.obj
 0001:000083e4       ??_C@_0DI@NLNHCCFG@No?5flags?5are?5valid?5for?5the?5secon@ 100093e4     useasm:useasm.obj
 0001:00008420       ??_C@_0EF@EFCBABKE@The?5second?5argument?5to?5dot3?1dot4@ 10009420     useasm:useasm.obj
 0001:00008468       ??_C@_0DJ@JGDEEONP@Invalid?5integer?5source?5for?5the?5t@ 10009468     useasm:useasm.obj
 0001:000084a8       ??_C@_0EE@ELFDABMP@Only?5the?5complement?5flag?5is?5vali@ 100094a8     useasm:useasm.obj
 0001:000084f0       ??_C@_0EC@DANPAEGJ@The?5third?5argument?5to?5aintrp1?5mu@ 100094f0     useasm:useasm.obj
 0001:00008534       ??_C@_0DK@OPCNMALF@Invalid?5integer?5source?5for?5the?5s@ 10009534     useasm:useasm.obj
 0001:00008570       ??_C@_0DG@NPKDEALG@No?5flags?5are?5valid?5for?5the?5secon@ 10009570     useasm:useasm.obj
 0001:000085a8       ??_C@_0ED@NIBLILEL@The?5second?5argument?5to?5aintrp1?5m@ 100095a8     useasm:useasm.obj
 0001:000085ec       ??_C@_0CM@NAFINKIH@The?5fifth?5argument?5to?5aadd?1asub?5@ 100095ec     useasm:useasm.obj
 0001:00008618       ??_C@_0DH@LBMFOABC@No?5flags?5are?5valid?5for?5the?5fifth@ 10009618     useasm:useasm.obj
 0001:00008650       ??_C@_0EE@NHDHBHPH@The?5fifth?5argument?5to?5aadd?1asub?5@ 10009650     useasm:useasm.obj
 0001:00008698       ??_C@_0EH@BNLGGDIJ@Only?5the?5complement?5flag?5is?5vali@ 10009698     useasm:useasm.obj
 0001:000086e0       ??_C@_0EF@BHNJGLAO@The?5fourth?5argument?5to?5aadd?1asub@ 100096e0     useasm:useasm.obj
 0001:00008728       ??_C@_0CM@LAIDNOIF@The?5third?5argument?5to?5aadd?1asub?5@ 10009728     useasm:useasm.obj
 0001:00008758       ??_C@_0EG@KPNPAEGJ@Only?5the?5complement?5flag?5is?5vali@ 10009758     useasm:useasm.obj
 0001:000087a0       ??_C@_0EE@HCICJMII@The?5third?5argument?5to?5aadd?1asub?5@ 100097a0     useasm:useasm.obj
 0001:000087e8       ??_C@_0FM@FCNEOKCI@Invalid?5choice?5for?5the?5second?5ar@ 100097e8     useasm:useasm.obj
 0001:00008848       ??_C@_0EH@COHNMHNB@Only?5the?5complement?5flag?5is?5vali@ 10009848     useasm:useasm.obj
 0001:00008890       ??_C@_0EF@KIDHKMNN@The?5second?5argument?5to?5aadd?1asub@ 10009890     useasm:useasm.obj
 0001:000088d8       ??_C@_0DO@NPGGCMGL@The?5first?5argument?5to?5aadd?1asub?5@ 100098d8     useasm:useasm.obj
 0001:00008918       ??_C@_0CN@JFFLIFPF@An?5integer?5source?5selection?5is?5n@ 10009918     useasm:useasm.obj
 0001:00008948       ??_C@_0DH@DLDDAMMA@No?5flags?5are?5valid?5for?5the?5first@ 10009948     useasm:useasm.obj
 0001:00008980       ??_C@_0EE@BEBPNCHP@The?5first?5argument?5to?5aadd?1asub?5@ 10009980     useasm:useasm.obj
 0001:000089c4       ??_C@_0CN@IACABJMC@Coissued?5instruction?5with?5no?5alp@ 100099c4     useasm:useasm.obj
 0001:000089f4       ??_C@_0BP@IIAMCHDC@Integer?5dot4?5can?8t?5be?5coissued?$AA@ 100099f4     useasm:useasm.obj
 0001:00008a14       ??_C@_0DF@OBCJJOLL@Maximum?5repeat?5count?5on?5an?5integ@ 10009a14     useasm:useasm.obj
 0001:00008a50       ??_C@_0EN@JPNNFBOP@Only?5?4bytemask1111?5is?5supported?5@ 10009a50     useasm:useasm.obj
 0001:00008aa0       ??_C@_0FG@MFNCNONI@Only?5?4bytemask1111?5is?5supported?5@ 10009aa0     useasm:useasm.obj
 0001:00008af8       ??_C@_0DM@GCKABEIE@Conditional?5code?5update?5isn?8t?5av@ 10009af8     useasm:useasm.obj
 0001:00008b38       ??_C@_0EP@POLKDPLI@For?5a?5test?5instruction?5with?5a?5re@ 10009b38     useasm:useasm.obj
 0001:00008b88       ??_C@_0EC@NOAGCNPB@A?5repeated?5dotproduct?5with?5test?5@ 10009b88     useasm:useasm.obj
 0001:00008bcc       ??_C@_0DO@IKLPLKIL@A?5repeated?5test?5instruction?5isn?8@ 10009bcc     useasm:useasm.obj
 0001:00008c0c       ??_C@_0DE@KBHBIIMG@The?5maximum?5repeat?5count?5for?5thi@ 10009c0c     useasm:useasm.obj
 0001:00008c40       ??_C@_0DB@JAOCBPNH@A?5repeat?5count?5is?5not?5valid?5for?5@ 10009c40     useasm:useasm.obj
 0001:00008c74       ??_C@_0DA@INBPMMOK@A?5repeat?5mask?5is?5not?5valid?5for?5t@ 10009c74     useasm:useasm.obj
 0001:00008ca8       ??_C@_0HE@BDIBHBCH@For?5?$CFs?5with?5test?5the?5type?5of?5sou@ 10009ca8     useasm:useasm.obj
 0001:00008d1c       ??_C@_0CM@MLIIJFEL@The?5maximum?5predicate?5register?5n@ 10009d1c     useasm:useasm.obj
 0001:00008d48       ??_C@_0CG@GNGAJDLD@Predicate?5registers?5are?5not?5inde@ 10009d48     useasm:useasm.obj
 0001:00008d70       ??_C@_0EL@MGFIGPBH@The?5second?5destination?5for?5a?5tes@ 10009d70     useasm:useasm.obj
 0001:00008dbc       ??_C@_0DM@JKJAHMJO@No?5flags?5are?5valid?5for?5the?5predi@ 10009dbc     useasm:useasm.obj
 0001:00008df8       ??_C@_0BH@CFEGILC@Unknown?5test?5mask?5type?$AA@ 10009df8     useasm:useasm.obj
 0001:00008e10       ??_C@_0BP@LBJMFOHM@Unknown?5channel?5combine?5option?$AA@ 10009e10     useasm:useasm.obj
 0001:00008e30       ??_C@_0CO@KFAIKBA@?4cperchan?5isn?8t?5supported?5on?5thi@ 10009e30     useasm:useasm.obj
 0001:00008e60       ??_C@_0DL@CIAFLBE@Partial?5modifier?5is?5only?5availab@ 10009e60     useasm:useasm.obj
 0001:00008ea0       ??_C@_0EP@HBANCFBC@Saturation?5modifier?5is?5only?5avai@ 10009ea0     useasm:useasm.obj
 0001:00008ef0       ??_C@_0FG@HDDPHDFM@Only?5?40?5is?5a?5valid?5component?5sel@ 10009ef0     useasm:useasm.obj
 0001:00008f48       ??_C@_0FM@BHACNAEE@Only?5?40?5and?5?42?5are?5valid?5compone@ 10009f48     useasm:useasm.obj
 0001:00008fa4       ??_C@_0CL@ONLJAILI@The?5maximum?5number?5of?5a?5drc?5regi@ 10009fa4     useasm:useasm.obj
 0001:00008fd0       ??_C@_0DJ@KMKOLKOO@No?5flags?5are?5valid?5for?5a?5depende@ 10009fd0     useasm:useasm.obj
 0001:00009010       ??_C@_0EE@BEFGELHF@A?5dependent?5read?5counter?5registe@ 1000a010     useasm:useasm.obj
 0001:00009058       ??_C@_0FI@PNECLJK@The?5last?5argument?5to?5a?5normalise@ 1000a058     useasm:useasm.obj
 0001:000090b0       ??_C@_0CF@LANAPEBC@Invalid?5choice?5for?5argument?5?$CFd?5t@ 1000a0b0     useasm:useasm.obj
 0001:000090d8       ??_C@_0CK@DBEGJBPP@Integer?5source?5selectors?5aren?8t?5@ 1000a0d8     useasm:useasm.obj
 0001:00009104       ??_C@_0CJ@GGNGAINM@No?5flags?5are?5valid?5for?5argument?5@ 1000a104     useasm:useasm.obj
 0001:00009130       ??_C@_0DH@CDAHKKKK@Argument?5?$CFd?5to?5?$CFs?5should?5be?5an?5i@ 1000a130     useasm:useasm.obj
 0001:00009168       ??_C@_0CB@FIJFOLFN@Invalid?5swizzle?5component?5select@ 1000a168     useasm:useasm.obj
 0001:0000918c       ??_C@_0CB@LDONDCDD@No?5flags?5are?5valid?5for?5a?5swizzle@ 1000a18c     useasm:useasm.obj
 0001:000091b0       ??_C@_0CM@FIPFFMDN@A?5swizzle?5can?8t?5be?5accessed?5in?5i@ 1000a1b0     useasm:useasm.obj
 0001:000091dc       ??_C@_0DN@HIOOPOOE@The?5third?5argument?5to?5a?5fnrm16?5i@ 1000a1dc     useasm:useasm.obj
 0001:00009220       ??_C@_0FJ@MPJBDJBG@The?5destination?5for?5a?5normalise?5@ 1000a220     useasm:useasm.obj
 0001:0000927c       ??_C@_0CE@CEEDGDDA@fnrm32?5isn?8t?5supported?5on?5this?5c@ 1000a27c     useasm:useasm.obj
 0001:000092a0       ??_C@_0DH@NJHBIBLI@The?5normalise?5instruction?5isn?8t?5@ 1000a2a0     useasm:useasm.obj
 0001:000092d8       ??_C@_0BG@BCKONFFM@sop2?5must?5be?5coissued?$AA@ 1000a2d8     useasm:useasm.obj
 0001:000092f0       ??_C@_0EP@OFCLCBOD@Invalid?5choice?5for?5the?5fifth?5arg@ 1000a2f0     useasm:useasm.obj
 0001:00009340       ??_C@_0DC@FMNAGAJ@No?5flags?5are?5valid?5for?5the?5fifth@ 1000a340     useasm:useasm.obj
 0001:00009378       ??_C@_0FK@HNEAMMLH@Invalid?5choice?5for?5the?5fourth?5ar@ 1000a378     useasm:useasm.obj
 0001:000093d4       ??_C@_0DE@HFBEDGPO@No?5flags?5are?5valid?5for?5the?5fourt@ 1000a3d4     useasm:useasm.obj
 0001:00009408       ??_C@_0EC@PPEKPMIP@The?5fourth?5argument?5to?5asop2?5sho@ 1000a408     useasm:useasm.obj
 0001:00009450       ??_C@_0FO@OLALHECM@Invalid?5choice?5for?5the?5third?5arg@ 1000a450     useasm:useasm.obj
 0001:000094b0       ??_C@_0DE@CMCBMCHC@Only?5?4comp?5is?5valid?5for?5the?5thir@ 1000a4b0     useasm:useasm.obj
 0001:000094e8       ??_C@_0EB@OGKIIKPK@The?5third?5argument?5to?5asop2?5shou@ 1000a4e8     useasm:useasm.obj
 0001:00009530       ??_C@_0GB@FOOKGLAG@Invalid?5choice?5for?5the?5second?5ar@ 1000a530     useasm:useasm.obj
 0001:00009594       ??_C@_0DF@BKFNFPMB@Only?5?4comp?5is?5valid?5for?5the?5seco@ 1000a594     useasm:useasm.obj
 0001:000095d0       ??_C@_0EC@JKPDJLLN@The?5second?5argument?5to?5asop2?5sho@ 1000a5d0     useasm:useasm.obj
 0001:00009614       ??_C@_0DD@KLICCPHA@No?5flags?5are?5valid?5for?5the?5first@ 1000a614     useasm:useasm.obj
 0001:00009648       ??_C@_0EB@BIMJBGCB@The?5first?5argument?5to?5asop2?5shou@ 1000a648     useasm:useasm.obj
 0001:0000968c       ??_C@_0CB@PNFMFKCL@sop2?5must?5be?5coissued?5with?5asop2@ 1000a68c     useasm:useasm.obj
 0001:000096b0       ??_C@_0FJ@BADDHEFO@Invalid?5choice?5for?5the?5seventh?5a@ 1000a6b0     useasm:useasm.obj
 0001:0000970c       ??_C@_0DE@KEDJMMFI@No?5flags?5are?5valid?5for?5the?5seven@ 1000a70c     useasm:useasm.obj
 0001:00009740       ??_C@_0EC@HGMCGKBA@The?5seventh?5argument?5to?5sop2?5sho@ 1000a740     useasm:useasm.obj
 0001:00009788       ??_C@_0HE@GKGLGGOL@Invalid?5choice?5for?5the?5sixth?5arg@ 1000a788     useasm:useasm.obj
 0001:000097fc       ??_C@_0DM@OGJGMIAI@Only?5the?5?4comp?5flag?5is?5valid?5for@ 1000a7fc     useasm:useasm.obj
 0001:00009838       ??_C@_0EA@JBHMMHBL@The?5sixth?5argument?5to?5sop2?5shoul@ 1000a838     useasm:useasm.obj
 0001:00009878       ??_C@_0HG@HJBDHCLG@Invalid?5choice?5for?5the?5fifth?5arg@ 1000a878     useasm:useasm.obj
 0001:000098f0       ??_C@_0DM@OEOABLFP@Only?5the?5?4comp?5flag?5is?5valid?5for@ 1000a8f0     useasm:useasm.obj
 0001:00009930       ??_C@_0EA@PEDOBCNH@The?5fifth?5argument?5to?5sop2?5shoul@ 1000a930     useasm:useasm.obj
 0001:00009970       ??_C@_0FB@HBOJEBLF@Invalid?5choices?5for?5the?5fourth?5a@ 1000a970     useasm:useasm.obj
 0001:000099c4       ??_C@_0DD@GDJINGEN@No?5flags?5are?5valid?5for?5the?5fourt@ 1000a9c4     useasm:useasm.obj
 0001:000099f8       ??_C@_0EB@JLEKLKIL@The?5fourth?5argument?5to?5sop2?5shou@ 1000a9f8     useasm:useasm.obj
 0001:00009a3c       ??_C@_0DF@CEJLKMBG@Only?5nearest?5rounding?5is?5support@ 1000aa3c     useasm:useasm.obj
 0001:00009a74       ??_C@_0CM@OHMDJNLO@An?5integer?5source?5selector?5can?8t@ 1000aa74     useasm:useasm.obj
 0001:00009aa0       ??_C@_0DC@PDLMCMGO@No?5flags?5are?5valid?5for?5an?5intege@ 1000aaa0     useasm:useasm.obj
 0001:00009ad8       ??_C@_0EP@KFBPJKBI@The?5fourth?5argument?5to?5a?5pack?5in@ 1000aad8     useasm:useasm.obj
 0001:00009b28       ??_C@_0FK@IMCFLHOE@Invalid?5bytemask?5specified?5?$CIlega@ 1000ab28     useasm:useasm.obj
 0001:00009b84       ??_C@_0DM@CMGEAEEG@Invalid?5bytemask?5specified?5?$CIlega@ 1000ab84     useasm:useasm.obj
 0001:00009bc0       ??_C@_0DD@DLOGHDFD@The?5renable?5flag?5isn?8t?5supported@ 1000abc0     useasm:useasm.obj
 0001:00009bf8       ??_C@_0EO@CDMEKOCM@The?5renable?5flag?5is?5only?5valid?5w@ 1000abf8     useasm:useasm.obj
 0001:00009c48       ??_C@_0FI@FHLKJJEN@The?5scale?5flag?5is?5only?5valid?5whe@ 1000ac48     useasm:useasm.obj
 0001:00009ca0       ??_C@_0CD@DJDKIHIP@The?5maximum?5predicate?5number?5is?5@ 1000aca0     useasm:useasm.obj
 0001:00009cc4       ??_C@_0CF@LNBFBGED@Predicate?5registers?5can?8t?5be?5ind@ 1000acc4     useasm:useasm.obj
 0001:00009cec       ??_C@_0DF@HMHEIKHA@No?5flags?5are?5valid?5for?5the?5predi@ 1000acec     useasm:useasm.obj
 0001:00009d24       ??_C@_0CP@OJDGHEAF@The?5second?5argument?5to?5rlp?5must?5@ 1000ad24     useasm:useasm.obj
 0001:00009d58       ??_C@_0IC@LCJCDNFN@An?5immediate?5source?5argument?5to?5@ 1000ad58     useasm:useasm.obj
 0001:00009ddc       ??_C@_0DB@JHGOCNIO@imul8?1imulu8?5is?5only?5valid?5with?5@ 1000addc     useasm:useasm.obj
 0001:00009e10       ??_C@_0DC@NCLFMCHI@fpadd8?1fpsub8?5is?5only?5valid?5with@ 1000ae10     useasm:useasm.obj
 0001:00009e44       ??_C@_0DA@KAKEJMDJ@A?5mask?5is?5not?5valid?5on?5a?5dotprod@ 1000ae44     useasm:useasm.obj
 0001:00009e74       ??_C@_0DC@PDHCBKCD@A?5repeat?5is?5not?5valid?5on?5a?5dotpr@ 1000ae74     useasm:useasm.obj
 0001:00009ea8       ??_C@_0EI@JILLLJML@This?5instruction?5isn?8t?5available@ 1000aea8     useasm:useasm.obj
 0001:00009ef0       ??_C@_0CE@PCBCMLOI@The?5maximum?5clip?5plane?5number?5is@ 1000aef0     useasm:useasm.obj
 0001:00009f14       ??_C@_0CH@BBGNDHF@A?5clip?5plane?5argument?5is?5not?5ind@ 1000af14     useasm:useasm.obj
 0001:00009f3c       ??_C@_0CM@KGNDPEIK@No?5flags?5are?5valid?5for?5a?5clippla@ 1000af3c     useasm:useasm.obj
 0001:00009f68       ??_C@_0EL@OICFHNIF@The?5second?5argument?5to?5a?5fdpc?5in@ 1000af68     useasm:useasm.obj
 0001:00009fb4       ??_C@_0DI@HLMNAEHK@Only?5i0?5and?5i1?5may?5be?5destinatio@ 1000afb4     useasm:useasm.obj
 0001:00009fec       ??_C@_0CF@KCFJPPBJ@Internal?5registers?5are?5not?5index@ 1000afec     useasm:useasm.obj
 0001:0000a014       ??_C@_0DF@KGNOHAA@No?5flags?5are?5valid?5for?5an?5intern@ 1000b014     useasm:useasm.obj
 0001:0000a050       ??_C@_0FC@GFPCKLPP@The?5second?5argument?5to?5a?5fddp?5in@ 1000b050     useasm:useasm.obj
 0001:0000a0a8       ??_C@_0EL@NPBIKIOJ@The?5fourth?5argument?5to?5a?5fdpc?5in@ 1000b0a8     useasm:useasm.obj
 0001:0000a0f8       ??_C@_0EL@DBBJIGNF@The?5third?5argument?5to?5a?5fddpc?5in@ 1000b0f8     useasm:useasm.obj
 0001:0000a148       ??_C@_0FD@HOIBEICL@The?5second?5argument?5to?5a?5fddpc?5i@ 1000b148     useasm:useasm.obj
 0001:0000a19c       ??_C@_0DG@EDCHLIHP@Only?5?4tz?0?5?4t?$CBz?0?5?4tn?5or?5?4tp?$HMz?5are@ 1000b19c     useasm:useasm.obj
 0001:0000a1d8       ??_C@_0EG@LBAJMGGK@A?5movc?5instruction?5must?5specify?5@ 1000b1d8     useasm:useasm.obj
 0001:0000a220       ??_C@_0GA@OJMMLLIA@On?5this?5processor?5MOVC?5on?5C10?5fo@ 1000b220     useasm:useasm.obj
 0001:0000a280       ??_C@_0DP@CLFDAIAM@A?5movc?5instruction?5must?5include?5@ 1000b280     useasm:useasm.obj
 0001:0000a2c0       ??_C@_0FL@OJDHBDDM@The?5instruction?5is?5affected?5by?5B@ 1000b2c0     useasm:useasm.obj
 0001:0000a320       ??_C@_0IC@ONGMFPGB@The?5instruction?5is?5affected?5by?5B@ 1000b320     useasm:useasm.obj
 0001:0000a3a4       ??_C@_0DP@GHIBIMHL@The?5maximum?5repeat?5count?5for?5an?5@ 1000b3a4     useasm:useasm.obj
 0001:0000a3e8       ??_C@_0EC@JJHLNPNF@The?5seventh?5argument?5to?5sop2wm?5i@ 1000b3e8     useasm:useasm.obj
 0001:0000a42c       ??_C@_0DG@GBFNJGMB@No?5flags?5are?5valid?5for?5the?5seven@ 1000b42c     useasm:useasm.obj
 0001:0000a468       ??_C@_0EE@EGJILBFH@The?5seventh?5argument?5to?5sop2wm?5s@ 1000b468     useasm:useasm.obj
 0001:0000a4b0       ??_C@_0EA@HOMFHCNO@The?5sixth?5argument?5to?5sop2wm?5is?5@ 1000b4b0     useasm:useasm.obj
 0001:0000a4f0       ??_C@_0DE@FDGMDKAF@No?5flags?5are?5valid?5for?5the?5sixth@ 1000b4f0     useasm:useasm.obj
 0001:0000a528       ??_C@_0EC@NALFAHH@The?5sixth?5argument?5to?5sop2wm?5sho@ 1000b528     useasm:useasm.obj
 0001:0000a56c       ??_C@_0DP@BGLACGDG@The?5fifth?5argument?5to?5sop2wm?5is?5@ 1000b56c     useasm:useasm.obj
 0001:0000a5ac       ??_C@_0DM@MLIHGKIL@Only?5?4comp?5is?5a?5valid?5flag?5for?5t@ 1000b5ac     useasm:useasm.obj
 0001:0000a5e8       ??_C@_0EC@JMPNILCM@The?5fifth?5argument?5to?5sop2wm?5sho@ 1000b5e8     useasm:useasm.obj
 0001:0000a630       ??_C@_0EA@NCGPJLOA@The?5fourth?5argument?5to?5sop2wm?5is@ 1000b630     useasm:useasm.obj
 0001:0000a670       ??_C@_0DN@NLJCHBJL@Only?5?4comp?5is?5a?5valid?5flag?5for?5t@ 1000b670     useasm:useasm.obj
 0001:0000a6b0       ??_C@_0ED@FCPONNNK@The?5fourth?5argument?5to?5sop2wm?5sh@ 1000b6b0     useasm:useasm.obj
 0001:0000a6f8       ??_C@_0EN@MDJOPIF@Invalid?5choice?5for?5the?5third?5arg@ 1000b6f8     useasm:useasm.obj
 0001:0000a748       ??_C@_0DC@DCENAPP@No?5flags?5are?5valid?5for?5the?5third@ 1000b748     useasm:useasm.obj
 0001:0000a77c       ??_C@_0DO@EELLDBBD@The?5third?5argument?5to?5asop?5must?5@ 1000b77c     useasm:useasm.obj
 0001:0000a7c0       ??_C@_0HF@CBIPLOPP@Invalid?5choice?5for?5the?5second?5ar@ 1000b7c0     useasm:useasm.obj
 0001:0000a838       ??_C@_0DL@GPHBDAAM@Only?5?4comp?5is?5a?5valid?5flag?5for?5t@ 1000b838     useasm:useasm.obj
 0001:0000a874       ??_C@_0DP@KOIBPLMG@The?5second?5argument?5to?5asop?5must@ 1000b874     useasm:useasm.obj
 0001:0000a8b8       ??_C@_0HE@JFMMNFAC@Invalid?5choice?5for?5the?5first?5arg@ 1000b8b8     useasm:useasm.obj
 0001:0000a92c       ??_C@_0DK@OKDCCLBL@Only?5?4comp?5is?5a?5valid?5flag?5for?5t@ 1000b92c     useasm:useasm.obj
 0001:0000a968       ??_C@_0DO@EOKHKJGH@The?5first?5argument?5to?5asop?5must?5@ 1000b968     useasm:useasm.obj
 0001:0000a9a8       ??_C@_0CA@LJJNKDND@lrp1?5must?5be?5coissued?5with?5asop?$AA@ 1000b9a8     useasm:useasm.obj
 0001:0000a9c8       ??_C@_0BH@DOCDFOCO@lrp1?5must?5be?5coisssued?$AA@ 1000b9c8     useasm:useasm.obj
 0001:0000a9e0       ??_C@_0BG@CHKAJNEL@lrp1?5must?5be?5coissued?$AA@ 1000b9e0     useasm:useasm.obj
 0001:0000a9f8       ??_C@_0EO@FKMJCGBG@Invalid?5choice?5for?5the?5seventh?5a@ 1000b9f8     useasm:useasm.obj
 0001:0000aa48       ??_C@_0DE@MPNHBAIK@No?5flags?5are?5valid?5for?5the?5seven@ 1000ba48     useasm:useasm.obj
 0001:0000aa80       ??_C@_0EB@NCENCBNO@The?5seventh?5argument?5to?5lrp1?5mus@ 1000ba80     useasm:useasm.obj
 0001:0000aac8       ??_C@_0EN@NGJPOHKM@Invalid?5choice?5for?5the?5sixth?5arg@ 1000bac8     useasm:useasm.obj
 0001:0000ab18       ??_C@_0DM@INHIBENK@Only?5the?5?4comp?5flag?5is?5valid?5for@ 1000bb18     useasm:useasm.obj
 0001:0000ab54       ??_C@_0DP@NEMNCNNA@The?5sixth?5argument?5to?5lrp1?5must?5@ 1000bb54     useasm:useasm.obj
 0001:0000ab98       ??_C@_0FA@BCOHELNN@Invalid?5choice?5for?5the?5fifth?5arg@ 1000bb98     useasm:useasm.obj
 0001:0000abe8       ??_C@_0CM@KDAMEKKC@An?5integer?5source?5selector?5is?5no@ 1000bbe8     useasm:useasm.obj
 0001:0000ac14       ??_C@_0DM@IPAOMHIN@Only?5the?5?4comp?5flag?5is?5valid?5for@ 1000bc14     useasm:useasm.obj
 0001:0000ac50       ??_C@_0DP@CGMBCHII@The?5fifth?5argument?5to?5lrp1?5must?5@ 1000bc50     useasm:useasm.obj
 0001:0000ac90       ??_C@_0BG@IEPGBLOC@lrp2?5must?5be?5coissued?$AA@ 1000bc90     useasm:useasm.obj
 0001:0000aca8       ??_C@_0EJ@KJLKFMN@Only?5zero?0?5one?5and?5s2a?5are?5valid@ 1000bca8     useasm:useasm.obj
 0001:0000acf4       ??_C@_0DE@FDNIJKHO@Only?5?4comp?5is?5valid?5for?5the?5seco@ 1000bcf4     useasm:useasm.obj
 0001:0000ad28       ??_C@_0DP@GCMJDOBH@The?5second?5argument?5to?5alrp?5must@ 1000bd28     useasm:useasm.obj
 0001:0000ad68       ??_C@_0EI@POLJNHOP@Only?5zero?0?5one?5and?5s1a?5are?5valid@ 1000bd68     useasm:useasm.obj
 0001:0000adb0       ??_C@_0DD@LEOOHHIE@Only?5?4comp?5is?5valid?5for?5the?5firs@ 1000bdb0     useasm:useasm.obj
 0001:0000ade4       ??_C@_0DO@ICOPGMLG@The?5first?5argument?5to?5alrp?5must?5@ 1000bde4     useasm:useasm.obj
 0001:0000ae24       ??_C@_0CA@BBLPFF@lrp2?5must?5be?5coissued?5with?5alrp?$AA@ 1000be24     useasm:useasm.obj
 0001:0000ae48       ??_C@_0FD@JFBMKMNH@Invalid?5choice?5for?5the?5seventh?5a@ 1000be48     useasm:useasm.obj
 0001:0000aea0       ??_C@_0EN@GMGJLELO@If?5the?5seventh?5argument?5to?5lrp2?5@ 1000bea0     useasm:useasm.obj
 0001:0000aef0       ??_C@_0FB@FJHLFMAN@If?5the?5seventh?5argument?5to?5lrp2?5@ 1000bef0     useasm:useasm.obj
 0001:0000af48       ??_C@_0EP@GBKEKGGN@If?5the?5seventh?5argument?5to?5lrp2?5@ 1000bf48     useasm:useasm.obj
 0001:0000af98       ??_C@_0EK@MPPLIHCI@If?5the?5seventh?5argument?5to?5lrp2?5@ 1000bf98     useasm:useasm.obj
 0001:0000afe4       ??_C@_0DN@BJBDMCPE@Only?5the?5?4comp?5flag?5is?5valid?5for@ 1000bfe4     useasm:useasm.obj
 0001:0000b028       ??_C@_0EA@MACNPBPH@The?5eighth?5argument?5to?5lrp2?5must@ 1000c028     useasm:useasm.obj
 0001:0000b068       ??_C@_0DO@GLBNDEGP@Only?5the?5?4comp?5flag?5is?5valid?5for@ 1000c068     useasm:useasm.obj
 0001:0000b0a8       ??_C@_0EB@JPKFCBLJ@The?5seventh?5argument?5to?5lrp2?5mus@ 1000c0a8     useasm:useasm.obj
 0001:0000b0f0       ??_C@_0HH@IBAGBKNH@Invalid?5choice?5for?5the?5sixth?5arg@ 1000c0f0     useasm:useasm.obj
 0001:0000b168       ??_C@_0DM@KGFFEHBJ@Only?5the?5?4comp?5flag?5is?5valid?5for@ 1000c168     useasm:useasm.obj
 0001:0000b1a4       ??_C@_0DP@JJCFCNLH@The?5sixth?5argument?5to?5lrp2?5must?5@ 1000c1a4     useasm:useasm.obj
 0001:0000b1e8       ??_C@_0HI@KGJMFIGE@Invalid?5choice?5for?5the?5fifth?5arg@ 1000c1e8     useasm:useasm.obj
 0001:0000b260       ??_C@_0DM@PNPLCKBO@Only?5the?5?4comp?5flag?5is?5valid?5for@ 1000c260     useasm:useasm.obj
 0001:0000b29c       ??_C@_0DP@JFIMNECE@The?5fifth?5argument?5to?5sop3?5must?5@ 1000c29c     useasm:useasm.obj
 0001:0000b2e0       ??_C@_0EP@LFLPCFJM@Invalid?5choice?5for?5the?5second?5ar@ 1000c2e0     useasm:useasm.obj
 0001:0000b330       ??_C@_0DE@GEPIHLDC@No?5flags?5are?5valid?5for?5the?5secon@ 1000c330     useasm:useasm.obj
 0001:0000b368       ??_C@_0EA@CILJPHKB@The?5second?5argument?5to?5arsop?5mus@ 1000c368     useasm:useasm.obj
 0001:0000b3a8       ??_C@_0FO@BGCOGJJP@Invalid?5choice?5for?5the?5first?5arg@ 1000c3a8     useasm:useasm.obj
 0001:0000b408       ??_C@_0DE@LFEIHKHD@Only?5?4comp?5is?5valid?5for?5the?5firs@ 1000c408     useasm:useasm.obj
 0001:0000b43c       ??_C@_0DP@IJIIECIN@The?5first?5argument?5to?5arsop?5must@ 1000c43c     useasm:useasm.obj
 0001:0000b480       ??_C@_0EK@DIJKPKNM@SOP3?5with?5ARSOP?5and?5a?5complement@ 1000c480     useasm:useasm.obj
 0001:0000b4d0       ??_C@_0EO@BNBKMGBP@Invalid?5choice?5for?5the?5second?5ar@ 1000c4d0     useasm:useasm.obj
 0001:0000b520       ??_C@_0DD@KDAMLAMK@No?5flags?5are?5valid?5for?5the?5secon@ 1000c520     useasm:useasm.obj
 0001:0000b558       ??_C@_0FN@ONPCNNEO@Invalid?5choice?5for?5the?5first?5arg@ 1000c558     useasm:useasm.obj
 0001:0000b5b8       ??_C@_0DD@KIGKAAGO@Only?5?4comp?5is?5valid?5for?5the?5firs@ 1000c5b8     useasm:useasm.obj
 0001:0000b5f0       ??_C@_0FE@LNCOBNA@Invalid?5choice?5for?5the?5first?5arg@ 1000c5f0     useasm:useasm.obj
 0001:0000b648       ??_C@_0FE@JJEFPIJ@Invalid?5choice?5for?5the?5first?5arg@ 1000c648     useasm:useasm.obj
 0001:0000b6a0       ??_C@_0ED@PGOFNOAD@sop3?5with?5a?5negate?5destination?5m@ 1000c6a0     useasm:useasm.obj
 0001:0000b6e4       ??_C@_0CE@OHCGBBLC@sop3?5without?5a?5coissued?5instruct@ 1000c6e4     useasm:useasm.obj
 0001:0000b708       ??_C@_0BG@MFEMFFAE@sop3?5must?5be?5coissued?$AA@ 1000c708     useasm:useasm.obj
 0001:0000b720       ??_C@_0EL@GLFHPIPJ@Invalid?5choice?5for?5eighth?5argume@ 1000c720     useasm:useasm.obj
 0001:0000b770       ??_C@_0EA@DOIIACDM@The?5eighth?5argument?5to?5sop3?5must@ 1000c770     useasm:useasm.obj
 0001:0000b7b0       ??_C@_0EP@LLOJFENH@Invalid?5choice?5for?5the?5seventh?5a@ 1000c7b0     useasm:useasm.obj
 0001:0000b800       ??_C@_0DE@LNCCPNBJ@No?5flags?5are?5valid?5for?5the?5seven@ 1000c800     useasm:useasm.obj
 0001:0000b838       ??_C@_0EB@GBAANCHC@The?5seventh?5argument?5to?5sop3?5mus@ 1000c838     useasm:useasm.obj
 0001:0000b880       ??_C@_0HE@NOFOGDCI@Invalid?5choice?5for?5the?5sixth?5arg@ 1000c880     useasm:useasm.obj
 0001:0000b8f4       ??_C@_0DK@GPFHLHKL@Only?5?4comp?5is?5a?5valid?5flag?5for?5t@ 1000c8f4     useasm:useasm.obj
 0001:0000b930       ??_C@_0DP@GHIANOHM@The?5sixth?5argument?5to?5sop3?5must?5@ 1000c930     useasm:useasm.obj
 0001:0000b970       ??_C@_0HE@OENIBECC@Invalid?5choice?5for?5the?5fifth?5arg@ 1000c970     useasm:useasm.obj
 0001:0000b9e4       ??_C@_0DK@GNCBGEPM@Only?5?4comp?5is?5a?5valid?5flag?5for?5t@ 1000c9e4     useasm:useasm.obj
 0001:0000ba20       ??_C@_0BH@NMPINIEC@sop3?5can?8t?5be?5repeated?$AA@ 1000ca20     useasm:useasm.obj
 0001:0000ba38       ??_C@_0DK@OMANMEPM@Only?5s2a?5is?5a?5valid?5choice?5for?5t@ 1000ca38     useasm:useasm.obj
 0001:0000ba74       ??_C@_0DK@DPJMNKAL@Only?5?4comp?5is?5a?5valid?5flag?5for?5t@ 1000ca74     useasm:useasm.obj
 0001:0000bab0       ??_C@_0DP@BFGILNHD@The?5tenth?5argument?5to?5ima8?5must?5@ 1000cab0     useasm:useasm.obj
 0001:0000baf0       ??_C@_0DL@FMNMANPN@Only?5s1a?5is?5a?5valid?5choice?5for?5t@ 1000caf0     useasm:useasm.obj
 0001:0000bb2c       ??_C@_0DL@PMLPCLJP@Only?5?4comp?5is?5a?5valid?5flag?5for?5t@ 1000cb2c     useasm:useasm.obj
 0001:0000bb68       ??_C@_0EA@OKAGHCFL@The?5nineth?5argument?5to?5ima8?5must@ 1000cb68     useasm:useasm.obj
 0001:0000bba8       ??_C@_0ED@FKCOCDED@Only?5s0a?5and?5s1a?5are?5valid?5choic@ 1000cba8     useasm:useasm.obj
 0001:0000bbec       ??_C@_0DL@HABGHCJK@Only?5?4comp?5is?5a?5valid?5flag?5for?5t@ 1000cbec     useasm:useasm.obj
 0001:0000bc28       ??_C@_0EA@EABBPNKK@The?5eighth?5argument?5to?5ima8?5must@ 1000cc28     useasm:useasm.obj
 0001:0000bc68       ??_C@_0ED@FDKGPKDC@Only?5s2?5and?5s2a?5are?5valid?5choice@ 1000cc68     useasm:useasm.obj
 0001:0000bcac       ??_C@_0DM@LBKALADI@Only?5?4comp?5is?5a?5valid?5flag?5for?5t@ 1000ccac     useasm:useasm.obj
 0001:0000bce8       ??_C@_0EB@BPJJCNOE@The?5seventh?5argument?5to?5ima8?5mus@ 1000cce8     useasm:useasm.obj
 0001:0000bd30       ??_C@_0EB@CLJBDDPJ@Only?5s1?5and?5s1a?5are?5valid?5choice@ 1000cd30     useasm:useasm.obj
 0001:0000bd74       ??_C@_0DK@BBBOOAIP@Only?5?4comp?5is?5a?5valid?5flag?5for?5t@ 1000cd74     useasm:useasm.obj
 0001:0000bdb0       ??_C@_0DP@BJBJCBOK@The?5sixth?5argument?5to?5ima8?5must?5@ 1000cdb0     useasm:useasm.obj
 0001:0000bdf0       ??_C@_0EK@KADHKBHD@Only?5s0?0?5s1?0?5s0a?5and?5s1a?5are?5val@ 1000cdf0     useasm:useasm.obj
 0001:0000be3c       ??_C@_0DK@BDGIDDNI@Only?5?4comp?5is?5a?5valid?5flag?5for?5t@ 1000ce3c     useasm:useasm.obj
 0001:0000be78       ??_C@_0DP@OLBFCLLC@The?5fifth?5argument?5to?5ima8?5must?5@ 1000ce78     useasm:useasm.obj
 0001:0000beb8       ??_C@_0EK@HCFFGHCH@Third?5argument?5to?5ima16?5is?58?9bit@ 1000ceb8     useasm:useasm.obj
 0001:0000bf08       ??_C@_0EL@EFNHNPFP@Second?5argument?5to?5ima16?5is?58?9bi@ 1000cf08     useasm:useasm.obj
 0001:0000bf54       ??_C@_0DD@DHKGKKGN@No?5flags?5are?5valid?5for?5the?5sixth@ 1000cf54     useasm:useasm.obj
 0001:0000bf88       ??_C@_0CM@KFKJJGEN@The?5sixth?5argument?5to?5ima16?5isn?8@ 1000cf88     useasm:useasm.obj
 0001:0000bfb4       ??_C@_0DC@FLFMKFFD@The?5sixth?5argument?5to?5ima16?5must@ 1000cfb4     useasm:useasm.obj
 0001:0000bfe8       ??_C@_0EN@LDKLHMAN@Invalid?5source?5data?5format?5for?5i@ 1000cfe8     useasm:useasm.obj
 0001:0000c038       ??_C@_0DD@MCKLBIOJ@No?5flags?5are?5valid?5for?5the?5fifth@ 1000d038     useasm:useasm.obj
 0001:0000c06c       ??_C@_0CM@LHIIENBO@The?5fifth?5argument?5to?5ima16?5isn?8@ 1000d06c     useasm:useasm.obj
 0001:0000c098       ??_C@_0DC@CIEPCOAH@The?5fifth?5argument?5to?5ima16?5must@ 1000d098     useasm:useasm.obj
 0001:0000c0cc       ??_C@_0DJ@KMFCNFLN@Only?5one?5of?5?4s?5and?5?4u?5can?5be?5spe@ 1000d0cc     useasm:useasm.obj
 0001:0000c108       ??_C@_0DN@LMMEBOND@The?5maximum?5destination?5shift?5fo@ 1000d108     useasm:useasm.obj
 0001:0000c148       ??_C@_0EA@BEAJFKLN@The?5maximum?5register?5number?5for?5@ 1000d148     useasm:useasm.obj
 0001:0000c188       ??_C@_0CL@DOOAPBOB@The?5eighth?5source?5to?5imae?5can?8t?5@ 1000d188     useasm:useasm.obj
 0001:0000c1b4       ??_C@_0DB@PKHIFEJJ@No?5flags?5are?5valid?5for?5the?5eight@ 1000d1b4     useasm:useasm.obj
 0001:0000c1e8       ??_C@_0EI@OMIBHEJN@The?5eighth?5source?5to?5imae?5should@ 1000d1e8     useasm:useasm.obj
 0001:0000c230       ??_C@_0EH@DLKGLNI@Only?5cie?5or?5nothing?5are?5valid?5ch@ 1000d230     useasm:useasm.obj
 0001:0000c278       ??_C@_0DE@MMHOIJCE@No?5flags?5are?5valid?5for?5the?5seven@ 1000d278     useasm:useasm.obj
 0001:0000c2ac       ??_C@_0CN@IKCGDAFI@The?5seventh?5argument?5to?5imae?5isn@ 1000d2ac     useasm:useasm.obj
 0001:0000c2dc       ??_C@_0DE@IAOPODPF@The?5seventh?5argument?5to?5imae?5mus@ 1000d2dc     useasm:useasm.obj
 0001:0000c310       ??_C@_0EF@JBDPGDKG@Only?5coe?5or?5nothing?5are?5valid?5ch@ 1000d310     useasm:useasm.obj
 0001:0000c358       ??_C@_0DC@GPPMJACC@No?5flags?5are?5valid?5for?5the?5sixth@ 1000d358     useasm:useasm.obj
 0001:0000c38c       ??_C@_0CL@CDIKAGGM@The?5sixth?5argument?5to?5imae?5isn?8t@ 1000d38c     useasm:useasm.obj
 0001:0000c3b8       ??_C@_0DC@HDJGOJKK@The?5sixth?5argument?5to?5imae?5must?5@ 1000d3b8     useasm:useasm.obj
 0001:0000c3ec       ??_C@_0DD@DNBAOKIA@?4low?5and?5?4high?5are?5meaningless?5f@ 1000d3ec     useasm:useasm.obj
 0001:0000c420       ??_C@_0EG@PNOIEBGC@One?5of?5?4low?5or?5?4high?5should?5be?5s@ 1000d420     useasm:useasm.obj
 0001:0000c468       ??_C@_0EH@DLDLJEEK@One?5of?5?4low?5or?5?4high?5should?5be?5s@ 1000d468     useasm:useasm.obj
 0001:0000c4b0       ??_C@_0EG@HGBJOGAP@One?5of?5?4low?5or?5?4high?5should?5be?5s@ 1000d4b0     useasm:useasm.obj
 0001:0000c4f8       ??_C@_0BN@MCMCHHHO@Invalid?5data?5format?5for?5imae?$AA@ 1000d4f8     useasm:useasm.obj
 0001:0000c518       ??_C@_0DC@GNIKEDHF@No?5flags?5are?5valid?5for?5the?5fifth@ 1000d518     useasm:useasm.obj
 0001:0000c54c       ??_C@_0CL@LFLIAFDF@The?5fifth?5argument?5to?5imae?5isn?8t@ 1000d54c     useasm:useasm.obj
 0001:0000c578       ??_C@_0DB@NOAIOELF@The?5fifth?5argument?5to?5imae?5must?5@ 1000d578     useasm:useasm.obj
 0001:0000c5ac       ??_C@_0DM@EHOELKCO@The?5maximum?5destination?5shift?5fo@ 1000d5ac     useasm:useasm.obj
 0001:0000c5e8       ??_C@_0DE@JCLFGKBG@Maximum?5repeat?5count?5on?5an?5integ@ 1000d5e8     useasm:useasm.obj
 0001:0000c620       ??_C@_0EG@JFIEFIAN@Only?5u8?5or?5s8?5are?5valid?5as?5a?5cho@ 1000d620     useasm:useasm.obj
 0001:0000c668       ??_C@_0DF@BFAJNMNE@No?5flags?5are?5valid?5for?5the?5ninet@ 1000d668     useasm:useasm.obj
 0001:0000c6a0       ??_C@_0EB@EPNJCIMP@The?5nineth?5argument?5to?5ssum16?5mu@ 1000d6a0     useasm:useasm.obj
 0001:0000c6e8       ??_C@_0EM@CDDPPEDE@Only?5iadd?5or?5nothing?5is?5valid?5as@ 1000d6e8     useasm:useasm.obj
 0001:0000c734       ??_C@_0DF@HKMJENGI@No?5flags?5are?5valid?5for?5the?5eight@ 1000d734     useasm:useasm.obj
 0001:0000c770       ??_C@_0EB@IFMJPNMK@The?5eighth?5argument?5to?5ssum16?5mu@ 1000d770     useasm:useasm.obj
 0001:0000c7b8       ??_C@_0ED@OAGGGGIH@Only?5i0?5or?5r1?5valid?5as?5a?5choice?5@ 1000d7b8     useasm:useasm.obj
 0001:0000c7fc       ??_C@_0CF@BGFEHLBP@An?5internal?5register?5isn?8t?5index@ 1000d7fc     useasm:useasm.obj
 0001:0000c824       ??_C@_0DG@GDJPLBEI@No?5flags?5are?5valid?5for?5the?5seven@ 1000d824     useasm:useasm.obj
 0001:0000c860       ??_C@_0EC@BEPCBJIN@The?5seventh?5argument?5to?5ssum16?5m@ 1000d860     useasm:useasm.obj
 0001:0000c8a8       ??_C@_0EL@BECKFGPA@Only?5iadd?5or?5nothing?5is?5valid?5as@ 1000d8a8     useasm:useasm.obj
 0001:0000c8f4       ??_C@_0DE@FBKOBNIM@No?5flags?5are?5valid?5for?5the?5sixth@ 1000d8f4     useasm:useasm.obj
 0001:0000c928       ??_C@_0EA@PDEMLEIG@The?5sixth?5argument?5to?5ssum16?5mus@ 1000d928     useasm:useasm.obj
 0001:0000c968       ??_C@_0EL@HFHGKGHC@Only?5idst?5or?5nothing?5is?5valid?5as@ 1000d968     useasm:useasm.obj
 0001:0000c9b4       ??_C@_0CL@KCGNBGBH@An?5integer?5source?5selector?5isn?8t@ 1000d9b4     useasm:useasm.obj
 0001:0000c9e0       ??_C@_0DE@LLIOFHAH@No?5flags?5are?5valid?5for?5the?5fifth@ 1000d9e0     useasm:useasm.obj
 0001:0000ca18       ??_C@_0EA@JGAOGBEK@The?5fifth?5argument?5to?5ssum16?5mus@ 1000da18     useasm:useasm.obj
 0001:0000ca58       ??_C@_0DE@IJOOAFAA@Maximum?5repeat?5count?5on?5an?5SSUM1@ 1000da58     useasm:useasm.obj
 0001:0000ca8c       ??_C@_0CJ@EGABLJED@ssum16?5isn?8t?5available?5on?5this?5p@ 1000da8c     useasm:useasm.obj
 0001:0000cab8       ??_C@_0EL@LEHINHKP@Only?5scale?5or?5nothing?5is?5valid?5a@ 1000dab8     useasm:useasm.obj
 0001:0000cb04       ??_C@_0DD@MBMDINHI@No?5flags?5are?5valid?5for?5the?5eight@ 1000db04     useasm:useasm.obj
 0001:0000cb38       ??_C@_0DP@DNLIJOFH@The?5eighth?5argument?5to?5firv?5must@ 1000db38     useasm:useasm.obj
 0001:0000cb78       ??_C@_0EL@PLEHJOGF@Only?5iadd?5or?5nothing?5is?5valid?5as@ 1000db78     useasm:useasm.obj
 0001:0000cbc4       ??_C@_0DE@LOMDNFBJ@No?5flags?5are?5valid?5for?5the?5seven@ 1000dbc4     useasm:useasm.obj
 0001:0000cbf8       ??_C@_0EA@LAOANIGO@The?5seventh?5argument?5to?5firv?5mus@ 1000dbf8     useasm:useasm.obj
 0001:0000cc38       ??_C@_0EM@PPMBHMLB@Only?5?$CLsrc2?42?5or?5nothing?5is?5valid@ 1000dc38     useasm:useasm.obj
 0001:0000cc84       ??_C@_0DC@BNEBMMBP@No?5flags?5are?5valid?5for?5the?5sixth@ 1000dc84     useasm:useasm.obj
 0001:0000ccb8       ??_C@_0DO@IGFJMJCL@The?5sixth?5argument?5to?5firv?5must?5@ 1000dcb8     useasm:useasm.obj
 0001:0000ccf8       ??_C@_0CL@MDHBFNJL@The?5fifth?5argument?5to?5firv?5isn?8t@ 1000dcf8     useasm:useasm.obj
 0001:0000cd24       ??_C@_0DC@BPDHBPEI@No?5flags?5are?5valid?5for?5the?5fifth@ 1000dd24     useasm:useasm.obj
 0001:0000cd58       ??_C@_0DP@LCJNOCNN@The?5fifth?5argument?5to?5firv?5must?5@ 1000dd58     useasm:useasm.obj
 0001:0000cd98       ??_C@_0HP@FKECLPEM@The?5register?5bank?5for?5firv?5sourc@ 1000dd98     useasm:useasm.obj
 0001:0000ce18       ??_C@_0EG@NEGMNEOD@The?5register?5banks?5for?5source?50?5@ 1000de18     useasm:useasm.obj
 0001:0000ce60       ??_C@_0CD@BDBMNPHP@Maximum?5repeat?5count?5on?5firv?5is?5@ 1000de60     useasm:useasm.obj
 0001:0000ce88       ??_C@_0EK@MMLIIHNN@Only?5scale?5or?5nothing?5is?5valid?5a@ 1000de88     useasm:useasm.obj
 0001:0000ced8       ??_C@_0EJ@NGJACPPH@Only?5iadd?5or?5nothing?5is?5valid?5as@ 1000ded8     useasm:useasm.obj
 0001:0000cf24       ??_C@_0DO@OIFDNPHI@The?5fifth?5argument?5to?5firv?5must?5@ 1000df24     useasm:useasm.obj
 0001:0000cf68       ??_C@_0EN@EIOOMBFD@Only?5?$CLsrc2?42?5or?5nothing?5is?5valid@ 1000df68     useasm:useasm.obj
 0001:0000cfb8       ??_C@_0DP@FGKELBIB@The?5fourth?5argument?5to?5firv?5must@ 1000dfb8     useasm:useasm.obj
 0001:0000cff8       ??_C@_0EE@EGNLBLOB@The?5register?5bank?5for?5firvh?5sour@ 1000dff8     useasm:useasm.obj
 0001:0000d03c       ??_C@_0CE@HBKLLEAA@Maximum?5repeat?5count?5on?5firvh?5is@ 1000e03c     useasm:useasm.obj
 0001:0000d060       ??_C@_0CI@CFGKFHCM@firvh?5isn?8t?5available?5on?5this?5pr@ 1000e060     useasm:useasm.obj
 0001:0000d088       ??_C@_0EA@CNFLJPLE@The?5nineth?5argument?5to?5bilin?5mus@ 1000e088     useasm:useasm.obj
 0001:0000d0c8       ??_C@_0DE@OJKKKHIL@No?5flags?5are?5valid?5for?5the?5ninet@ 1000e0c8     useasm:useasm.obj
 0001:0000d0fc       ??_C@_0CN@DJDNLEIC@The?5nineth?5argument?5to?5bilin?5isn@ 1000e0fc     useasm:useasm.obj
 0001:0000d12c       ??_C@_0DH@HFBBMNAM@The?5nineth?5argument?5to?5bilin?5mus@ 1000e12c     useasm:useasm.obj
 0001:0000d168       ??_C@_0EA@OPFHNAEG@The?5eighth?5argument?5to?5bilin?5mus@ 1000e168     useasm:useasm.obj
 0001:0000d1a8       ??_C@_0DE@JJEMPKFN@No?5flags?5are?5valid?5for?5the?5eight@ 1000e1a8     useasm:useasm.obj
 0001:0000d1dc       ??_C@_0CN@MBAHDJDB@The?5eighth?5argument?5to?5bilin?5isn@ 1000e1dc     useasm:useasm.obj
 0001:0000d210       ??_C@_0EJ@BIMEJMPB@The?5eighth?5argument?5to?5bilin?5mus@ 1000e210     useasm:useasm.obj
 0001:0000d260       ??_C@_0EB@LANPAAAI@The?5seventh?5argument?5to?5bilin?5mu@ 1000e260     useasm:useasm.obj
 0001:0000d2a4       ??_C@_0DF@KDIGKLML@No?5flags?5are?5valid?5for?5the?5seven@ 1000e2a4     useasm:useasm.obj
 0001:0000d2dc       ??_C@_0CO@HELDAPEL@The?5seventh?5argument?5to?5bilin?5is@ 1000e2dc     useasm:useasm.obj
 0001:0000d310       ??_C@_0EF@CJMNJFOI@The?5seventh?5argument?5to?5bilin?5mu@ 1000e310     useasm:useasm.obj
 0001:0000d358       ??_C@_0EG@CPMAHDPO@The?5sixth?5argument?5to?5bilin?5must@ 1000e358     useasm:useasm.obj
 0001:0000d3a0       ??_C@_0DD@EKEGIMOH@No?5flags?5are?5valid?5for?5the?5sixth@ 1000e3a0     useasm:useasm.obj
 0001:0000d3d4       ??_C@_0CM@FFKOFHMI@The?5sixth?5argument?5to?5bilin?5isn?8@ 1000e3d4     useasm:useasm.obj
 0001:0000d400       ??_C@_0EA@HDMMDEFM@The?5sixth?5argument?5to?5bilin?5must@ 1000e400     useasm:useasm.obj
 0001:0000d440       ??_C@_0EA@BGIOOBJA@The?5fifth?5argument?5to?5bilin?5must@ 1000e440     useasm:useasm.obj
 0001:0000d480       ??_C@_0DD@LPELDOGD@No?5flags?5are?5valid?5for?5the?5fifth@ 1000e480     useasm:useasm.obj
 0001:0000d4b4       ??_C@_0CM@EHIPIMJL@The?5fifth?5argument?5to?5bilin?5isn?8@ 1000e4b4     useasm:useasm.obj
 0001:0000d4e0       ??_C@_0EB@ILBDCOKI@The?5fifth?5argument?5to?5bilin?5must@ 1000e4e0     useasm:useasm.obj
 0001:0000d524       ??_C@_0CE@PONMLKAD@Maximum?5repeat?5count?5on?5bilin?5is@ 1000e524     useasm:useasm.obj
 0001:0000d548       ??_C@_0DE@JHKIEKPM@The?5range?5of?5the?5nineth?5argument@ 1000e548     useasm:useasm.obj
 0001:0000d57c       ??_C@_0DH@KHNFKIAG@The?5nineth?5argument?5to?5firh?5must@ 1000e57c     useasm:useasm.obj
 0001:0000d5b4       ??_C@_0DF@JCFPNCKH@The?5range?5of?5the?5eighth?5argument@ 1000e5b4     useasm:useasm.obj
 0001:0000d5ec       ??_C@_0DH@BGJCEECP@The?5eighth?5argument?5to?5firh?5must@ 1000e5ec     useasm:useasm.obj
 0001:0000d624       ??_C@_0CI@HEOOLMFP@The?5maximum?5filter?5coefficent?5se@ 1000e624     useasm:useasm.obj
 0001:0000d64c       ??_C@_0DC@CJJPPKOA@No?5flags?5are?5valid?5for?5a?5filter?5@ 1000e64c     useasm:useasm.obj
 0001:0000d680       ??_C@_0CI@BPHBGDKA@Filter?5coefficent?5sets?5aren?8t?5in@ 1000e680     useasm:useasm.obj
 0001:0000d6a8       ??_C@_0DN@NIIJMAFI@The?5seventh?5argument?5to?5firh?5mus@ 1000e6a8     useasm:useasm.obj
 0001:0000d6e8       ??_C@_0CK@MCCCMAME@No?5flags?5are?5valid?5for?5an?5immedi@ 1000e6e8     useasm:useasm.obj
 0001:0000d714       ??_C@_0CE@BOJPMEGF@An?5immediate?5value?5is?5not?5indexa@ 1000e714     useasm:useasm.obj
 0001:0000d738       ??_C@_0DK@HBKJDJHH@The?5sixth?5argument?5to?5firh?5must?5@ 1000e738     useasm:useasm.obj
 0001:0000d774       ??_C@_0DC@MLHGCAJH@No?5flags?5are?5valid?5for?5the?5fifth@ 1000e774     useasm:useasm.obj
 0001:0000d7a8       ??_C@_0CL@PEPPBDAK@The?5fifth?5argument?5to?5firh?5isn?8t@ 1000e7a8     useasm:useasm.obj
 0001:0000d7d4       ??_C@_0DN@JOJEKONN@The?5fifth?5argument?5to?5firh?5must?5@ 1000e7d4     useasm:useasm.obj
 0001:0000d818       ??_C@_0HP@FIJDICNA@The?5register?5bank?5for?5firh?5sourc@ 1000e818     useasm:useasm.obj
 0001:0000d898       ??_C@_0EG@FDFDPJHP@The?5register?5banks?5for?5source?50?5@ 1000e898     useasm:useasm.obj
 0001:0000d8e0       ??_C@_0CD@HKCNPMGG@Maximum?5repeat?5count?5on?5firh?5is?5@ 1000e8e0     useasm:useasm.obj
 0001:0000d904       ??_C@_0DP@DKFIGMEP@The?5destination?5argument?5to?5firh@ 1000e904     useasm:useasm.obj
 0001:0000d944       ??_C@_0DF@BDOGECIG@The?5range?5of?5the?5nineth?5argument@ 1000e944     useasm:useasm.obj
 0001:0000d97c       ??_C@_0DI@PJONGPDL@The?5nineth?5argument?5to?5firhh?5mus@ 1000e97c     useasm:useasm.obj
 0001:0000d9b4       ??_C@_0DG@KGIDPMLA@The?5range?5of?5the?5eighth?5argument@ 1000e9b4     useasm:useasm.obj
 0001:0000d9ec       ??_C@_0DI@LLOOLALL@The?5eighth?5argument?5to?5firhh?5mus@ 1000e9ec     useasm:useasm.obj
 0001:0000da24       ??_C@_0DO@EEFEJEHK@The?5seventh?5argument?5to?5firhh?5mu@ 1000ea24     useasm:useasm.obj
 0001:0000da64       ??_C@_0DL@OHNCDOMJ@The?5sixth?5argument?5to?5firhh?5must@ 1000ea64     useasm:useasm.obj
 0001:0000daa0       ??_C@_0DD@MDIEJBGI@No?5flags?5are?5valid?5for?5the?5fifth@ 1000eaa0     useasm:useasm.obj
 0001:0000dad4       ??_C@_0CM@DLIOMDAE@The?5fifth?5argument?5to?5firhh?5isn?8@ 1000ead4     useasm:useasm.obj
 0001:0000db00       ??_C@_0DO@NGNIOBOG@The?5fifth?5argument?5to?5firhh?5must@ 1000eb00     useasm:useasm.obj
 0001:0000db40       ??_C@_0IA@FCFJDLLG@The?5register?5bank?5for?5firhh?5sour@ 1000eb40     useasm:useasm.obj
 0001:0000dbc0       ??_C@_0EH@HPAOOKCK@The?5register?5banks?5for?5source?50?5@ 1000ebc0     useasm:useasm.obj
 0001:0000dc08       ??_C@_0CE@BFKJCNOD@Maximum?5repeat?5count?5on?5firhh?5is@ 1000ec08     useasm:useasm.obj
 0001:0000dc2c       ??_C@_0CI@CPDCNICP@firhh?5isn?8t?5available?5on?5this?5pr@ 1000ec2c     useasm:useasm.obj
 0001:0000dc54       ??_C@_0DC@OJMFLOPA@A?5repeat?5count?5isn?8t?5supported?5o@ 1000ec54     useasm:useasm.obj
 0001:0000dc88       ??_C@_0DJ@PFEOBFIJ@Valid?5values?5for?5argument?5?$CFd?5to?5@ 1000ec88     useasm:useasm.obj
 0001:0000dcc4       ??_C@_0DK@PJMBECMK@On?5this?5core?5SMP?5result?5format?5c@ 1000ecc4     useasm:useasm.obj
 0001:0000dd00       ??_C@_0FI@CPMJEANO@The?5fourth?5argument?5to?5a?5sampler@ 1000ed00     useasm:useasm.obj
 0001:0000dd58       ??_C@_0FD@LADDBKEH@The?5destination?5for?5a?5SMP?5must?5b@ 1000ed58     useasm:useasm.obj
 0001:0000ddac       ??_C@_0CM@KHPAMMAK@The?5destination?5for?5an?5SMP?5can?8t@ 1000edac     useasm:useasm.obj
 0001:0000ddd8       ??_C@_0DC@EEBJMIBO@A?5?$CFs?5instruction?5can?8t?5be?5predic@ 1000edd8     useasm:useasm.obj
 0001:0000de0c       ??_C@_0DC@DNHACGFH@?4fcfill?5and?5?4bypassl1?5can?8t?5be?5s@ 1000ee0c     useasm:useasm.obj
 0001:0000de40       ??_C@_0DD@BEGMGHDH@?4bpcache?5and?5?4bypassl1?5can?8t?5be?5@ 1000ee40     useasm:useasm.obj
 0001:0000de74       ??_C@_0DB@JCFACDNN@?4bpcache?5and?5?4fcfill?5can?8t?5be?5sp@ 1000ee74     useasm:useasm.obj
 0001:0000dea8       ??_C@_0FD@KGBKPKPH@The?5last?5argument?5to?5a?5load?5inst@ 1000eea8     useasm:useasm.obj
 0001:0000defc       ??_C@_0CL@NHIEGIGG@The?5destination?5for?5an?5LD?5can?8t?5@ 1000eefc     useasm:useasm.obj
 0001:0000df28       ??_C@_0FD@DHDGKGAN@The?5destination?5for?5an?5LD?5must?5b@ 1000ef28     useasm:useasm.obj
 0001:0000df7c       ??_C@_0DD@ECJPHDDF@A?5load?1store?5can?8t?5be?5both?5pre?9?5@ 1000ef7c     useasm:useasm.obj
 0001:0000dfb0       ??_C@_0FC@LJJNHLCE@?$CFs?5can?8t?5be?5used?5with?5non?9pre?1po@ 1000efb0     useasm:useasm.obj
 0001:0000e008       ??_C@_0EN@GCEEDLLB@Pre?1post?9increment?5can?8t?5be?5spec@ 1000f008     useasm:useasm.obj
 0001:0000e058       ??_C@_0ED@IMFMHAAP@Source?51?5can?8t?5be?5immediate?5for?5@ 1000f058     useasm:useasm.obj
 0001:0000e09c       ??_C@_0CA@BFMOGGHL@?$CFs?5isn?8t?5supported?5on?5this?5core?$AA@ 1000f09c     useasm:useasm.obj
 0001:0000e0bc       ??_C@_0CJ@NLADGPEP@The?5argument?5to?5a?5branch?5must?5be@ 1000f0bc     useasm:useasm.obj
 0001:0000e0e8       ??_C@_0DD@COOIGJEM@Pn?5isn?8t?5a?5valid?5predicate?5for?5b@ 1000f0e8     useasm:useasm.obj
 0001:0000e11c       ??_C@_0DI@LKENEFMD@Only?5drc0?5can?5be?5used?5with?5PBE?5d@ 1000f11c     useasm:useasm.obj
 0001:0000e154       ??_C@_0BL@DDAKDDCD@Invalid?5data?5path?5selector?$AA@ 1000f154     useasm:useasm.obj
 0001:0000e170       ??_C@_0CM@EIBHGDCN@No?5flags?5are?5valid?5for?5a?5data?5pa@ 1000f170     useasm:useasm.obj
 0001:0000e19c       ??_C@_0CG@LCIGPPNF@A?5data?5path?5selector?5is?5not?5inde@ 1000f19c     useasm:useasm.obj
 0001:0000e1c4       ??_C@_0DI@IKADLPJL@The?5second?5argument?5to?5idf?5must?5@ 1000f1c4     useasm:useasm.obj
 0001:0000e1fc       ??_C@_0CG@BCCKICBA@The?5maximum?5drc?5register?5number?5@ 1000f1fc     useasm:useasm.obj
 0001:0000e224       ??_C@_0CG@NKPGJMIA@No?5flags?5are?5valid?5for?5a?5drc?5reg@ 1000f224     useasm:useasm.obj
 0001:0000e24c       ??_C@_0CA@BNCKADBN@A?5drc?5register?5is?5not?5indexable?$AA@ 1000f24c     useasm:useasm.obj
 0001:0000e26c       ??_C@_0DB@EIJIPLBA@The?5first?5argument?5to?5idf?5must?5b@ 1000f26c     useasm:useasm.obj
 0001:0000e2a0       ??_C@_0CL@HOIKEHND@The?5argument?5to?5wdf?5must?5be?5a?5dr@ 1000f2a0     useasm:useasm.obj
 0001:0000e2cc       ??_C@_0DI@ECFOFJCH@The?5last?5argument?5to?5an?5emit?5mus@ 1000f2cc     useasm:useasm.obj
 0001:0000e308       ??_C@_0EE@FPKMHEIB@The?5maximum?5immediate?5value?5for?5@ 1000f308     useasm:useasm.obj
 0001:0000e34c       ??_C@_0DJ@EENABCEN@The?5first?5argument?5to?5an?5emit?5mu@ 1000f34c     useasm:useasm.obj
 0001:0000e388       ??_C@_0CF@OIPADGLP@?$CFs?5isn?8t?5supported?5on?5this?5proce@ 1000f388     useasm:useasm.obj
 0001:0000e3b0       ??_C@_0CL@BLKOKIML@No?5flags?5are?5valid?5for?5argument?5@ 1000f3b0     useasm:useasm.obj
 0001:0000e3e0       ??_C@_0FK@GPIOMEID@Argument?5?$CFd?5to?5smoa?5is?5not?5a?5leg@ 1000f3e0     useasm:useasm.obj
 0001:0000e43c       ??_C@_0CM@OICCJGCF@Argument?5?$CFd?5to?5smoa?5must?5be?5an?5a@ 1000f43c     useasm:useasm.obj
 0001:0000e468       ??_C@_0CL@BPCDNEHJ@No?5flags?5are?5valid?5for?5argument?5@ 1000f468     useasm:useasm.obj
 0001:0000e494       ??_C@_0CF@KHLJFLDD@Argument?5?$CFd?5to?5smoa?5can?8t?5be?5ind@ 1000f494     useasm:useasm.obj
 0001:0000e4c0       ??_C@_0EB@LMPOCDMD@Argument?5?$CFd?5to?5smoa?5is?5out?5of?5ra@ 1000f4c0     useasm:useasm.obj
 0001:0000e504       ??_C@_0CP@JENPMIGB@Argument?5?$CFd?5to?5smoa?5must?5be?5an?5i@ 1000f504     useasm:useasm.obj
 0001:0000e538       ??_C@_0EI@CHCGIOOA@Loading?5the?5MOE?5state?5from?5regis@ 1000f538     useasm:useasm.obj
 0001:0000e580       ??_C@_0DA@OPFKEKGA@Argument?5?$CFd?5to?5smlsi?5should?5be?5a@ 1000f580     useasm:useasm.obj
 0001:0000e5b0       ??_C@_0EG@BJPEDDED@Argument?5?$CFd?5to?5smlsi?5is?5out?5of?5r@ 1000f5b0     useasm:useasm.obj
 0001:0000e5f8       ??_C@_0DA@FCAKILOF@Argument?5?$CFd?5to?5smlsi?5must?5be?5an?5@ 1000f5f8     useasm:useasm.obj
 0001:0000e628       ??_C@_0CM@LFIFLNIO@No?5flags?5are?5valid?5for?5argument?5@ 1000f628     useasm:useasm.obj
 0001:0000e654       ??_C@_0CG@PJFPKLPN@Argument?5?$CFd?5to?5smlsi?5can?8t?5be?5in@ 1000f654     useasm:useasm.obj
 0001:0000e67c       ??_C@_0DP@NNLBIBNI@Argument?5?$CFd?5to?5smlsi?5is?5out?5of?5r@ 1000f67c     useasm:useasm.obj
 0001:0000e6bc       ??_C@_0CL@MJEEEJFH@Argument?5?$CFd?5to?5smlsi?5isn?8t?5a?5val@ 1000f6bc     useasm:useasm.obj
 0001:0000e6e8       ??_C@_0DM@BDMFEIMC@Argument?5?$CFd?5uses?5component?5selec@ 1000f6e8     useasm:useasm.obj
 0001:0000e724       ??_C@_0DN@CBDPLAND@Argument?5?$CFd?5to?5smlsi?5must?5be?5an?5@ 1000f724     useasm:useasm.obj
 0001:0000e768       ??_C@_0EH@PIBJEHLO@Loading?5the?5MOE?5state?5from?5regis@ 1000f768     useasm:useasm.obj
 0001:0000e7b0       ??_C@_0CD@DAICKOIL@Argument?5?$CFd?5to?5?$CFs?5can?8t?5be?5index@ 1000f7b0     useasm:useasm.obj
 0001:0000e7d4       ??_C@_0DL@DAGJDBAJ@Argument?5?$CFd?5to?5?$CFs?5is?5out?5of?5rang@ 1000f7d4     useasm:useasm.obj
 0001:0000e810       ??_C@_0DN@OPLIFLFN@Argument?5?$CFd?5to?5imo?5is?5out?5of?5ran@ 1000f810     useasm:useasm.obj
 0001:0000e850       ??_C@_0DH@LBKJPHME@Argument?5?$CFd?5to?5smr?1smbo?1imo?5must@ 1000f850     useasm:useasm.obj
 0001:0000e888       ??_C@_0EC@LGDHIHKO@Loading?5the?5MOE?5state?5from?5regis@ 1000f888     useasm:useasm.obj
 0001:0000e8cc       ??_C@_03PKDHGMJG@smr?$AA@  1000f8cc     useasm:useasm.obj
 0001:0000e8d0       ??_C@_04OHNFNFAF@smbo?$AA@ 1000f8d0     useasm:useasm.obj
 0001:0000e8d8       ??_C@_03DKPPLHHB@imo?$AA@  1000f8d8     useasm:useasm.obj
 0001:0000e8dc       ??_C@_0CM@PAFKAACO@No?5flags?5are?5valid?5for?5argument?5@ 1000f8dc     useasm:useasm.obj
 0001:0000e908       ??_C@_0CG@JIFDPGCJ@Argument?5?$CFd?5to?5setfc?5can?8t?5be?5in@ 1000f908     useasm:useasm.obj
 0001:0000e930       ??_C@_0DA@FIKLGADO@Argument?5?$CFd?5to?5setfc?5is?5must?5be?5@ 1000f930     useasm:useasm.obj
 0001:0000e960       ??_C@_0DA@PNIDFAOJ@Argument?5?$CFd?5to?5setfc?5must?5be?5an?5@ 1000f960     useasm:useasm.obj
 0001:0000e990       ??_C@_0DC@IGFMAGID@Only?5?$CFd?5mutex?$CIes?$CJ?5are?5supported?5@ 1000f990     useasm:useasm.obj
 0001:0000e9c4       ??_C@_0CE@FKFABDHJ@An?5immediate?5value?5can?8t?5be?5inde@ 1000f9c4     useasm:useasm.obj
 0001:0000e9e8       ??_C@_0CK@FKJKMHCB@No?5flags?5are?5valid?5for?5the?5argum@ 1000f9e8     useasm:useasm.obj
 0001:0000ea14       ??_C@_0CI@GKLFIIMC@The?5argument?5to?5?$CFs?5must?5be?5an?5im@ 1000fa14     useasm:useasm.obj
 0001:0000ea40       ??_C@_0EI@IMBJAMEN@The?5maximum?5immediate?5value?5for?5@ 1000fa40     useasm:useasm.obj
 0001:0000ea88       ??_C@_0DB@KGKPELKC@The?5third?5argument?5to?5ldr?5must?5b@ 1000fa88     useasm:useasm.obj
 0001:0000eac0       ??_C@_0EP@HFAIINHO@The?5destination?5for?5ldr?5must?5be?5@ 1000fac0     useasm:useasm.obj
 0001:0000eb10       ??_C@_0CJ@PBDIHBBP@The?5destination?5for?5ldr?5can?8t?5be@ 1000fb10     useasm:useasm.obj
 0001:0000eb3c       ??_C@_0DP@EOJFCBDD@The?5seventh?5argument?5to?5atst8?5mu@ 1000fb3c     useasm:useasm.obj
 0001:0000eb7c       ??_C@_0DC@GPFGCALA@An?5integer?5source?5selector?5value@ 1000fb7c     useasm:useasm.obj
 0001:0000ebb0       ??_C@_0DM@KLBODCDM@The?5sixth?5argument?5to?5atst8?5must@ 1000fbb0     useasm:useasm.obj
 0001:0000ebf0       ??_C@_0EF@HHNKPNHB@No?5flags?5except?5disable?5writebac@ 1000fbf0     useasm:useasm.obj
 0001:0000ec38       ??_C@_0CG@EAILMAJF@A?5predicate?5register?5is?5not?5inde@ 1000fc38     useasm:useasm.obj
 0001:0000ec60       ??_C@_0DP@IJEBNLPN@The?5destination?5argument?5to?5atst@ 1000fc60     useasm:useasm.obj
 0001:0000eca0       ??_C@_0DJ@CANNFGLC@The?5fifth?5argument?5to?5depthf?5mus@ 1000fca0     useasm:useasm.obj
 0001:0000ecdc       ??_C@_0DO@JJIFGFHO@The?5fourth?5argument?5to?5depthf?5mu@ 1000fcdc     useasm:useasm.obj
 0001:0000ed1c       ??_C@_0DG@DJLDOPBE@The?5maximum?5monitor?5supported?5on@ 1000fd1c     useasm:useasm.obj
 0001:0000ed54       ??_C@_0CM@EANNIMNI@Monitors?5aren?8t?5supported?5on?5thi@ 1000fd54     useasm:useasm.obj
 0001:0000ed80       ??_C@_0DA@NGKNOLIJ@The?5argument?5to?5setm?5must?5be?5an?5@ 1000fd80     useasm:useasm.obj
 0001:0000edb0       ??_C@_0CK@FLEIDBJB@The?5maximum?5immediate?5value?5for?5@ 1000fdb0     useasm:useasm.obj
 0001:0000eddc       ??_C@_0CP@KDAJINNH@The?5argument?5to?5wop?5must?5be?5an?5i@ 1000fddc     useasm:useasm.obj
 0001:0000ee0c       ??_C@_0BE@CMNIOOMH@Unknown?5instruction?$AA@ 1000fe0c     useasm:useasm.obj
 0001:0000ee20       ??_C@_0BN@FNBEMNH@?$CFs?5should?5have?5been?5coissued?$AA@ 1000fe20     useasm:useasm.obj
 0001:0000ee40       ??_C@_0BI@KBNBGPKO@Label?5?$CFs?5is?5not?5defined?$AA@ 1000fe40     useasm:useasm.obj
 0001:0000ee58       ??_C@_05NCHGGDHJ@sprvv?$AA@ 1000fe58     useasm:usetab.obj
 0001:0000ee60       ??_C@_06HFBPFKMP@idxscw?$AA@ 1000fe60     useasm:usetab.obj
 0001:0000ee68       ??_C@_06IGIKOIK@idxscr?$AA@ 1000fe68     useasm:usetab.obj
 0001:0000ee70       ??_C@_0L@JLOMIJPI@vpckc10c10?$AA@ 1000fe70     useasm:usetab.obj
 0001:0000ee7c       ??_C@_0M@ECFENLNA@vpckfc10f32?$AA@ 1000fe7c     useasm:usetab.obj
 0001:0000ee88       ??_C@_0L@PKGINOEM@vpckc10f16?$AA@ 1000fe88     useasm:usetab.obj
 0001:0000ee94       ??_C@_0L@PONMFEDE@vpckf32c10?$AA@ 1000fe94     useasm:usetab.obj
 0001:0000eea0       ??_C@_0L@PILABCOK@vpckf32f32?$AA@ 1000fea0     useasm:usetab.obj
 0001:0000eeac       ??_C@_0L@JPFIADIA@vpckf32f16?$AA@ 1000feac     useasm:usetab.obj
 0001:0000eeb8       ??_C@_0L@PIJPKECN@vpckf32s16?$AA@ 1000feb8     useasm:usetab.obj
 0001:0000eec4       ??_C@_0L@NNPEPLPB@vpckf32u16?$AA@ 1000fec4     useasm:usetab.obj
 0001:0000eed0       ??_C@_09PGEODABJ@vpckf32o8?$AA@ 1000fed0     useasm:usetab.obj
 0001:0000eedc       ??_C@_09ODHCGKAN@vpckf32s8?$AA@ 1000fedc     useasm:usetab.obj
 0001:0000eee8       ??_C@_08OHIHMNPI@vpckf2u8?$AA@ 1000fee8     useasm:usetab.obj
 0001:0000eef4       ??_C@_0L@EGJEFDPP@vpckf16c10?$AA@ 1000fef4     useasm:usetab.obj
 0001:0000ef00       ??_C@_0L@EAPIBFCB@vpckf16f32?$AA@ 1000ff00     useasm:usetab.obj
 0001:0000ef0c       ??_C@_0L@CHBAAEEL@vpckf16f16?$AA@ 1000ff0c     useasm:usetab.obj
 0001:0000ef18       ??_C@_0L@EANHKDOG@vpckf16s16?$AA@ 1000ff18     useasm:usetab.obj
 0001:0000ef24       ??_C@_0L@GFLMPMDK@vpckf16u16?$AA@ 1000ff24     useasm:usetab.obj
 0001:0000ef30       ??_C@_09DOMPECO@vpckf16o8?$AA@ 1000ff30     useasm:usetab.obj
 0001:0000ef3c       ??_C@_09BGNAKODK@vpckf16s8?$AA@ 1000ff3c     useasm:usetab.obj
 0001:0000ef48       ??_C@_09BCFNNCII@vpckf16u8?$AA@ 1000ff48     useasm:usetab.obj
 0001:0000ef54       ??_C@_0M@MABDAOCA@vpcks16sf32?$AA@ 1000ff54     useasm:usetab.obj
 0001:0000ef60       ??_C@_0L@BCPGLHCC@vpcks16f16?$AA@ 1000ff60     useasm:usetab.obj
 0001:0000ef6c       ??_C@_0L@HFDBBAIP@vpcks16s16?$AA@ 1000ff6c     useasm:usetab.obj
 0001:0000ef78       ??_C@_0L@FAFKEPFD@vpcks16u16?$AA@ 1000ff78     useasm:usetab.obj
 0001:0000ef84       ??_C@_09FAPHGHAG@vpcks16o8?$AA@ 1000ff84     useasm:usetab.obj
 0001:0000ef90       ??_C@_09EFMLDNBC@vpcks16s8?$AA@ 1000ff90     useasm:usetab.obj
 0001:0000ef9c       ??_C@_09EBEGEBKA@vpcks16u8?$AA@ 1000ff9c     useasm:usetab.obj
 0001:0000efa8       ??_C@_0M@GHMAHKH@vpcku16sf32?$AA@ 1000ffa8     useasm:usetab.obj
 0001:0000efb4       ??_C@_0L@HBCGICBI@vpcku16f16?$AA@ 1000ffb4     useasm:usetab.obj
 0001:0000efc0       ??_C@_0L@BGOBCFLF@vpcku16s16?$AA@ 1000ffc0     useasm:usetab.obj
 0001:0000efcc       ??_C@_0L@DDIKHKGJ@vpcku16u16?$AA@ 1000ffcc     useasm:usetab.obj
 0001:0000efd8       ??_C@_09IGKOIEBL@vpcku16o8?$AA@ 1000ffd8     useasm:usetab.obj
 0001:0000efe4       ??_C@_09JDJCNOAP@vpcku16s8?$AA@ 1000ffe4     useasm:usetab.obj
 0001:0000eff0       ??_C@_09JHBPKCLN@vpcku16u8?$AA@ 1000fff0     useasm:usetab.obj
 0001:0000effc       ??_C@_0L@GCHMNGAD@vpcko8sf32?$AA@ 1000fffc     useasm:usetab.obj
 0001:0000f008       ??_C@_09BKFPOGAB@vpcko8f16?$AA@ 10010008     useasm:usetab.obj
 0001:0000f014       ??_C@_09HNJIEBKM@vpcko8s16?$AA@ 10010014     useasm:usetab.obj
 0001:0000f020       ??_C@_09FIPDBOHA@vpcko8u16?$AA@ 10010020     useasm:usetab.obj
 0001:0000f02c       ??_C@_08JEJLGJEL@vpcko8o8?$AA@ 1001002c     useasm:usetab.obj
 0001:0000f038       ??_C@_08IBKHDDFP@vpcko8s8?$AA@ 10010038     useasm:usetab.obj
 0001:0000f044       ??_C@_08IFCKEPON@vpcko8u8?$AA@ 10010044     useasm:usetab.obj
 0001:0000f050       ??_C@_0L@MCACCALJ@vpcks8sf32?$AA@ 10010050     useasm:usetab.obj
 0001:0000f05c       ??_C@_09GOELCEOB@vpcks8f16?$AA@ 1001005c     useasm:usetab.obj
 0001:0000f068       ??_C@_09JIMIDEM@vpcks8s16?$AA@ 10010068     useasm:usetab.obj
 0001:0000f074       ??_C@_09CMOHNMJA@vpcks8u16?$AA@ 10010074     useasm:usetab.obj
 0001:0000f080       ??_C@_08DBILBDMI@vpcks8o8?$AA@ 10010080     useasm:usetab.obj
 0001:0000f08c       ??_C@_08CELHEJNM@vpcks8s8?$AA@ 1001008c     useasm:usetab.obj
 0001:0000f098       ??_C@_08CADKDFGO@vpcks8u8?$AA@ 10010098     useasm:usetab.obj
 0001:0000f0a4       ??_C@_0L@KBNCBFID@vpcku8sf32?$AA@ 100100a4     useasm:usetab.obj
 0001:0000f0b0       ??_C@_09LIBCMHPM@vpcku8f16?$AA@ 100100b0     useasm:usetab.obj
 0001:0000f0bc       ??_C@_09NPNFGAFB@vpcku8s16?$AA@ 100100bc     useasm:usetab.obj
 0001:0000f0c8       ??_C@_09PKLODPIN@vpcku8u16?$AA@ 100100c8     useasm:usetab.obj
 0001:0000f0d4       ??_C@_08LOMLOGGI@vpcku8o8?$AA@ 100100d4     useasm:usetab.obj
 0001:0000f0e0       ??_C@_08KLPHLMHM@vpcku8s8?$AA@ 100100e0     useasm:usetab.obj
 0001:0000f0ec       ??_C@_08KPHKMAMO@vpcku8u8?$AA@ 100100ec     useasm:usetab.obj
 0001:0000f0f8       ??_C@_04DGGKFKKC@vexp?$AA@ 100100f8     useasm:usetab.obj
 0001:0000f100       ??_C@_04FHIICEEL@vlog?$AA@ 10010100     useasm:usetab.obj
 0001:0000f108       ??_C@_04OOOKOLCE@vrsq?$AA@ 10010108     useasm:usetab.obj
 0001:0000f110       ??_C@_04OLNHHJBF@vrcp?$AA@ 10010110     useasm:usetab.obj
 0001:0000f118       ??_C@_06BKGGAFJG@vf16dp?$AA@ 10010118     useasm:usetab.obj
 0001:0000f120       ??_C@_07JOHMCFEH@vf16max?$AA@ 10010120     useasm:usetab.obj
 0001:0000f128       ??_C@_07IMPHMBCI@vf16min?$AA@ 10010128     useasm:usetab.obj
 0001:0000f130       ??_C@_07OFMNCMJC@vf16dsy?$AA@ 10010130     useasm:usetab.obj
 0001:0000f138       ??_C@_07PMNGBNND@vf16dsx?$AA@ 10010138     useasm:usetab.obj
 0001:0000f140       ??_C@_07POCLHEPF@vf16frc?$AA@ 10010140     useasm:usetab.obj
 0001:0000f148       ??_C@_07DEBGAFEJ@vf16add?$AA@ 10010148     useasm:usetab.obj
 0001:0000f150       ??_C@_07KLPNPJLO@vf16mul?$AA@ 10010150     useasm:usetab.obj
 0001:0000f158       ??_C@_07HIALHIBK@vf16mad?$AA@ 10010158     useasm:usetab.obj
 0001:0000f160       ??_C@_03PAAOMFKJ@vdp?$AA@  10010160     useasm:usetab.obj
 0001:0000f164       ??_C@_04FDEBGJGP@vdsy?$AA@ 10010164     useasm:usetab.obj
 0001:0000f16c       ??_C@_04EKFKFICO@vdsx?$AA@ 1001016c     useasm:usetab.obj
 0001:0000f174       ??_C@_04CIPAGALK@vmax?$AA@ 10010174     useasm:usetab.obj
 0001:0000f17c       ??_C@_04DKHLIENF@vmin?$AA@ 1001017c     useasm:usetab.obj
 0001:0000f184       ??_C@_04EIKHDBAI@vfrc?$AA@ 10010184     useasm:usetab.obj
 0001:0000f18c       ??_C@_04ICJKEALE@vadd?$AA@ 1001018c     useasm:usetab.obj
 0001:0000f194       ??_C@_04BNHBLMED@vmul?$AA@ 10010194     useasm:usetab.obj
 0001:0000f19c       ??_C@_04MOIHDNOH@vmad?$AA@ 1001019c     useasm:usetab.obj
 0001:0000f1a4       ??_C@_07PJIFHDOJ@vmovcu8?$AA@ 100101a4     useasm:usetab.obj
 0001:0000f1ac       ??_C@_05IPANMIKP@vmovc?$AA@ 100101ac     useasm:usetab.obj
 0001:0000f1b4       ??_C@_04LMONGADO@vmov?$AA@ 100101b4     useasm:usetab.obj
 0001:0000f1bc       ??_C@_05HKPHADDM@vmov4?$AA@ 100101bc     useasm:usetab.obj
 0001:0000f1c4       ??_C@_05DFLGJFPL@vmov3?$AA@ 100101c4     useasm:usetab.obj
 0001:0000f1cc       ??_C@_05LKKHNEHN@vssq4?$AA@ 100101cc     useasm:usetab.obj
 0001:0000f1d4       ??_C@_05PFOGECLK@vssq3?$AA@ 100101d4     useasm:usetab.obj
 0001:0000f1dc       ??_C@_05IBKMJGII@vsub4?$AA@ 100101dc     useasm:usetab.obj
 0001:0000f1e4       ??_C@_05MOONAAEP@vsub3?$AA@ 100101e4     useasm:usetab.obj
 0001:0000f1ec       ??_C@_05HHKEBOCC@vadd4?$AA@ 100101ec     useasm:usetab.obj
 0001:0000f1f4       ??_C@_05DIOFIIOF@vadd3?$AA@ 100101f4     useasm:usetab.obj
 0001:0000f1fc       ??_C@_05FEOCJCGB@vmul4?$AA@ 100101fc     useasm:usetab.obj
 0001:0000f204       ??_C@_05BLKDAEKG@vmul3?$AA@ 10010204     useasm:usetab.obj
 0001:0000f20c       ??_C@_05IFIKADBB@vmad4?$AA@ 1001020c     useasm:usetab.obj
 0001:0000f214       ??_C@_05MKMLJFNG@vmad3?$AA@ 10010214     useasm:usetab.obj
 0001:0000f21c       ??_C@_04BENAOGHO@vdp4?$AA@ 1001021c     useasm:usetab.obj
 0001:0000f224       ??_C@_04FLJBHALJ@vdp3?$AA@ 10010224     useasm:usetab.obj
 0001:0000f22c       ??_C@_0N@JGJIGCK@emitvcbstate?$AA@ 1001022c     useasm:usetab.obj
 0001:0000f23c       ??_C@_0O@IBKGEAGF@emitvcbvertex?$AA@ 1001023c     useasm:usetab.obj
 0001:0000f24c       ??_C@_0N@JECFFMDK@emitmtestate?$AA@ 1001024c     useasm:usetab.obj
 0001:0000f25c       ??_C@_0O@JMIMBMNL@emitmtevertex?$AA@ 1001025c     useasm:usetab.obj
 0001:0000f26c       ??_C@_03PENBPHC@cfi?$AA@   1001026c     useasm:usetab.obj
 0001:0000f270       ??_C@_02POBAIDHK@ci?$AA@   10010270     useasm:usetab.obj
 0001:0000f274       ??_C@_02HJIIJPLF@cf?$AA@   10010274     useasm:usetab.obj
 0001:0000f278       ??_C@_05PACJMPIO@moest?$AA@ 10010278     useasm:usetab.obj
 0001:0000f280       ??_C@_06FOOALFNH@fnrm16?$AA@ 10010280     useasm:usetab.obj
 0001:0000f288       ??_C@_06DJAIKELN@fnrm32?$AA@ 10010288     useasm:usetab.obj
 0001:0000f290       ??_C@_06KNGBBCNH@sablnd?$AA@ 10010290     useasm:usetab.obj
 0001:0000f298       ??_C@_06DPIIDNJL@fpsub8?$AA@ 10010298     useasm:usetab.obj
 0001:0000f2a0       ??_C@_06MJIALFDB@fpadd8?$AA@ 100102a0     useasm:usetab.obj
 0001:0000f2a8       ??_C@_06OKMGDJHC@fpmul8?$AA@ 100102a8     useasm:usetab.obj
 0001:0000f2b0       ??_C@_06BELDBAKP@isubu8?$AA@ 100102b0     useasm:usetab.obj
 0001:0000f2b8       ??_C@_06CCEGFCNB@iaddu8?$AA@ 100102b8     useasm:usetab.obj
 0001:0000f2c0       ??_C@_04HIHJCIAG@fpma?$AA@ 100102c0     useasm:usetab.obj
 0001:0000f2c8       ??_C@_06BODAOOPP@movmsk?$AA@ 100102c8     useasm:usetab.obj
 0001:0000f2d0       ??_C@_04CFJGHAMN@movc?$AA@ 100102d0     useasm:usetab.obj
 0001:0000f2d8       ??_C@_07MKEAMJFF@padding?$AA@ 100102d8     useasm:usetab.obj
 0001:0000f2e0       ??_C@_07BANDBPIA@iaddu32?$AA@ 100102e0     useasm:usetab.obj
 0001:0000f2e8       ??_C@_06DBFEDEDN@imov16?$AA@ 100102e8     useasm:usetab.obj
 0001:0000f2f0       ??_C@_06MNLAAEHH@imulu8?$AA@ 100102f0     useasm:usetab.obj
 0001:0000f2f8       ??_C@_05KNHGNCD@imul8?$AA@ 100102f8     useasm:usetab.obj
 0001:0000f300       ??_C@_05NPJJGJMK@isub8?$AA@ 10010300     useasm:usetab.obj
 0001:0000f308       ??_C@_05CJJBOBGA@iadd8?$AA@ 10010308     useasm:usetab.obj
 0001:0000f310       ??_C@_06KMLOELCJ@iadd32?$AA@ 10010310     useasm:usetab.obj
 0001:0000f318       ??_C@_07EIGBPOGB@imulu16?$AA@ 10010318     useasm:usetab.obj
 0001:0000f320       ??_C@_07MALAKHJD@isubu16?$AA@ 10010320     useasm:usetab.obj
 0001:0000f328       ??_C@_07HHDLAOOK@iaddu16?$AA@ 10010328     useasm:usetab.obj
 0001:0000f330       ??_C@_06CEKAAMOF@imul16?$AA@ 10010330     useasm:usetab.obj
 0001:0000f338       ??_C@_06PNKDBIDN@isub16?$AA@ 10010338     useasm:usetab.obj
 0001:0000f340       ??_C@_06MLFGFKED@iadd16?$AA@ 10010340     useasm:usetab.obj
 0001:0000f348       ??_C@_05OJCDMDMI@asop2?$AA@ 10010348     useasm:usetab.obj
 0001:0000f350       ??_C@_04BNKIMGJI@lrp2?$AA@ 10010350     useasm:usetab.obj
 0001:0000f358       ??_C@_04DGIFJFFL@lrp1?$AA@ 10010358     useasm:usetab.obj
 0001:0000f360       ??_C@_04JEDFNLGM@alrp?$AA@ 10010360     useasm:usetab.obj
 0001:0000f368       ??_C@_05BLLJMLJF@arsop?$AA@ 10010368     useasm:usetab.obj
 0001:0000f370       ??_C@_04IILBKMIG@asop?$AA@ 10010370     useasm:usetab.obj
 0001:0000f378       ??_C@_04OBPEPKPD@asub?$AA@ 10010378     useasm:usetab.obj
 0001:0000f380       ??_C@_04FAFKALCG@aadd?$AA@ 10010380     useasm:usetab.obj
 0001:0000f388       ??_C@_07NOKJPFJG@aintrp2?$AA@ 10010388     useasm:usetab.obj
 0001:0000f390       ??_C@_07PFIEKGFF@aintrp1?$AA@ 10010390     useasm:usetab.obj
 0001:0000f398       ??_C@_04HDJKLMOD@phas?$AA@ 10010398     useasm:usetab.obj
 0001:0000f3a0       ??_C@_04IPMEAKK@setm?$AA@  100103a0     useasm:usetab.obj
 0001:0000f3a8       ??_C@_03EEOHENCN@wop?$AA@  100103a8     useasm:usetab.obj
 0001:0000f3ac       ??_C@_06CNLPFHCD@depthf?$AA@ 100103ac     useasm:usetab.obj
 0001:0000f3b4       ??_C@_05LMCKLHKJ@atst8?$AA@ 100103b4     useasm:usetab.obj
 0001:0000f3bc       ??_C@_05FFPFIJHE@ptoff?$AA@ 100103bc     useasm:usetab.obj
 0001:0000f3c4       ??_C@_06GIPMBBEA@pcoeff?$AA@ 100103c4     useasm:usetab.obj
 0001:0000f3cc       ??_C@_03OJMAPEGJ@str?$AA@  100103cc     useasm:usetab.obj
 0001:0000f3d0       ??_C@_03PNJMBANA@ldr?$AA@  100103d0     useasm:usetab.obj
 0001:0000f3d4       ??_C@_07KLENHKKM@fsubflr?$AA@ 100103d4     useasm:usetab.obj
 0001:0000f3dc       ??_C@_07EOGFDLKI@release?$AA@ 100103dc     useasm:usetab.obj
 0001:0000f3e4       ??_C@_04MKMCLCOO@lock?$AA@ 100103e4     useasm:usetab.obj
 0001:0000f3ec       ??_C@_06OPKGODIN@fddpc4?$AA@ 100103ec     useasm:usetab.obj
 0001:0000f3f4       ??_C@_06KAOHHFEK@fddpc3?$AA@ 100103f4     useasm:usetab.obj
 0001:0000f3fc       ??_C@_05FCEHFDPG@fddpc?$AA@ 100103fc     useasm:usetab.obj
 0001:0000f404       ??_C@_05KHLNJIGF@fddp4?$AA@ 10010404     useasm:usetab.obj
 0001:0000f40c       ??_C@_05OIPMAOKC@fddp3?$AA@ 1001040c     useasm:usetab.obj
 0001:0000f414       ??_C@_04PLAKPAFB@fddp?$AA@ 10010414     useasm:usetab.obj
 0001:0000f41c       ??_C@_05GGKGEFIE@fdpc4?$AA@ 1001041c     useasm:usetab.obj
 0001:0000f424       ??_C@_05CJOHNDED@fdpc3?$AA@ 10010424     useasm:usetab.obj
 0001:0000f42c       ??_C@_04IBMKLKGP@fdpc?$AA@ 1001042c     useasm:usetab.obj
 0001:0000f434       ??_C@_04HEDAHBPM@fdp4?$AA@ 10010434     useasm:usetab.obj
 0001:0000f43c       ??_C@_04DLHBOHDL@fdp3?$AA@ 1001043c     useasm:usetab.obj
 0001:0000f444       ??_C@_05HEIOGBDD@setfc?$AA@ 10010444     useasm:usetab.obj
 0001:0000f44c       ??_C@_04PKDBBMEC@smso?$AA@ 1001044c     useasm:usetab.obj
 0001:0000f454       ??_C@_04HFADBHGK@smia?$AA@ 10010454     useasm:usetab.obj
 0001:0000f45c       ??_C@_06EOEAAGLO@u16tnz?$AA@ 1001045c     useasm:usetab.obj
 0001:0000f464       ??_C@_05NKPLKFJF@u16tz?$AA@ 10010464     useasm:usetab.obj
 0001:0000f46c       ??_C@_04FMGLMKJC@ftnz?$AA@ 1001046c     useasm:usetab.obj
 0001:0000f474       ??_C@_03EGNONJMM@ftz?$AA@  10010474     useasm:usetab.obj
 0001:0000f478       ??_C@_03GJPGFFDI@nop?$AA@  10010478     useasm:usetab.obj
 0001:0000f47c       ??_C@_03FGBGECCC@dma?$AA@  1001047c     useasm:usetab.obj
 0001:0000f480       ??_C@_03ODCMFNNH@sms?$AA@  10010480     useasm:usetab.obj
 0001:0000f484       ??_C@_03BJDMMCMD@ams?$AA@  10010484     useasm:usetab.obj
 0001:0000f488       ??_C@_03DHGNGCAI@smm?$AA@  10010488     useasm:usetab.obj
 0001:0000f48c       ??_C@_03MNHNPNBM@amm?$AA@  1001048c     useasm:usetab.obj
 0001:0000f490       ??_C@_03JEAJBGIL@sda?$AA@  10010490     useasm:usetab.obj
 0001:0000f494       ??_C@_03DILMFJIH@sdm?$AA@  10010494     useasm:usetab.obj
 0001:0000f498       ??_C@_07KLCMLLPD@setpneq?$AA@ 10010498     useasm:usetab.obj
 0001:0000f4a0       ??_C@_07DCGPGNGK@setplte?$AA@ 100104a0     useasm:usetab.obj
 0001:0000f4a8       ??_C@_06IKNJBMPL@setplt?$AA@ 100104a8     useasm:usetab.obj
 0001:0000f4b0       ??_C@_06PIHPNDDB@setpeq?$AA@ 100104b0     useasm:usetab.obj
 0001:0000f4b8       ??_C@_07OFGOOKGL@setpgte?$AA@ 100104b8     useasm:usetab.obj
 0001:0000f4c0       ??_C@_06IGIMPDBK@setpgt?$AA@ 100104c0     useasm:usetab.obj
 0001:0000f4c8       ??_C@_04FDNECGOD@fsub?$AA@ 100104c8     useasm:usetab.obj
 0001:0000f4d0       ??_C@_04DGLGBLMD@fssq?$AA@ 100104d0     useasm:usetab.obj
 0001:0000f4d8       ??_C@_04OCHKNHDG@fadd?$AA@ 100104d8     useasm:usetab.obj
 0001:0000f4e0       ??_C@_04HNJBCLMB@fmul?$AA@ 100104e0     useasm:usetab.obj
 0001:0000f4e8       ??_C@_04NMANPHLM@fmov?$AA@ 100104e8     useasm:usetab.obj
 0001:0000f4f0       ??_C@_03CNBJFNFA@mov?$AA@  100104f0     useasm:usetab.obj
 0001:0000f4f4       ??_C@_07OLONFCKE@emitpds?$AA@ 100104f4     useasm:usetab.obj
 0001:0000f4fc       ??_C@_0O@LEENHJNO@emitprimitive?$AA@ 100104fc     useasm:usetab.obj
 0001:0000f50c       ??_C@_0L@FAAMFGJF@emitvertex?$AA@ 1001050c     useasm:usetab.obj
 0001:0000f518       ??_C@_09BIBIIHIO@emitstate?$AA@ 10010518     useasm:usetab.obj
 0001:0000f524       ??_C@_0L@ODEMBHIP@emitpixel2?$AA@ 10010524     useasm:usetab.obj
 0001:0000f530       ??_C@_0L@MIGBEEEM@emitpixel1?$AA@ 10010530     useasm:usetab.obj
 0001:0000f53c       ??_C@_03FECKBHBL@wdf?$AA@  1001053c     useasm:usetab.obj
 0001:0000f540       ??_C@_03OEOMDHLH@idf?$AA@  10010540     useasm:usetab.obj
 0001:0000f544       ??_C@_0L@JODEDCHK@bexception?$AA@ 10010544     useasm:usetab.obj
 0001:0000f550       ??_C@_04PMKEFCPM@lapc?$AA@ 10010550     useasm:usetab.obj
 0001:0000f558       ??_C@_02FGOECCNH@br?$AA@   10010558     useasm:usetab.obj
 0001:0000f55c       ??_C@_02DHALGDEF@ba?$AA@   1001055c     useasm:usetab.obj
 0001:0000f560       ??_C@_04GAAFJDCP@eldq?$AA@ 10010560     useasm:usetab.obj
 0001:0000f568       ??_C@_04FHLAHFDL@eldd?$AA@ 10010568     useasm:usetab.obj
 0001:0000f570       ??_C@_04GCOCNAN@sttq?$AA@  10010570     useasm:usetab.obj
 0001:0000f578       ??_C@_04DBJLMLBJ@sttd?$AA@ 10010578     useasm:usetab.obj
 0001:0000f580       ??_C@_04FAHEIKIL@sttw?$AA@ 10010580     useasm:usetab.obj
 0001:0000f588       ??_C@_04GHMBGMJP@sttb?$AA@ 10010588     useasm:usetab.obj
 0001:0000f590       ??_C@_04LEIHHKMB@ldtq?$AA@ 10010590     useasm:usetab.obj
 0001:0000f598       ??_C@_04IDDCJMNF@ldtd?$AA@ 10010598     useasm:usetab.obj
 0001:0000f5a0       ??_C@_04OCNNNNEH@ldtw?$AA@ 100105a0     useasm:usetab.obj
 0001:0000f5a8       ??_C@_04NFGIDLFD@ldtb?$AA@ 100105a8     useasm:usetab.obj
 0001:0000f5b0       ??_C@_04BEBLNPMF@stlq?$AA@ 100105b0     useasm:usetab.obj
 0001:0000f5b8       ??_C@_04CDKODJNB@stld?$AA@ 100105b8     useasm:usetab.obj
 0001:0000f5c0       ??_C@_04ECEBHIED@stlw?$AA@ 100105c0     useasm:usetab.obj
 0001:0000f5c8       ??_C@_04HFPEJOFH@stlb?$AA@ 100105c8     useasm:usetab.obj
 0001:0000f5d0       ??_C@_04KGLCIIAJ@ldlq?$AA@ 100105d0     useasm:usetab.obj
 0001:0000f5d8       ??_C@_04JBAHGOBN@ldld?$AA@ 100105d8     useasm:usetab.obj
 0001:0000f5e0       ??_C@_04PAOICPIP@ldlw?$AA@ 100105e0     useasm:usetab.obj
 0001:0000f5e8       ??_C@_04MHFNMJJL@ldlb?$AA@ 100105e8     useasm:usetab.obj
 0001:0000f5f0       ??_C@_04BMMDEMJG@staq?$AA@ 100105f0     useasm:usetab.obj
 0001:0000f5f8       ??_C@_04CLHGKKIC@stad?$AA@ 100105f8     useasm:usetab.obj
 0001:0000f600       ??_C@_04EKJJOLBA@staw?$AA@ 10010600     useasm:usetab.obj
 0001:0000f608       ??_C@_04HNCMANAE@stab?$AA@ 10010608     useasm:usetab.obj
 0001:0000f610       ??_C@_04KOGKBLFK@ldaq?$AA@ 10010610     useasm:usetab.obj
 0001:0000f618       ??_C@_04JJNPPNEO@ldad?$AA@ 10010618     useasm:usetab.obj
 0001:0000f620       ??_C@_04PIDALMNM@ldaw?$AA@ 10010620     useasm:usetab.obj
 0001:0000f628       ??_C@_04MPIFFKMI@ldab?$AA@ 10010628     useasm:usetab.obj
 0001:0000f630       ??_C@_09KIDJGAAM@smp3dgrad?$AA@ 10010630     useasm:usetab.obj
 0001:0000f63c       ??_C@_09OEOGLLI@smp2dgrad?$AA@ 1001063c     useasm:usetab.obj
 0001:0000f648       ??_C@_09DPKGHBCF@smp1dgrad?$AA@ 10010648     useasm:usetab.obj
 0001:0000f654       ??_C@_0N@IMLLGHGO@smp3dreplace?$AA@ 10010654     useasm:usetab.obj
 0001:0000f664       ??_C@_0N@GDHJAMFA@smp2dreplace?$AA@ 10010664     useasm:usetab.obj
 0001:0000f674       ??_C@_0N@IIEOLHFD@smp1dreplace?$AA@ 10010674     useasm:usetab.obj
 0001:0000f684       ??_C@_09OCECLLHE@smp3dbias?$AA@ 10010684     useasm:usetab.obj
 0001:0000f690       ??_C@_09EEDFLAMA@smp2dbias?$AA@ 10010690     useasm:usetab.obj
 0001:0000f69c       ??_C@_09HFNNKKFN@smp1dbias?$AA@ 1001069c     useasm:usetab.obj
 0001:0000f6a8       ??_C@_05OOKKMHDJ@smp3d?$AA@ 100106a8     useasm:usetab.obj
 0001:0000f6b0       ??_C@_05OPGIKNAO@smp2d?$AA@ 100106b0     useasm:usetab.obj
 0001:0000f6b8       ??_C@_05ONCOBDFH@smp1d?$AA@ 100106b8     useasm:usetab.obj
 0001:0000f6c0       ??_C@_06GGGOMLOL@ssum16?$AA@ 100106c0     useasm:usetab.obj
 0001:0000f6c8       ??_C@_05COGELEAH@firhh?$AA@ 100106c8     useasm:usetab.obj
 0001:0000f6d0       ??_C@_04JDNAGPBH@firh?$AA@ 100106d0     useasm:usetab.obj
 0001:0000f6d8       ??_C@_05FCKLBLAM@bilin?$AA@ 100106d8     useasm:usetab.obj
 0001:0000f6e0       ??_C@_05DINMDKHN@firvh?$AA@ 100106e0     useasm:usetab.obj
 0001:0000f6e8       ??_C@_04EHJBFAMI@firv?$AA@ 100106e8     useasm:usetab.obj
 0001:0000f6f0       ??_C@_07DLAPIEBJ@adifsum?$AA@ 100106f0     useasm:usetab.obj
 0001:0000f6f8       ??_C@_04FNGKAKMF@adif?$AA@ 100106f8     useasm:usetab.obj
 0001:0000f700       ??_C@_04CHNIFDFF@idiv?$AA@ 10010700     useasm:usetab.obj
 0001:0000f708       ??_C@_05EIKDCMOM@ima32?$AA@ 10010708     useasm:usetab.obj
 0001:0000f710       ??_C@_04DFCMAMPF@imae?$AA@ 10010710     useasm:usetab.obj
 0001:0000f718       ??_C@_05CPELDNIG@ima16?$AA@ 10010718     useasm:usetab.obj
 0001:0000f720       ??_C@_04DKDJCPOM@ima8?$AA@ 10010720     useasm:usetab.obj
 0001:0000f728       ??_C@_0L@DAOCLPMG@u16dot4off?$AA@ 10010728     useasm:usetab.obj
 0001:0000f734       ??_C@_0L@ICMCGDNG@u16dot3off?$AA@ 10010734     useasm:usetab.obj
 0001:0000f740       ??_C@_09GIAJOEKF@u8dot4off?$AA@ 10010740     useasm:usetab.obj
 0001:0000f74c       ??_C@_09NKCJDILF@u8dot3off?$AA@ 1001074c     useasm:usetab.obj
 0001:0000f758       ??_C@_07EFHPPAJH@u16dot4?$AA@ 10010758     useasm:usetab.obj
 0001:0000f760       ??_C@_07KDOGGFA@u16dot3?$AA@ 10010760     useasm:usetab.obj
 0001:0000f768       ??_C@_06NDMPFPGO@u8dot4?$AA@ 10010768     useasm:usetab.obj
 0001:0000f770       ??_C@_06JMIOMJKJ@u8dot3?$AA@ 10010770     useasm:usetab.obj
 0001:0000f778       ??_C@_04EEHAHIMI@sop3?$AA@ 10010778     useasm:usetab.obj
 0001:0000f780       ??_C@_06GEKMOMGC@sop2wm?$AA@ 10010780     useasm:usetab.obj
 0001:0000f788       ??_C@_04FNGLEJIJ@sop2?$AA@ 10010788     useasm:usetab.obj
 0001:0000f790       ??_C@_03HBHPADEG@rlp?$AA@  10010790     useasm:usetab.obj
 0001:0000f794       ??_C@_03JFEOOAEC@rol?$AA@  10010794     useasm:usetab.obj
 0001:0000f798       ??_C@_03BGJPHNPI@asr?$AA@  10010798     useasm:usetab.obj
 0001:0000f79c       ??_C@_03PMPMKOHN@shr?$AA@  1001079c     useasm:usetab.obj
 0001:0000f7a0       ??_C@_03CILNJBKC@shl?$AA@  100107a0     useasm:usetab.obj
 0001:0000f7a4       ??_C@_03COLCDPPJ@xor?$AA@  100107a4     useasm:usetab.obj
 0001:0000f7a8       ??_C@_02FODMLBIE@or?$AA@   100107a8     useasm:usetab.obj
 0001:0000f7ac       ??_C@_03BOPJPIAM@and?$AA@  100107ac     useasm:usetab.obj
 0001:0000f7b0       ??_C@_0M@CDGCCNBB@unpckc10c10?$AA@ 100107b0     useasm:usetab.obj
 0001:0000f7bc       ??_C@_09KNIBBCKD@unpcku8u8?$AA@ 100107bc     useasm:usetab.obj
 0001:0000f7c8       ??_C@_0M@MLPMEEHP@unpcks16c10?$AA@ 100107c8     useasm:usetab.obj
 0001:0000f7d4       ??_C@_0L@GDPGIBDB@unpcks16o8?$AA@ 100107d4     useasm:usetab.obj
 0001:0000f7e0       ??_C@_0L@HGMKNLCF@unpcks16s8?$AA@ 100107e0     useasm:usetab.obj
 0001:0000f7ec       ??_C@_0L@HCEHKHJH@unpcks16u8?$AA@ 100107ec     useasm:usetab.obj
 0001:0000f7f8       ??_C@_0M@MNLPLEGG@unpcks16s16?$AA@ 100107f8     useasm:usetab.obj
 0001:0000f804       ??_C@_0M@OINEOLLK@unpcks16u16?$AA@ 10010804     useasm:usetab.obj
 0001:0000f810       ??_C@_0M@KKHIBDML@unpcks16f16?$AA@ 10010810     useasm:usetab.obj
 0001:0000f81c       ??_C@_0M@KICMHBEF@unpcku16c10?$AA@ 1001081c     useasm:usetab.obj
 0001:0000f828       ??_C@_0L@LFKPGCCM@unpcku16o8?$AA@ 10010828     useasm:usetab.obj
 0001:0000f834       ??_C@_0L@KAJDDIDI@unpcku16s8?$AA@ 10010834     useasm:usetab.obj
 0001:0000f840       ??_C@_0L@KEBOEEIK@unpcku16u8?$AA@ 10010840     useasm:usetab.obj
 0001:0000f84c       ??_C@_0M@KOGPIBFM@unpcku16s16?$AA@ 1001084c     useasm:usetab.obj
 0001:0000f858       ??_C@_0M@ILAENOIA@unpcku16u16?$AA@ 10010858     useasm:usetab.obj
 0001:0000f864       ??_C@_0M@MJKICGPB@unpcku16f16?$AA@ 10010864     useasm:usetab.obj
 0001:0000f870       ??_C@_0M@POBKPHBG@unpckf16c10?$AA@ 10010870     useasm:usetab.obj
 0001:0000f87c       ??_C@_0L@DAONBCBJ@unpckf16o8?$AA@ 1001087c     useasm:usetab.obj
 0001:0000f888       ??_C@_0L@CFNBEIAN@unpckf16s8?$AA@ 10010888     useasm:usetab.obj
 0001:0000f894       ??_C@_0L@CBFMDELP@unpckf16u8?$AA@ 10010894     useasm:usetab.obj
 0001:0000f8a0       ??_C@_0M@PIFJAHAP@unpckf16s16?$AA@ 100108a0     useasm:usetab.obj
 0001:0000f8ac       ??_C@_0M@NNDCFIND@unpckf16u16?$AA@ 100108ac     useasm:usetab.obj
 0001:0000f8b8       ??_C@_0M@JPJOKAKC@unpckf16f16?$AA@ 100108b8     useasm:usetab.obj
 0001:0000f8c4       ??_C@_0M@EGFCPANN@unpckf32c10?$AA@ 100108c4     useasm:usetab.obj
 0001:0000f8d0       ??_C@_0L@MFEPNGCO@unpckf32o8?$AA@ 100108d0     useasm:usetab.obj
 0001:0000f8dc       ??_C@_0L@NAHDIMDK@unpckf32s8?$AA@ 100108dc     useasm:usetab.obj
 0001:0000f8e8       ??_C@_0L@NEPOPAII@unpckf32u8?$AA@ 100108e8     useasm:usetab.obj
 0001:0000f8f4       ??_C@_0M@EABBAAME@unpckf32s16?$AA@ 100108f4     useasm:usetab.obj
 0001:0000f900       ??_C@_0M@GFHKFPBI@unpckf32u16?$AA@ 10010900     useasm:usetab.obj
 0001:0000f90c       ??_C@_0M@CHNGKHGJ@unpckf32f16?$AA@ 1001090c     useasm:usetab.obj
 0001:0000f918       ??_C@_0M@EADOLGAD@unpckf32f32?$AA@ 10010918     useasm:usetab.obj
 0001:0000f924       ??_C@_09DDFDIML@pckc10s16?$AA@ 10010924     useasm:usetab.obj
 0001:0000f930       ??_C@_09CGFOGHBH@pckc10u16?$AA@ 10010930     useasm:usetab.obj
 0001:0000f93c       ??_C@_09GEPCJPGG@pckc10f16?$AA@ 1001093c     useasm:usetab.obj
 0001:0000f948       ??_C@_09DBKIOAM@pckc10f32?$AA@ 10010948     useasm:usetab.obj
 0001:0000f954       ??_C@_08IDEMMIKL@pcko8s16?$AA@ 10010954     useasm:usetab.obj
 0001:0000f960       ??_C@_08KGCHJHHH@pcko8u16?$AA@ 10010960     useasm:usetab.obj
 0001:0000f96c       ??_C@_08OEILGPAG@pcko8f16?$AA@ 1001096c     useasm:usetab.obj
 0001:0000f978       ??_C@_08IDGDHOGM@pcko8f32?$AA@ 10010978     useasm:usetab.obj
 0001:0000f984       ??_C@_08PHFIAKEL@pcks8s16?$AA@ 10010984     useasm:usetab.obj
 0001:0000f990       ??_C@_08NCDDFFJH@pcks8u16?$AA@ 10010990     useasm:usetab.obj
 0001:0000f99c       ??_C@_08JAJPKNOG@pcks8f16?$AA@ 1001099c     useasm:usetab.obj
 0001:0000f9a8       ??_C@_08PHHHLMIM@pcks8f32?$AA@ 100109a8     useasm:usetab.obj
 0001:0000f9b4       ??_C@_08CBABOJFG@pcku8s16?$AA@ 100109b4     useasm:usetab.obj
 0001:0000f9c0       ??_C@_08EGKLGIK@pcku8u16?$AA@ 100109c0     useasm:usetab.obj
 0001:0000f9cc       ??_C@_08EGMGEOPL@pcku8f16?$AA@ 100109cc     useasm:usetab.obj
 0001:0000f9d8       ??_C@_08CBCOFPJB@pcku8f32?$AA@ 100109d8     useasm:usetab.obj
 0001:0000f9e4       ??_C@_09OLKLFBKF@pcks16s16?$AA@ 100109e4     useasm:usetab.obj
 0001:0000f9f0       ??_C@_09MOMAAOHJ@pcks16u16?$AA@ 100109f0     useasm:usetab.obj
 0001:0000f9fc       ??_C@_09IMGMPGAI@pcks16f16?$AA@ 100109fc     useasm:usetab.obj
 0001:0000fa08       ??_C@_09OLIEOHGC@pcks16f32?$AA@ 10010a08     useasm:usetab.obj
 0001:0000fa14       ??_C@_09IIHLGEJP@pcku16s16?$AA@ 10010a14     useasm:usetab.obj
 0001:0000fa20       ??_C@_09KNBADLED@pcku16u16?$AA@ 10010a20     useasm:usetab.obj
 0001:0000fa2c       ??_C@_09OPLMMDDC@pcku16f16?$AA@ 10010a2c     useasm:usetab.obj
 0001:0000fa38       ??_C@_09IIFENCFI@pcku16f32?$AA@ 10010a38     useasm:usetab.obj
 0001:0000fa44       ??_C@_09NOENOCMM@pckf16s16?$AA@ 10010a44     useasm:usetab.obj
 0001:0000fa50       ??_C@_09PLCGLNBA@pckf16u16?$AA@ 10010a50     useasm:usetab.obj
 0001:0000fa5c       ??_C@_09LJIKEFGB@pckf16f16?$AA@ 10010a5c     useasm:usetab.obj
 0001:0000fa68       ??_C@_09NOGCFEAL@pckf16f32?$AA@ 10010a68     useasm:usetab.obj
 0001:0000fa74       ??_C@_03HMHMOHCI@efo?$AA@  10010a74     useasm:usetab.obj
 0001:0000fa78       ??_C@_07BJAGEKCG@fmaxmin?$AA@ 10010a78     useasm:usetab.obj
 0001:0000fa80       ??_C@_07IHOEOAG@fminmax?$AA@ 10010a80     useasm:usetab.obj
 0001:0000fa88       ??_C@_06ICDMGFKB@fmad16?$AA@ 10010a88     useasm:usetab.obj
 0001:0000fa90       ??_C@_04DDKBPOON@fdsy?$AA@ 10010a90     useasm:usetab.obj
 0001:0000fa98       ??_C@_04CKLKMPKM@fdsx?$AA@ 10010a98     useasm:usetab.obj
 0001:0000faa0       ??_C@_04EIBAPHDI@fmax?$AA@ 10010aa0     useasm:usetab.obj
 0001:0000faa8       ??_C@_04FKJLBDFH@fmin?$AA@ 10010aa8     useasm:usetab.obj
 0001:0000fab0       ??_C@_03KABHJCDG@fdp?$AA@  10010ab0     useasm:usetab.obj
 0001:0000fab4       ??_C@_04EBKFHEMK@fcos?$AA@ 10010ab4     useasm:usetab.obj
 0001:0000fabc       ??_C@_04OKFNDDPL@fsin?$AA@ 10010abc     useasm:usetab.obj
 0001:0000fac4       ??_C@_05OBEHOPDB@fsqrt?$AA@ 10010ac4     useasm:usetab.obj
 0001:0000facc       ??_C@_04FGIKMNCA@fexp?$AA@ 10010acc     useasm:usetab.obj
 0001:0000fad4       ??_C@_04DHGILDMJ@flog?$AA@ 10010ad4     useasm:usetab.obj
 0001:0000fadc       ??_C@_04IOAKHMKG@frsq?$AA@ 10010adc     useasm:usetab.obj
 0001:0000fae4       ??_C@_04ILDHOOJH@frcp?$AA@ 10010ae4     useasm:usetab.obj
 0001:0000faec       ??_C@_04CIEHKGIK@ffrc?$AA@ 10010aec     useasm:usetab.obj
 0001:0000faf4       ??_C@_04MMLCCJDO@fmsa?$AA@ 10010af4     useasm:usetab.obj
 0001:0000fafc       ??_C@_04DDLIGMHP@fadm?$AA@ 10010afc     useasm:usetab.obj
 0001:0000fb04       ??_C@_04KOGHKKGF@fmad?$AA@ 10010b04     useasm:usetab.obj
 0001:0000fb0c       ??_C@_0BC@EOODDAGN@filter?5coefficent?$AA@ 10010b0c     useasm:usetab.obj
 0001:0000fb20       ??_C@_0BE@FBIDIDIB@8?9bit?5source?5select?$AA@ 10010b20     useasm:usetab.obj
 0001:0000fb34       ??_C@_07FAJBBDOC@swizzle?$AA@ 10010b34     useasm:usetab.obj
 0001:0000fb3c       ??_C@_0N@KBLPGIGB@address?5mode?$AA@ 10010b3c     useasm:usetab.obj
 0001:0000fb4c       ??_C@_09DBIHEPNC@clipplane?$AA@ 10010b4c     useasm:usetab.obj
 0001:0000fb58       ??_C@_09OKBKKDGM@predicate?$AA@ 10010b58     useasm:usetab.obj
 0001:0000fb64       ??_C@_05IDCCNNGI@label?$AA@ 10010b64     useasm:usetab.obj
 0001:0000fb6c       ??_C@_03HDFKMEON@drc?$AA@  10010b6c     useasm:usetab.obj
 0001:0000fb70       ??_C@_04OHHBHOGB@link?$AA@ 10010b70     useasm:usetab.obj
 0001:0000fb78       ??_C@_09MBGEJPJA@immediate?$AA@ 10010b78     useasm:usetab.obj
 0001:0000fb84       ??_C@_08LEPPLCNF@internal?$AA@ 10010b84     useasm:usetab.obj
 0001:0000fb90       ??_C@_08KFDOCAEB@constant?$AA@ 10010b90     useasm:usetab.obj
 0001:0000fb9c       ??_C@_06FJKEMHGD@global?$AA@ 10010b9c     useasm:usetab.obj
 0001:0000fba4       ??_C@_05FKHKFDID@index?$AA@ 10010ba4     useasm:usetab.obj
 0001:0000fbac       ??_C@_0BE@EDPEAKOB@secondary?5attribute?$AA@ 10010bac     useasm:usetab.obj
 0001:0000fbc0       ??_C@_0BC@FEBGALFK@primary?5attribute?$AA@ 10010bc0     useasm:usetab.obj
 0001:0000fbd4       ??_C@_06DKIGHACF@output?$AA@ 10010bd4     useasm:usetab.obj
 0001:0000fbdc       ??_C@_09CAHPDAG@temporary?$AA@ 10010bdc     useasm:usetab.obj
 0001:0000fbe8       pszTypeToString            10010be8     useasm:usetab.obj
 0001:0000fc38       g_pfHardwareConstants      10010c38     useasm:usetab.obj
 0001:0000fd18       g_asUseInstDesc            10010d18     useasm:usetab.obj
 0001:00010dbc       ??_C@_06CMDGOKBM@SGX545?$AA@ 10011dbc     useasm:utils.obj
 0001:00010dc4       ??_C@_06HKGMENJK@SGX543?$AA@ 10011dc4     useasm:utils.obj
 0001:00010dcc       ??_C@_06EIFKCPBI@SGX541?$AA@ 10011dcc     useasm:utils.obj
 0001:00010dd4       ??_C@_06FBEBBOFJ@SGX540?$AA@ 10011dd4     useasm:utils.obj
 0001:00010ddc       ??_C@_06CJHJPMJJ@SGX535?$AA@ 10011ddc     useasm:utils.obj
 0001:00010de4       ??_C@_06ENBFDJJN@SGX531?$AA@ 10011de4     useasm:utils.obj
 0001:00010dec       ??_C@_06FEAOAINM@SGX530?$AA@ 10011dec     useasm:utils.obj
 0001:00010df4       ??_C@_06FFMMGCOL@SGX520?$AA@ 10011df4     useasm:utils.obj
 0001:000110a0       auLightSourceMemberSizes   100120a0     libffgen:ffgen.obj
 0001:000110d4       auPointParamsMemberSizes   100120d4     libffgen:ffgen.obj
 0001:000110f0       auMaterialMemberSizes      100120f0     libffgen:ffgen.obj
 0001:00011104       auLightProductMemberSizes  10012104     libffgen:ffgen.obj
 0001:00011110       auLightModelMemberSizes    10012110     libffgen:ffgen.obj
 0001:00011114       auLightModelProductMemberSizes 10012114     libffgen:ffgen.obj
 0001:00011118       ??_C@_0BI@KOKDJJDB@?1?$CK?5Runtime?5code?5log?5?$CK?1?6?$AA@ 10012118     libffgen:ffgen.obj
 0001:00011130       ??_C@_0CG@HEHGGNFE@DumpDisassembly?3?5Failed?5to?5open?5@ 10012130     libffgen:ffgen.obj
 0001:00011158       ??_C@_02CHHAKFFB@w?$CL?$AA@ 10012158     libffgen:ffgen.obj
 0001:00011180       ??_C@_0FA@LMDHKNMP@H?3?2WINCE600?2PLATFORM?2SMDKV210?2SR@ 10012180     libffgen:codegen.obj
 0001:000111d0       ??_C@_0ED@DEEDBAIC@FFTNLGenTexturing?3?5Dimension?5of?5@ 100121d0     libffgen:codegen.obj
 0001:00011214       ??_C@_0BN@BIDIPFNJ@Unrecogised?5output?5register?6?$AA@ 10012214     libffgen:codegen.obj
 0001:00011234       ??_C@_0CB@IEAJPHFE@Redirect?5output?5reg?5to?5input?5reg@ 10012234     libffgen:codegen.obj
 0001:00011258       ??_C@_0DL@ECBKIPGG@FFTNLRedirectOutputRegisterWrite@ 10012258     libffgen:codegen.obj
 0001:00011294       ??_C@_0BH@PLMPKNH@Calculate?5Eye?5position?$AA@ 10012294     libffgen:codegen.obj
 0001:000112ac       ??_C@_09EPPKEDM@MV?5Matrix?$AA@ 100122ac     libffgen:codegen.obj
 0001:000112b8       ??_C@_0BH@LMMCLBCC@Calculate?5eye?5position?$AA@ 100122b8     libffgen:codegen.obj
 0001:000112d0       ??_C@_0BC@NDNIKMLH@Normalise?5normals?$AA@ 100122d0     libffgen:codegen.obj
 0001:000112e4       ??_C@_0CB@EGGMGBKD@Normalise?5supplied?5normal?5vector@ 100122e4     libffgen:codegen.obj
 0001:00011308       ??_C@_0BI@HPNAAMDF@Pass?5through?5the?5normal?$AA@ 10012308     libffgen:codegen.obj
 0001:00011320       ??_C@_0CB@OJGIHKGB@No?5transformation?5?9?5pass?5through@ 10012320     libffgen:codegen.obj
 0001:00011344       ??_C@_0BK@NFEIADPI@Pass?5through?5the?5position?$AA@ 10012344     libffgen:codegen.obj
 0001:00011360       ??_C@_0BC@JADMGONK@Projection?5matrix?$AA@ 10012360     libffgen:codegen.obj
 0001:00011374       ??_C@_0DA@EBFKIOIO@Transform?5the?5eye?5position?5by?5pr@ 10012374     libffgen:codegen.obj
 0001:000113a4       ??_C@_0CB@CHDFKHHG@Multiply?5normal?5?5by?5blend?5weight@ 100123a4     libffgen:codegen.obj
 0001:000113c8       ??_C@_0DA@LDEDLAN@Multiply?5normal?5?5by?5blend?5weight@ 100123c8     libffgen:codegen.obj
 0001:000113f8       ??_C@_0CF@ICKPHBEG@Transform?5the?5the?5normal?5by?5the?5@ 100123f8     libffgen:codegen.obj
 0001:00011420       ??_C@_0BE@GIAEEKOE@ITMV?5matrix?5palette?$AA@ 10012420     libffgen:codegen.obj
 0001:00011434       ??_C@_0CC@PNPKLBPI@Multiply?5position?5by?5blend?5weigh@ 10012434     libffgen:codegen.obj
 0001:00011458       ??_C@_0DB@LKKMBIBN@Multiply?5position?5by?5blend?5weigh@ 10012458     libffgen:codegen.obj
 0001:0001148c       ??_C@_0CF@GKPDHNCO@Transform?5the?5the?5position?5by?5th@ 1001248c     libffgen:codegen.obj
 0001:000114b4       ??_C@_0BC@HKKMIJAG@MV?5matrix?5palette?$AA@ 100124b4     libffgen:codegen.obj
 0001:000114c8       ??_C@_09MLECJNKA@MV?5matrix?$AA@ 100124c8     libffgen:codegen.obj
 0001:000114d4       ??_C@_0CD@EKEHCEAI@?6?5?5?5?5?5?5?9?9?9?9?9?9?5Matrix?5?$CFd?5?9?9?9?9?9?9?6?5@ 100124d4     libffgen:codegen.obj
 0001:000114f8       ??_C@_0BA@ONANMFJF@Vertex?5Blending?$AA@ 100124f8     libffgen:codegen.obj
 0001:00011508       ??_C@_0P@MJEAACLN@Unpack?5indices?$AA@ 10012508     libffgen:codegen.obj
 0001:00011518       ??_C@_0BJ@IEODCOHA@Matrix?5index?5clamp?5value?$AA@ 10012518     libffgen:codegen.obj
 0001:00011534       ??_C@_0BP@CLJLEPCI@Matrix?5palette?5Vertex?5Blending?$AA@ 10012534     libffgen:codegen.obj
 0001:00011558       ??_C@_0HA@EIEEADBD@?6?5?5?5?5?5?5Reuse?5of?5MV?5matrix?5for?5no@ 10012558     libffgen:codegen.obj
 0001:000115c8       ??_C@_0CB@FBDKBHC@?6?5?5?5?5?5?5Clamp?5matrix?5indices?5?6?5?5?5@ 100125c8     libffgen:codegen.obj
 0001:000115ec       ??_C@_0DF@MAIOIMHG@Transform?5the?5the?5normal?5by?5the?5@ 100125ec     libffgen:codegen.obj
 0001:00011624       ??_C@_0M@DGLABAHO@ITMV?5matrix?$AA@ 10012624     libffgen:codegen.obj
 0001:00011630       ??_C@_0BC@ENBCCJDP@Transform?5Normals?$AA@ 10012630     libffgen:codegen.obj
 0001:00011644       ??_C@_0BI@KIFEHIED@Standard?5Transformation?$AA@ 10012644     libffgen:codegen.obj
 0001:0001165c       ??_C@_0L@DNHKCKNL@MVP?5Matrix?$AA@ 1001265c     libffgen:codegen.obj
 0001:00011668       ??_C@_0CG@GGAHKDOG@Transform?5the?5the?5position?5by?5th@ 10012668     libffgen:codegen.obj
 0001:00011690       ??_C@_0BA@KEMAKNHM@Clip?5plane?5calc?$AA@ 10012690     libffgen:codegen.obj
 0001:000116a0       ??_C@_0O@HBGOANLF@User?5Clipping?$AA@ 100126a0     libffgen:codegen.obj
 0001:000116b0       ??_C@_0M@BLMFDEGP@Clip?5planes?$AA@ 100126b0     libffgen:codegen.obj
 0001:000116bc       ??_C@_0CB@IDPANOHL@Illegal?5setup?5of?5clipping?5state?6@ 100126bc     libffgen:codegen.obj
 0001:000116e0       ??_C@_0CC@ENNMODJA@Pass?5through?5the?5secondary?5colou@ 100126e0     libffgen:codegen.obj
 0001:00011704       ??_C@_07CLODDAIM@Colours?$AA@ 10012704     libffgen:codegen.obj
 0001:0001170c       ??_C@_0BI@KELALIOO@Pass?5through?5the?5colour?$AA@ 1001270c     libffgen:codegen.obj
 0001:00011728       ??_C@_0EH@KAKLLBOP@FFTNLGenFog?3?5FOGCOORD?5or?5FOGCOOR@ 10012728     libffgen:codegen.obj
 0001:00011770       ??_C@_0BL@DFFPPPMN@Pass?5through?5the?5fog?5coord?$AA@ 10012770     libffgen:codegen.obj
 0001:0001178c       ??_C@_0DH@MPANBPOG@FOG?5EXP2?5?9?5Multiply?5eye?5distance@ 1001278c     libffgen:codegen.obj
 0001:000117c4       ??_C@_09NLKABCGF@Square?5it?$AA@ 100127c4     libffgen:codegen.obj
 0001:000117d0       ??_C@_0DG@NFOPLGGO@FOG?5EXP?5?9?5Multiply?5eye?5distance?5@ 100127d0     libffgen:codegen.obj
 0001:00011808       ??_C@_0BG@EONNLBKJ@Get?5exponential?5value?$AA@ 10012808     libffgen:codegen.obj
 0001:00011820       ??_C@_0FM@PEHMBOCC@Linear?5Fog?5?9?5Multiple?5fog?5coord?5@ 10012820     libffgen:codegen.obj
 0001:0001187c       ??_C@_0L@OPPFCILO@Fog?5Params?$AA@ 1001287c     libffgen:codegen.obj
 0001:00011888       ??_C@_03JPDFGHP@Fog?$AA@   10012888     libffgen:codegen.obj
 0001:0001188c       ??_C@_0BF@GCMNLHLK@Vertex?5to?5Eye?5Vector?$AA@ 1001288c     libffgen:codegen.obj
 0001:000118a8       ??_C@_0EG@FJENDPOA@Calculate?5eye?5to?5vertex?5vector?5u@ 100128a8     libffgen:codegen.obj
 0001:000118f0       ??_C@_0DO@KCKEGFAC@lights?5and?5the?5texture?5generatio@ 100128f0     libffgen:codegen.obj
 0001:00011930       ??_C@_0CA@OOFFNHGE@Calculate?5normalised?5eye?5vector?$AA@ 10012930     libffgen:codegen.obj
 0001:00011950       ??_C@_0BM@CHDLEFEL@Pass?5through?5the?5point?5size?$AA@ 10012950     libffgen:codegen.obj
 0001:0001196c       ??_C@_0CD@LLEGIENP@Test?5if?5size?5is?5within?5min?5and?5m@ 1001296c     libffgen:codegen.obj
 0001:00011990       ??_C@_0BN@KFLIBCPG@Clamp?5the?5result?5if?5required?$AA@ 10012990     libffgen:codegen.obj
 0001:000119b0       ??_C@_0CN@HNMACHJM@Multiply?5attenuation?5by?5requeste@ 100129b0     libffgen:codegen.obj
 0001:000119e0       ??_C@_0CH@LABFJDID@Multiply?5attenuation?5by?5the?5poin@ 100129e0     libffgen:codegen.obj
 0001:00011a08       ??_C@_0CI@OCCNBPHJ@?5tDistAtten?5?$DN?51?40?0?5?$HMPe?$HM?0?5?$HMPe?$HM?$FO2?0@ 10012a08     libffgen:codegen.obj
 0001:00011a30       ??_C@_0BG@FJNHHMID@Calculate?5attenuation?$AA@ 10012a30     libffgen:codegen.obj
 0001:00011a48       ??_C@_0L@FPLAOIEA@Point?5size?$AA@ 10012a48     libffgen:codegen.obj
 0001:00011a54       ??_C@_0N@HIBMEMNP@Point?5params?$AA@ 10012a54     libffgen:codegen.obj
 0001:00011a64       ??_C@_06KANFALAM@Points?$AA@ 10012a64     libffgen:codegen.obj
 0001:00011a6c       ??_C@_0CA@PINIOJIJ@Generate?5?$CFs?5texture?5coordinates?$AA@ 10012a6c     libffgen:codegen.obj
 0001:00011a8c       ??_C@_0BL@MAEMHHOJ@Gen?5?$CFs?5texture?5coordinates?$AA@ 10012a8c     libffgen:codegen.obj
 0001:00011aa8       ??_C@_0DK@OONLNJOH@FFTNLGenTexturing?3?5?$CFs?5texture?5en@ 10012aa8     libffgen:codegen.obj
 0001:00011ae4       ??_C@_0P@PKLHGBMJ@Texture?5Matrix?$AA@ 10012ae4     libffgen:codegen.obj
 0001:00011af4       ??_C@_0BP@BNLBENAL@Transform?5by?5texture?5matrix?5?$CFd?$AA@ 10012af4     libffgen:codegen.obj
 0001:00011b14       ??_C@_0BO@JAFHPKIC@Texture?5matrix?5transformation?$AA@ 10012b14     libffgen:codegen.obj
 0001:00011b34       ??_C@_0P@HNCOOFJG@Reflection?5Map?$AA@ 10012b34     libffgen:codegen.obj
 0001:00011b44       ??_C@_0BH@MCNFCKIF@Reflection?5Map?5tex?5gen?$AA@ 10012b44     libffgen:codegen.obj
 0001:00011b5c       ??_C@_0N@KILGKFH@Position?5Map?$AA@ 10012b5c     libffgen:codegen.obj
 0001:00011b6c       ??_C@_0BF@IKEELLF@Position?5Map?5tex?5gen?$AA@ 10012b6c     libffgen:codegen.obj
 0001:00011b84       ??_C@_0L@DJHDICEL@Normal?5Map?$AA@ 10012b84     libffgen:codegen.obj
 0001:00011b90       ??_C@_0BD@MLPNOID@Normal?5Map?5tex?5gen?$AA@ 10012b90     libffgen:codegen.obj
 0001:00011ba4       ??_C@_0CI@FDNNJHBP@generate?5sphere?5map?5texture?5coor@ 10012ba4     libffgen:codegen.obj
 0001:00011bd0       ??_C@_0EP@CLFPLMJH@compute?5m?3?5r?$FLtT2?$FN?5?$DN?$CI?$CI0?45f?5?$CK?51?1sq@ 10012bd0     libffgen:codegen.obj
 0001:00011c20       ??_C@_0BD@FNCNFONL@Sphere?5Map?5tex?5gen?$AA@ 10012c20     libffgen:codegen.obj
 0001:00011c34       ??_C@_0CE@NCCPACHK@Sphere?5?$CL?5Reflection?5map?5common?5c@ 10012c34     libffgen:codegen.obj
 0001:00011c58       ??_C@_0CI@BBLKPMCO@Get?5angle?5between?5eye?5vector?5and@ 10012c58     libffgen:codegen.obj
 0001:00011c80       ??_C@_0CD@LENOOMFO@?5compute?5r?3?5r?$FLtT3?$FN?5?$DN?5r?4x?0?5r?4y?0?5r@ 10012c80     libffgen:codegen.obj
 0001:00011ca4       ??_C@_0O@IHPGOCE@Object?5Linear?$AA@ 10012ca4     libffgen:codegen.obj
 0001:00011cb4       ??_C@_0BG@CKPHPBLK@Object?5Linear?5tex?5gen?$AA@ 10012cb4     libffgen:codegen.obj
 0001:00011ccc       ??_C@_0L@EAPMGLA@Eye?5Linear?$AA@ 10012ccc     libffgen:codegen.obj
 0001:00011cd8       ??_C@_0BD@DLKLDGHI@Eye?5Linear?5tex?5gen?$AA@ 10012cd8     libffgen:codegen.obj
 0001:00011cec       ??_C@_0N@MDCPJLLL@Pass?5through?$AA@ 10012cec     libffgen:codegen.obj
 0001:00011cfc       ??_C@_0CB@LFNMKELF@Pass?5through?5texture?5coordinates@ 10012cfc     libffgen:codegen.obj
 0001:00011d20       ??_C@_09CLMKIHFD@Texturing?$AA@ 10012d20     libffgen:codegen.obj
 0001:00011d2c       ??_C@_0CE@DFPCDDOK@Emit?5Vertex?5Data?5and?5free?5partit@ 10012d2c     libffgen:codegen.obj
 0001:00011d50       ??_C@_0BE@MINPJGCC@Emit?5Vertex?5and?5End?$AA@ 10012d50     libffgen:codegen.obj
 0001:00011d64       ??_C@_0P@IACOIGLH@End?5of?5program?$AA@ 10012d64     libffgen:codegen.obj
 0001:00011d78       ??_C@_0EM@MNFKDKIG@H?3?2WINCE600?2PLATFORM?2SMDKV210?2SR@ 10012d78     libffgen:reg.obj
 0001:00011dc4       ??_C@_0CI@PEIAICB@This?5load?5size?5currently?5not?5sup@ 10012dc4     libffgen:reg.obj
 0001:00011dec       ??_C@_0BN@OKIFANLI@Failed?5to?5alloc?5offset?5reg?5?6?$AA@ 10012dec     libffgen:reg.obj
 0001:00011e0c       ??_C@_0BN@BPFEAGPL@Failed?5to?5alloc?5address?5reg?6?$AA@ 10012e0c     libffgen:reg.obj
 0001:00011e2c       ??_C@_0BH@GMOGLMGO@Store?5the?5?$CFs?5to?5memory?$AA@ 10012e2c     libffgen:reg.obj
 0001:00011e44       ??_C@_0CO@IDEIBDON@LoadConstant?$CI?$CJ?3?5Can?8t?5handle?5neg@ 10012e44     libffgen:reg.obj
 0001:00011e74       ??_C@_0CB@EHLOELJD@LoadConstant?$CI?$CJ?3?5No?5data?5to?5load?6@ 10012e74     libffgen:reg.obj
 0001:00011e98       ??_C@_0BL@DDDFGMDF@Failed?5to?5alloc?5const?5reg?6?$AA@ 10012e98     libffgen:reg.obj
 0001:00011eb4       ??_C@_0BO@OADPCFIM@input?5index?5?$CK?5stride?5?$CL?5offset?$AA@ 10012eb4     libffgen:reg.obj
 0001:00011ed4       ??_C@_0BL@DMGPOLHL@mov?5input?5offset?5into?5temp?$AA@ 10012ed4     libffgen:reg.obj
 0001:00011ef0       ??_C@_0BL@PAKBHIML@Failed?5to?5malloc?5register?6?$AA@ 10012ef0     libffgen:reg.obj
 0001:00011f10       ??_C@_0GJ@LCFPJFAA@GetReg?3?5Reg?5space?5must?5be?5reserv@ 10012f10     libffgen:reg.obj
 0001:00011f7c       ??_C@_0DL@HGGCFMD@GetReg?3?5Load?5offsets?5not?5valid?5f@ 10012f7c     libffgen:reg.obj
 0001:00011fb8       ??_C@_0FJ@JMBFGGAD@GetReg?3?5Can?5only?5reget?5constants@ 10012fb8     libffgen:reg.obj
 0001:00012018       ??_C@_0FJ@IPHPFJFP@GetReg?3?5Load?5offset?5?$CL?5size?5?$CI?$CFd?5?$CL@ 10013018     libffgen:reg.obj
 0001:00012078       ??_C@_0FN@GHKIOENE@GetReg?3?5If?5sizes?5match?5for?5exist@ 10013078     libffgen:reg.obj
 0001:000120d8       ??_C@_0DH@GOPDPMPC@GetReg?3?5Can?8t?5alloc?5space?5for?5th@ 100130d8     libffgen:reg.obj
 0001:00012110       ??_C@_0FD@KDOOHEOL@GetReg?3?5Can?8t?5reget?5register?5wit@ 10013110     libffgen:reg.obj
 0001:00012168       ??_C@_0FK@FAEDPFKH@GetReg?3?5Only?5valid?5input?5registe@ 10013168     libffgen:reg.obj
 0001:000121c4       ??_C@_0CD@OGFFNGFJ@GetReg?3?5Invalid?5reg?5type?5?$CI?$CFs?0?5?$CFd@ 100131c4     libffgen:reg.obj
 0001:000121e8       ??_C@_0BN@DAICFPHG@GetReg?3?5Size?5was?50?5?$CI?$CFs?0?5?$CFd?$CJ?6?$AA@ 100131e8     libffgen:reg.obj
 0001:00012208       ??_C@_0DI@MODDCAAB@GetReg?3?5Load?5offsets?5only?5valid?5@ 10013208     libffgen:reg.obj
 0001:00012240       ??_C@_0DP@GFPDICLF@StoreInstructionfn?3?5Failed?5to?5al@ 10013240     libffgen:inst.obj
 0001:00012280       ??_C@_0CI@JFGMKCCF@StoreInstruction?3?5Reg?5?$CFd?5was?5nul@ 10013280     libffgen:inst.obj
 0001:000122a8       ??_C@_0DN@CJDNBDCF@StoreInstruction?3?5Failed?5to?5allo@ 100132a8     libffgen:inst.obj
 0001:000122e8       ??_C@_0CM@CACCDEMK@GetLabel?3?5Error?0?5couldn?8t?5alloc?5@ 100132e8     libffgen:inst.obj
 0001:00012314       ??_C@_0M@GDJNOEBD@?$CFs_LABEL?$CFlu?$AA@ 10013314     libffgen:inst.obj
 0001:00012320       ??_C@_0CM@PALIDHOL@GetLabel?3?5Error?0?5couldn?8t?5alloc?5@ 10013320     libffgen:inst.obj
 0001:0001234c       ??_C@_0BI@CELJOCLM@Enable?5dest?5base?5offset?$AA@ 1001334c     libffgen:inst.obj
 0001:00012364       ??_C@_0BJ@PBBOCFKH@Disable?5dest?5base?5offset?$AA@ 10013364     libffgen:inst.obj
 0001:00012380       ??_C@_0EN@MEKLMKL@H?3?2WINCE600?2PLATFORM?2SMDKV210?2SR@ 10013380     libffgen:inst.obj
 0001:000123d0       ??_C@_0CJ@EIHLMMOJ@EncodeInstruction?3?5Reg?5?$CFd?5was?5nu@ 100133d0     libffgen:inst.obj
 0001:000123fc       ??_C@_0DH@FBCAJPKC@Following?5code?5need?5to?5be?5aligne@ 100133fc     libffgen:inst.obj
 0001:00012434       ??_C@_0BH@JCIFADOE@Enable?5dest?5increments?$AA@ 10013434     libffgen:inst.obj
 0001:0001244c       ??_C@_0BI@FFADPMMG@Disable?5dest?5increments?$AA@ 1001344c     libffgen:inst.obj
 0001:00012464       ??_C@_0CC@IONBMNAK@Move?5source?5vector?5into?5temporar@ 10013464     libffgen:inst.obj
 0001:00012488       ??_C@_0CM@NKIDJECP@IF_PRED?3?5Error?0?5maximum?5nested?5d@ 10013488     libffgen:inst.obj
 0001:000124b4       ??_C@_0CK@GJDOIHFF@END_PRED?3?5Error?0?5condition?5stack@ 100134b4     libffgen:inst.obj
 0001:000124e0       ??_C@_0FB@MGHDDCHB@H?3?2WINCE600?2PLATFORM?2SMDKV210?2SR@ 100134e0     libffgen:lighting.obj
 0001:00012534       ??_C@_0BI@JAJKGEDI@Calculate?5local?5ambient?$AA@ 10013534     libffgen:lighting.obj
 0001:0001254c       ??_C@_0CH@FGCBILAO@Calculate?5ambient?5components?5of?5@ 1001354c     libffgen:lighting.obj
 0001:00012574       ??_C@_0BI@CCMKNPCE@Calculate?5local?5diffuse?$AA@ 10013574     libffgen:lighting.obj
 0001:0001258c       ??_C@_0CH@PGHAKFN@Calculate?5diffuse?5components?5of?5@ 1001358c     libffgen:lighting.obj
 0001:000125b4       ??_C@_0BJ@OECLFEPJ@Calculate?5local?5specular?$AA@ 100135b4     libffgen:lighting.obj
 0001:000125d0       ??_C@_0CI@DCMHGBOG@Calculate?5specular?5components?5of@ 100135d0     libffgen:lighting.obj
 0001:000125f8       ??_C@_0N@CEILCPKB@End?5of?5light?$AA@ 100135f8     libffgen:lighting.obj
 0001:00012608       ??_C@_0DG@FCGOHAJD@Load?5reg?5with?51?40?5to?5get?5round?5r@ 10013608     libffgen:lighting.obj
 0001:00012640       ??_C@_0BK@OHEOCDDF@Calc?5specular?5half?5angle?5?$AA@ 10013640     libffgen:lighting.obj
 0001:00012660       ??_C@_0EN@OCFLHMLI@Set?5predicate?5for?5specular?5test?5@ 10013660     libffgen:lighting.obj
 0001:000126b0       ??_C@_0CD@HLLCFIJC@Do?5we?5need?5to?5calc?5specular?5coef@ 100136b0     libffgen:lighting.obj
 0001:000126d4       ??_C@_0P@CCJHPFLG@SpecLightCoeff?$AA@ 100136d4     libffgen:lighting.obj
 0001:000126e4       ??_C@_0BJ@HDJNOKLO@Calculate?5specular?5coeff?$AA@ 100136e4     libffgen:lighting.obj
 0001:00012700       ??_C@_0BB@JHGCHADD@NoSpecLightCoeff?$AA@ 10013700     libffgen:lighting.obj
 0001:00012714       ??_C@_0BI@CFPAIJCH@Set?5specular?5coeff?5to?50?$AA@ 10013714     libffgen:lighting.obj
 0001:0001272c       ??_C@_0BO@MIKNJBAA@Normalise?5specular?5half?5angle?$AA@ 1001372c     libffgen:lighting.obj
 0001:0001274c       ??_C@_0BG@GJMHPMIM@Load?5light?5half?5angle?$AA@ 1001374c     libffgen:lighting.obj
 0001:00012764       ??_C@_0CN@FAAJJLEL@Local?5viewer?5enabled?5?3?5h_i?5?$DN?5?$CIVP@ 10013764     libffgen:lighting.obj
 0001:00012794       ??_C@_0BI@BJHLPANM@Clamp?5diff?5angle?5to?50?40?$AA@ 10013794     libffgen:lighting.obj
 0001:000127b0       ??_C@_0GF@FHLDJOLL@Test?5result?5?9?5?$CB?$CB?5shift?5this?5test@ 100137b0     libffgen:lighting.obj
 0001:00012818       ??_C@_0EE@KEIMPFOB@Check?5if?5it?8s?5worth?5calculating?5@ 10013818     libffgen:lighting.obj
 0001:0001285c       ??_C@_0M@PMCFJDGB@AmbientOnly?$AA@ 1001385c     libffgen:lighting.obj
 0001:00012868       ??_C@_0BF@HKIFJBJI@Move?5onto?5next?5light?$AA@ 10013868     libffgen:lighting.obj
 0001:00012880       ??_C@_0L@KCMDIALA@EndOfLight?$AA@ 10013880     libffgen:lighting.obj
 0001:00012890       ??_C@_0EF@EMBOGPNI@Calculate?5angle?5between?5normal?5a@ 10013890     libffgen:lighting.obj
 0001:000128d8       ??_C@_0BN@KMMADCKC@Attenuate?5light?5coefficients?$AA@ 100138d8     libffgen:lighting.obj
 0001:000128f8       ??_C@_0DA@JGABDEMF@Local?5viewer?5disabled?5?3h_i?5?$DN?5?$CIVP@ 100138f8     libffgen:lighting.obj
 0001:00012928       ??_C@_0EO@ICIMPIAM@Get?5vertex?5to?5light?5vector?5?$CIfsub@ 10013928     libffgen:lighting.obj
 0001:00012978       ??_C@_0CB@FDFDOGMJ@Normalise?5vertex?5to?5light?5vector@ 10013978     libffgen:lighting.obj
 0001:0001299c       ??_C@_0DE@KMFGIAFA@Setup?5distance?5vector?5?5?$DN?5?$HL1?0?5?$HMVP@ 1001399c     libffgen:lighting.obj
 0001:000129d0       ??_C@_0BP@KEMKENJA@Calculate?5distance?5attenuation?$AA@ 100139d0     libffgen:lighting.obj
 0001:000129f0       ??_C@_07JBEAGHEM@?$CIatt_i?$CJ?$AA@ 100139f0     libffgen:lighting.obj
 0001:000129f8       ??_C@_0DK@CGKPLDHE@Calculate?5angle?5between?5normal?5a@ 100139f8     libffgen:lighting.obj
 0001:00012a38       ??_C@_0FA@JFACKHEB@Calculate?5angle?5between?5light?5to@ 10013a38     libffgen:lighting.obj
 0001:00012a88       ??_C@_0EL@HKGFEGHF@If?5vertex?5falls?5outside?5of?5?$CIcosi@ 10013a88     libffgen:lighting.obj
 0001:00012ad4       ??_C@_0CP@MHGPMFFM@Calculate?5attenuation?5due?5to?5spo@ 10013ad4     libffgen:lighting.obj
 0001:00012b04       ??_C@_0CL@PCMLNOCJ@Add?5spotlight?5calc?5to?5distance?5a@ 10013b04     libffgen:lighting.obj
 0001:00012b30       ??_C@_0BD@KNHKDHAM@Restore?5the?5normal?$AA@ 10013b30     libffgen:lighting.obj
 0001:00012b44       ??_C@_0BB@GLNHJEJ@?$CFs?5Light?5?$CFd?5?$CI?$CFs?$CJ?$AA@ 10013b44     libffgen:lighting.obj
 0001:00012b58       ??_C@_0P@HCGDDOH@Temp?5size?5?$DN?5?$CFd?$AA@ 10013b58     libffgen:lighting.obj
 0001:00012b68       ??_C@_05JODGIKH@Light?$AA@ 10013b68     libffgen:lighting.obj
 0001:00012b70       ??_C@_0O@OBACKCAK@Light?5Product?$AA@ 10013b70     libffgen:lighting.obj
 0001:00012b80       ??_C@_0BB@JFNLKFCP@without?5Specular?$AA@ 10013b80     libffgen:lighting.obj
 0001:00012b94       ??_C@_0O@ODJOONP@with?5Specular?$AA@ 10013b94     libffgen:lighting.obj
 0001:00012ba4       ??_C@_0L@EGIHIBEN@Local?5Spot?$AA@ 10013ba4     libffgen:lighting.obj
 0001:00012bb0       ??_C@_0O@MMKOGHI@Infinite?5Spot?$AA@ 10013bb0     libffgen:lighting.obj
 0001:00012bc0       ??_C@_0M@BDIGANNJ@Local?5Point?$AA@ 10013bc0     libffgen:lighting.obj
 0001:00012bcc       ??_C@_0P@EFHPIEJN@Infinite?5Point?$AA@ 10013bcc     libffgen:lighting.obj
 0001:00012bdc       ??_C@_0DJ@FCDMIGGI@Invert?5the?5normal?5for?5calculatin@ 10013bdc     libffgen:lighting.obj
 0001:00012c18       ??_C@_0BL@KNCGAANN@Use?5diffuse?5material?5alpha?$AA@ 10013c18     libffgen:lighting.obj
 0001:00012c34       ??_C@_0BI@EHJKGKMF@Use?5vertex?5colour?5alpha?$AA@ 10013c34     libffgen:lighting.obj
 0001:00012c4c       ??_C@_0CH@EONMBKHI@Scene?5colour?5?9?5Use?5light?5model?5p@ 10013c4c     libffgen:lighting.obj
 0001:00012c74       ??_C@_0BE@MJHGKBLI@Light?5Model?5Product?$AA@ 10013c74     libffgen:lighting.obj
 0001:00012c88       ??_C@_0DG@FCGODNCJ@Scene?5colour?5?9?5Use?5vertex?5colour@ 10013c88     libffgen:lighting.obj
 0001:00012cc0       ??_C@_0DH@NGDPMDEN@Scene?5colour?5?9?5Use?5vertex?5colour@ 10013cc0     libffgen:lighting.obj
 0001:00012cf8       ??_C@_0M@DCEJEFAF@Light?5Model?$AA@ 10013cf8     libffgen:lighting.obj
 0001:00012d04       ??_C@_08CPBFELGP@Material?$AA@ 10013d04     libffgen:lighting.obj
 0001:00012d10       ??_C@_0CJ@FCJPOOPD@Zero?5seperate?5specular?5reg?5?$CInon?5@ 10013d10     libffgen:lighting.obj
 0001:00012d3c       ??_C@_0BE@PHMJKILD@Lighting?5front?5face?$AA@ 10013d3c     libffgen:lighting.obj
 0001:00012d50       ??_C@_0BD@IHLDDDDM@Lighting?5back?5face?$AA@ 10013d50     libffgen:lighting.obj
 0001:00012d8c       InitAccumUSECodeBlocks     10013d8c f   accum.obj
 0001:00012f4c       FreeAccumUSECodeBlocks     10013f4c f   accum.obj
 0001:0001353c       SetupBGObject              1001453c f   accum.obj
 0001:000137b4       SendAccumulateObject       100147b4 f   accum.obj
 0001:00013940       CreateBufObjState          10014940 f   bufobj.obj
 0001:00013964       FreeBufObjState            10014964 f   bufobj.obj
 0001:00013ac8       SetupBufObjNameArray       10014ac8 f   bufobj.obj
 0001:00013ad8       glBindBuffer               10014ad8 f   bufobj.obj
 0001:00013c4c       glDeleteBuffers            10014c4c f   bufobj.obj
 0001:00013d1c       glGenBuffers               10014d1c f   bufobj.obj
 0001:00013d68       glBufferData               10014d68 f   bufobj.obj
 0001:00013f04       glBufferSubData            10014f04 f   bufobj.obj
 0001:00013ffc       glMapBufferOES             10014ffc f   bufobj.obj
 0001:000140c8       glUnmapBufferOES           100150c8 f   bufobj.obj
 0001:00014150       InitClearUSECodeBlocks     10015150 f   clear.obj
 0001:00014294       FreeClearUSECodeBlocks     10015294 f   clear.obj
 0001:000149c8       SendClearPrims             100159c8 f   clear.obj
 0001:00014bd8       glClear                    10015bd8 f   clear.obj
 0001:00014d00       glClearColor               10015d00 f   clear.obj
 0001:00014d94       glClearColorx              10015d94 f   clear.obj
 0001:00014ec0       glClearDepthf              10015ec0 f   clear.obj
 0001:00014eec       glClearDepthx              10015eec f   clear.obj
 0001:00014f44       glClearStencil             10015f44 f   clear.obj
 0001:000156fc       glDrawTexsOES              100166fc f   drawtex.obj
 0001:000157bc       glDrawTexiOES              100167bc f   drawtex.obj
 0001:0001587c       glDrawTexfOES              1001687c f   drawtex.obj
 0001:000158c0       glDrawTexxOES              100168c0 f   drawtex.obj
 0001:000159e8       glDrawTexsvOES             100169e8 f   drawtex.obj
 0001:00015a9c       glDrawTexivOES             10016a9c f   drawtex.obj
 0001:00015b50       glDrawTexfvOES             10016b50 f   drawtex.obj
 0001:00015b8c       glDrawTexxvOES             10016b8c f   drawtex.obj
 0001:00017268       AttachAllUsedResourcesToCurrentSurface 10018268 f   drawvarray.obj
 0001:000175cc       glDrawArrays               100185cc f   drawvarray.obj
 0001:000177a4       glDrawElements             100187a4 f   drawvarray.obj
 0001:000187ac       glMultiDrawArrays          100197ac f   drawvarray.obj
 0001:00018b40       glMultiDrawElements        10019b40 f   drawvarray.obj
 0001:0001a688       ReleaseImageFromTexture    1001b688 f   eglimage.obj
 0001:0001a814       glEGLImageTargetTexture2DOES 1001b814 f   eglimage.obj
 0001:0001a930       glEGLImageTargetRenderbufferStorageOES 1001b930 f   eglimage.obj
 0001:0001a9d8       ReleaseImageFromRenderbuffer 1001b9d8 f   eglimage.obj
 0001:0001a9f8       GLESGetImageSource         1001b9f8 f   eglimage.obj
 0001:0001ad70       IsColorAttachmentTwiddled  1001bd70 f   fbo.obj
 0001:0001ade0       FlushAttachableIfNeeded    1001bde0 f   fbo.obj
 0001:0001aec0       DestroyFBOAttachableRenderSurface 1001bec0 f   fbo.obj
 0001:0001afac       SetupRenderBufferNameArray 1001bfac f   fbo.obj
 0001:0001afbc       SetupFrameBufferObjectNameArray 1001bfbc f   fbo.obj
 0001:0001afcc       CreateFrameBufferState     1001bfcc f   fbo.obj
 0001:0001b034       RemoveFrameBufferAttachment 1001c034 f   fbo.obj
 0001:0001b150       ChangeDrawableParams       1001c150 f   fbo.obj
 0001:0001b7e8       GetFrameBufferCompleteness 1001c7e8 f   fbo.obj
 0001:0001b8b4       FBOAttachableHasBeenModified 1001c8b4 f   fbo.obj
 0001:0001b8e8       glIsRenderbufferOES        1001c8e8 f   fbo.obj
 0001:0001b944       glBindRenderbufferOES      1001c944 f   fbo.obj
 0001:0001ba84       glDeleteRenderbuffersOES   1001ca84 f   fbo.obj
 0001:0001bb3c       glGenRenderbuffersOES      1001cb3c f   fbo.obj
 0001:0001bb8c       glRenderbufferStorageOES   1001cb8c f   fbo.obj
 0001:0001be60       SetupRenderbufferFromEGLImage 1001ce60 f   fbo.obj
 0001:0001bf68       glGetRenderbufferParameterivOES 1001cf68 f   fbo.obj
 0001:0001c0c0       glIsFramebufferOES         1001d0c0 f   fbo.obj
 0001:0001c11c       glBindFramebufferOES       1001d11c f   fbo.obj
 0001:0001c2e4       glDeleteFramebuffersOES    1001d2e4 f   fbo.obj
 0001:0001c3a8       glGenFramebuffersOES       1001d3a8 f   fbo.obj
 0001:0001c3f4       glCheckFramebufferStatusOES 1001d3f4 f   fbo.obj
 0001:0001c44c       glFramebufferTexture2DOES  1001d44c f   fbo.obj
 0001:0001c614       glFramebufferRenderbufferOES 1001d614 f   fbo.obj
 0001:0001c764       glGetFramebufferAttachmentParameterivOES 1001d764 f   fbo.obj
 0001:0001c8dc       glGenerateMipmapOES        1001d8dc f   fbo.obj
 0001:0001ca30       FreeFrameBufferState       1001da30 f   fbo.obj
 0001:0001cd14       glFogfv                    1001dd14 f   fog.obj
 0001:0001cd38       glFogf                     1001dd38 f   fog.obj
 0001:0001cd90       glFogxv                    1001dd90 f   fog.obj
 0001:0001cee0       glFogx                     1001dee0 f   fog.obj
 0001:0001d390       DestroyHashedBlendState    1001e390 f   fftex.obj
 0001:0001d5dc       AddFFTextureBinding        1001e5dc f   fftex.obj
 0001:0001d670       ValidateFFTextureConstants 1001e670 f   fftex.obj
 0001:0001d738       ValidateFFTextureBlending  1001e738 f   fftex.obj
 0001:00021294       CreateIntegerFragmentProgramFromFF 10022294 f   fftexhw.obj
 0001:00021654       FFGENMalloc                10022654 f   fftnlgles.obj
 0001:0002165c       FFGENCalloc                1002265c f   fftnlgles.obj
 0001:00021664       FFGENRealloc               10022664 f   fftnlgles.obj
 0001:00021670       FFGENFree                  10022670 f   fftnlgles.obj
 0001:00021680       FFGENPrintf                10022680 f   fftnlgles.obj
 0001:000216c4       DestroyFFTNLCode           100226c4 f   fftnlgles.obj
 0001:00021718       InitFFTNLState             10022718 f   fftnlgles.obj
 0001:000217f8       FreeFFTNLState             100227f8 f   fftnlgles.obj
 0001:00021f2c       SetupFFTNLShaderOutputs    10022f2c f   fftnlgles.obj
 0001:0002217c       SetupBuildFFTNLShaderConstants 1002317c f   fftnlgles.obj
 0001:00022df0       SetupFFTNLShader           10023df0 f   fftnlgles.obj
 0001:00024348       glIsTexture                10025348 f   get.obj
 0001:000243a4       glIsBuffer                 100253a4 f   get.obj
 0001:00024400       glGetBufferParameteriv     10025400 f   get.obj
 0001:000244ec       glGetBufferPointervOES     100254ec f   get.obj
 0001:00024594       glGetMaterialfv            10025594 f   get.obj
 0001:000245c0       glGetMaterialxv            100255c0 f   get.obj
 0001:00024684       glGetLightfv               10025684 f   get.obj
 0001:000246b0       glGetLightxv               100256b0 f   get.obj
 0001:00024830       glGetTexEnvfv              10025830 f   get.obj
 0001:0002485c       glGetTexEnvxv              1002585c f   get.obj
 0001:00024948       glGetTexEnviv              10025948 f   get.obj
 0001:000249e0       glGetClipPlanef            100259e0 f   get.obj
 0001:00024a34       glGetClipPlanex            10025a34 f   get.obj
 0001:00024b24       glGetTexParameteriv        10025b24 f   get.obj
 0001:00024b50       glGetTexParameterfv        10025b50 f   get.obj
 0001:00024c40       glGetTexParameterxv        10025c40 f   get.obj
 0001:00024cd8       glGetTexGenivOES           10025cd8 f   get.obj
 0001:00024d28       glGetTexGenfvOES           10025d28 f   get.obj
 0001:00024d8c       glGetTexGenxvOES           10025d8c f   get.obj
 0001:00024dd4       glGetPointerv              10025dd4 f   get.obj
 0001:00024ec4       glIsEnabled                10025ec4 f   get.obj
 0001:00024ee8       glGetError                 10025ee8 f   get.obj
 0001:00024f08       glGetString                10025f08 f   get.obj
 0001:00026610       glGetFixedv                10027610 f   get.obj
 0001:00026638       glGetFloatv                10027638 f   get.obj
 0001:00026660       glGetBooleanv              10027660 f   get.obj
 0001:00026688       glGetIntegerv              10027688 f   get.obj
 0001:0002712c       HardwareMakeTextureMipmapLevels 1002812c f   makemips.obj
 0001:00027638       MakeTextureMipmapLevels    10028638 f   makemips.obj
 0001:00028388       PickMatrixProcs            10029388 f   matrix.obj
 0001:000283b0       PickInvTransposeProcs      100293b0 f   matrix.obj
 0001:000283c8       TransposeMatrix            100293c8 f   matrix.obj
 0001:0002844c       ComputeInverseTranspose    1002944c f   matrix.obj
 0001:00028568       InvertTransposeMatrix      10029568 f   matrix.obj
 0001:00029be4       CopyMatrix                 1002abe4 f   matrix.obj
 0001:00029c70       MakeIdentity               1002ac70 f   matrix.obj
 0001:00029cc0       MultMatrix                 1002acc0 f   matrix.obj
 0001:0002a050       DoMultMatrix               1002b050 f   matrix.obj
 0001:0002a1f0       DoLoadMatrix               1002b1f0 f   matrix.obj
 0001:0002a30c       MultiplyMatrix             1002b30c f   matrix.obj
 0001:0002a3f8       ScaleMatrix                1002b3f8 f   matrix.obj
 0001:0002a598       TranslateMatrix            1002b598 f   matrix.obj
 0001:0002a830       PushModelViewMatrix        1002b830 f   matrix.obj
 0001:0002a890       PopModelViewMatrix         1002b890 f   matrix.obj
 0001:0002a8cc       LoadIdentityModelViewMatrix 1002b8cc f   matrix.obj
 0001:0002a938       PushMatrixPaletteMatrix    1002b938 f   matrix.obj
 0001:0002a93c       PopMatrixPaletteMatrix     1002b93c f   matrix.obj
 0001:0002a940       LoadIdentityMatrixPaletteMatrix 1002b940 f   matrix.obj
 0001:0002a9b8       PushProjectionMatrix       1002b9b8 f   matrix.obj
 0001:0002aa14       PopProjectionMatrix        1002ba14 f   matrix.obj
 0001:0002aa50       LoadIdentityProjectionMatrix 1002ba50 f   matrix.obj
 0001:0002aaac       PushTextureMatrix          1002baac f   matrix.obj
 0001:0002ab2c       PopTextureMatrix           1002bb2c f   matrix.obj
 0001:0002ab90       LoadIdentityTextureMatrix  1002bb90 f   matrix.obj
 0001:0002abf0       PushProgramMatrix          1002bbf0 f   matrix.obj
 0001:0002ac50       PopProgramMatrix           1002bc50 f   matrix.obj
 0001:0002ac98       LoadIdentityProgramMatrix  1002bc98 f   matrix.obj
 0001:0002acd8       FreeTransformState         1002bcd8 f   matrix.obj
 0001:0002ad84       glCurrentPaletteMatrixOES  1002bd84 f   matrix.obj
 0001:0002ade0       glLoadPaletteFromModelViewMatrixOES 1002bde0 f   matrix.obj
 0001:0002ae1c       InitTransformState         1002be1c f   matrix.obj
 0001:0002b0a4       Clampf                     1002c0a4 f   misc.obj
 0001:0002b108       Clampi                     1002c108 f   misc.obj
 0001:0002b12c       FloatToHWByte              1002c12c f   misc.obj
 0001:0002b2d0       ColorConvertToHWFormat     1002c2d0 f   misc.obj
 0001:0002b314       ColorConvertFromHWFormat   1002c314 f   misc.obj
 0001:0002b3f0       Normalize                  1002c3f0 f   misc.obj
 0001:0002b58c       FloorLog2                  1002c58c f   misc.obj
 0001:0002b5ac       glFinish                   1002c5ac f   misc.obj
 0001:0002b6c4       glFlush                    1002c6c4 f   misc.obj
 0001:0002b704       glQueryMatrixxOES          1002c704 f   misc.obj
 0001:0002b854       SetError                   1002c854 f   misc.obj
 0001:0002b864       GetApplicationHints        1002c864 f   misc.obj
 0001:0002bbc4       BuildExtensionString       1002cbc4 f   misc.obj
 0001:0002bbdc       DestroyExtensionString     1002cbdc f   misc.obj
 0001:0002bc00       glHint                     1002cc00 f   misc.obj
 0001:0002bc94       SetErrorFRM                1002cc94 f   misc.obj
 0001:0002bcb0       CreateNamesArray           1002ccb0 f   names.obj
 0001:0002bd4c       NamesArrayGenNames         1002cd4c f   names.obj
 0001:0002be1c       NamesArrayMapFunction      1002ce1c f   names.obj
 0001:0002be90       DestroyNamesArray          1002ce90 f   names.obj
 0001:0002beec       InsertNamedItem            1002ceec f   names.obj
 0001:0002bfc0       NamedItemAddRef            1002cfc0 f   names.obj
 0001:0002c050       NamedItemDelRef            1002d050 f   names.obj
 0001:0002c128       NamedItemDelRefByName      1002d128 f   names.obj
 0001:0002c284       glPixelStorei              1002d284 f   pixop.obj
 0001:0002c590       SetupReadPixelsSpanInfo    1002d590 f   pixop.obj
 0001:0002c968       glReadPixels               1002d968 f   pixop.obj
 0001:0002cc30       DestroyHashedPDSVariant    1002dc30 f   shader.obj
 0001:0002cd6c       ReclaimUSEShaderVariantMemFRM 1002dd6c f   shader.obj
 0001:0002cd70       DestroyUSECodeVariantGhostFRM 1002dd70 f   shader.obj
 0001:0002cd74       DestroyVertexVariants      1002dd74 f   shader.obj
 0001:0002cdd8       FreeShader                 1002ddd8 f   shader.obj
 0001:0002ce1c       FreeProgramState           1002de1c f   shader.obj
 0001:0002ce84       InitScissorUSECodeBlocks   1002de84 f   scissor.obj
 0001:0002cefc       FreeScissorUSECodeBlocks   1002defc f   scissor.obj
 0001:0002d7e4       SendDrawMaskForPrimitive   1002e7e4 f   scissor.obj
 0001:0002d9bc       SendDrawMaskForClear       1002e9bc f   scissor.obj
 0001:0002da84       glScissor                  1002ea84 f   scissor.obj
 0001:0002db5c       WaitForTA                  1002eb5c f   sgxif.obj
 0001:0002dff8       PrepareToDraw              1002eff8 f   sgxif.obj
 0001:0002e858       ScheduleTA                 1002f858 f   sgxif.obj
 0001:0002e974       KickLimit_ScheduleTA       1002f974 f   sgxif.obj
 0001:0002e998       SpanPack16                 1002f998 f   spanpack.obj
 0001:0002e9e8       SpanPack32                 1002f9e8 f   spanpack.obj
 0001:0002ea38       SpanPackARGB4444toRGBA4444 1002fa38 f   spanpack.obj
 0001:0002ea74       SpanPackARGB1555toRGBA5551 1002fa74 f   spanpack.obj
 0001:0002eab0       SpanPackARGB8888toABGR8888 1002fab0 f   spanpack.obj
 0001:0002eaf8       SpanPackARGB8888toXBGR8888 1002faf8 f   spanpack.obj
 0001:0002eb40       SpanPackARGB8888toRGB565   1002fb40 f   spanpack.obj
 0001:0002eb90       SpanPackARGB8888toARGB4444 1002fb90 f   spanpack.obj
 0001:0002ebe8       SpanPackARGB8888toARGB1555 1002fbe8 f   spanpack.obj
 0001:0002ec3c       SpanPackARGB8888toLuminanceAlpha 1002fc3c f   spanpack.obj
 0001:0002ec74       SpanPackARGB8888toLuminance 1002fc74 f   spanpack.obj
 0001:0002ecac       SpanPackAXXX8888toAlpha    1002fcac f   spanpack.obj
 0001:0002ece4       SpanPackABGR8888toARGB8888 1002fce4 f   spanpack.obj
 0001:0002ed2c       SpanPackABGR8888toXBGR8888 1002fd2c f   spanpack.obj
 0001:0002ed74       SpanPackABGR8888toRGB565   1002fd74 f   spanpack.obj
 0001:0002edc4       SpanPackABGR8888toARGB4444 1002fdc4 f   spanpack.obj
 0001:0002ee1c       SpanPackABGR8888toARGB1555 1002fe1c f   spanpack.obj
 0001:0002ee74       SpanPackABGR8888toLuminanceAlpha 1002fe74 f   spanpack.obj
 0001:0002eeb4       SpanPackABGR8888toLuminance 1002feb4 f   spanpack.obj
 0001:0002eee8       SpanPackARGB4444toABGR8888 1002fee8 f   spanpack.obj
 0001:0002ef58       SpanPackARGB4444toXBGR8888 1002ff58 f   spanpack.obj
 0001:0002efc0       SpanPackARGB4444toARGB8888 1002ffc0 f   spanpack.obj
 0001:0002f030       SpanPackARGB4444toRGB565   10030030 f   spanpack.obj
 0001:0002f0b4       SpanPackARGB4444toARGB1555 100300b4 f   spanpack.obj
 0001:0002f13c       SpanPackARGB4444toLuminanceAlpha 1003013c f   spanpack.obj
 0001:0002f190       SpanPackARGB4444toLuminance 10030190 f   spanpack.obj
 0001:0002f1cc       SpanPackARGB4444toAlpha    100301cc f   spanpack.obj
 0001:0002f208       SpanPackARGB1555toABGR8888 10030208 f   spanpack.obj
 0001:0002f284       SpanPackARGB1555toXBGR8888 10030284 f   spanpack.obj
 0001:0002f2f8       SpanPackARGB1555toARGB8888 100302f8 f   spanpack.obj
 0001:0002f36c       SpanPackARGB1555toRGB565   1003036c f   spanpack.obj
 0001:0002f3d0       SpanPackARGB1555toARGB4444 100303d0 f   spanpack.obj
 0001:0002f428       SpanPackARGB1555toLuminanceAlpha 10030428 f   spanpack.obj
 0001:0002f484       SpanPackARGB1555toLuminance 10030484 f   spanpack.obj
 0001:0002f4c8       SpanPackARGB1555toAlpha    100304c8 f   spanpack.obj
 0001:0002f510       SpanPackRGB565toXBGR8888   10030510 f   spanpack.obj
 0001:0002f580       SpanPackRGB565toLuminance  10030580 f   spanpack.obj
 0001:0002f5bc       glEnable                   100305bc f   state.obj
 0001:0002f9f4       glDisable                  100309f4 f   state.obj
 0001:0002fecc       glAlphaFunc                10030ecc f   state.obj
 0001:0002fef0       glAlphaFuncx               10030ef0 f   state.obj
 0001:0002ff4c       glBlendEquationOES         10030f4c f   state.obj
 0001:0002ffd0       glBlendEquationSeparateOES 10030fd0 f   state.obj
 0001:00030204       glBlendFuncSeparateOES     10031204 f   state.obj
 0001:00030240       glBlendFunc                10031240 f   state.obj
 0001:00030274       glCullFace                 10031274 f   state.obj
 0001:000302e4       glDepthFunc                100312e4 f   state.obj
 0001:0003033c       glDepthMask                1003133c f   state.obj
 0001:00030388       glLineWidth                10031388 f   state.obj
 0001:00030458       glLineWidthx               10031458 f   state.obj
 0001:00030670       glPointSize                10031670 f   state.obj
 0001:0003068c       glPointSizex               1003168c f   state.obj
 0001:00030870       glPointParameterfv         10031870 f   state.obj
 0001:00030894       glPointParameterf          10031894 f   state.obj
 0001:000308ec       glPointParameterxv         100318ec f   state.obj
 0001:000309c0       glPointParameterx          100319c0 f   state.obj
 0001:00030a60       glFrontFace                10031a60 f   state.obj
 0001:00030ab8       glLogicOp                  10031ab8 f   state.obj
 0001:00030b10       glPolygonOffset            10031b10 f   state.obj
 0001:00030b84       glPolygonOffsetx           10031b84 f   state.obj
 0001:00030c58       glShadeModel               10031c58 f   state.obj
 0001:00030cc0       glStencilFunc              10031cc0 f   state.obj
 0001:00030d6c       glStencilOp                10031d6c f   state.obj
 0001:00030f2c       glStencilMask              10031f2c f   state.obj
 0001:00030f80       glColorMask                10031f80 f   state.obj
 0001:00031000       glSampleCoverage           10032000 f   state.obj
 0001:00031034       glSampleCoveragex          10032034 f   state.obj
 0001:00031094       HashTableCreate            10032094 f   statehash.obj
 0001:000310e8       HashTableDestroy           100320e8 f   statehash.obj
 0001:0003116c       HashFunc                   1003216c f   statehash.obj
 0001:0003119c       HashTableSearch            1003219c f   statehash.obj
 0001:00031254       HashTableDelete            10032254 f   statehash.obj
 0001:0003137c       HashTableInsert            1003237c f   statehash.obj
 0001:000315a0       CopyTexturePVRTC           100325a0 f   tex.obj
 0001:0003161c       CopyTextureETC1            1003261c f   tex.obj
 0001:0003169c       CopyTexture8888BGRAto8888RGBA 1003269c f   tex.obj
 0001:00031718       CopyTexture32Bits          10032718 f   tex.obj
 0001:00031770       CopyTexture16Bits          10032770 f   tex.obj
 0001:000317c8       CopyTexture8Bits           100327c8 f   tex.obj
 0001:0003181c       CopyTexture5551            1003281c f   tex.obj
 0001:0003187c       CopyTexture4444            1003287c f   tex.obj
 0001:000318dc       CopyTexture888X            100328dc f   tex.obj
 0001:00031950       CopyTexture888to565        10032950 f   tex.obj
 0001:000319d4       CopyTexture565toRGBX8888   100329d4 f   tex.obj
 0001:00031a54       CopyTexture5551to4444      10032a54 f   tex.obj
 0001:00031af8       CopyTexture5551toBGRA8888  10032af8 f   tex.obj
 0001:00031b88       CopyTexture5551toRGBA8888  10032b88 f   tex.obj
 0001:00031c18       CopyTexture4444to5551      10032c18 f   tex.obj
 0001:00031cb8       CopyTexture4444toBGRA8888  10032cb8 f   tex.obj
 0001:00031d38       CopyTexture4444toRGBA8888  10032d38 f   tex.obj
 0001:00031db8       CopyTextureRGBA8888to5551  10032db8 f   tex.obj
 0001:00031e48       CopyTextureBGRA8888to5551  10032e48 f   tex.obj
 0001:00031ed4       CopyTextureRGBA8888to4444  10032ed4 f   tex.obj
 0001:00031f64       CopyTextureBGRA8888to4444  10032f64 f   tex.obj
 0001:00032448       SetTextureFormat           10033448 f   tex.obj
 0001:000324e0       glActiveTexture            100334e0 f   tex.obj
 0001:00032524       BindTexture                10033524 f   tex.obj
 0001:00032690       glBindTexture              10033690 f   tex.obj
 0001:00032720       glDeleteTextures           10033720 f   tex.obj
 0001:00032828       glGenTextures              10033828 f   tex.obj
 0001:00032bf8       glTexImage2D               10033bf8 f   tex.obj
 0001:000330bc       glTexSubImage2D            100340bc f   tex.obj
 0001:000339c8       glCompressedTexImage2D     100349c8 f   tex.obj
 0001:00034090       glCompressedTexSubImage2D  10035090 f   tex.obj
 0001:00034248       glCopyTexImage2D           10035248 f   tex.obj
 0001:000348e4       glCopyTexSubImage2D        100358e4 f   tex.obj
 0001:00035748       glTexEnvfv                 10036748 f   tex.obj
 0001:00035774       glTexEnvf                  10036774 f   tex.obj
 0001:00035b88       glTexEnvxv                 10036b88 f   tex.obj
 0001:00035bb4       glTexEnvx                  10036bb4 f   tex.obj
 0001:00036058       glTexEnviv                 10037058 f   tex.obj
 0001:00036084       glTexEnvi                  10037084 f   tex.obj
 0001:000364ac       glTexParameterf            100374ac f   tex.obj
 0001:00036524       glTexParameterx            10037524 f   tex.obj
 0001:00036580       glTexParameteri            10037580 f   tex.obj
 0001:000365dc       glTexParameterfv           100375dc f   tex.obj
 0001:000366c4       glTexParameteriv           100376c4 f   tex.obj
 0001:0003673c       glTexParameterxv           1003773c f   tex.obj
 0001:00036808       glTexGeniOES               10037808 f   tex.obj
 0001:00036834       glTexGenivOES              10037834 f   tex.obj
 0001:00036860       glTexGenfOES               10037860 f   tex.obj
 0001:000368ac       glTexGenfvOES              100378ac f   tex.obj
 0001:000368f8       glTexGenxOES               100378f8 f   tex.obj
 0001:00036924       glTexGenxvOES              10037924 f   tex.obj
 0001:00036950       InitTexCombineState        10037950 f   texcombine.obj
 0001:000369d4       TexEnvCombine              100379d4 f   texcombine.obj
 0001:000371e0       HardwareSubTextureTwiddle  100381e0 f   texdata.obj
 0001:00037654       HardwareCopySubTextureTwiddle 10038654 f   texdata.obj
 0001:00037878       HardwareTextureTwiddle     10038878 f   texdata.obj
 0001:00037a9c       GetMipMapOffset            10038a9c f   texdata.obj
 0001:00037ac8       GetCompressedMipMapOffset  10038ac8 f   texdata.obj
 0001:00037b3c       TranslateLevel             10038b3c f   texdata.obj
 0001:00037de8       ReadBackTextureData        10038de8 f   texdata.obj
 0001:000380fc       SetupTwiddleFns            100390fc f   texdata.obj
 0001:00038160       CopyTextureData            10039160 f   texdata.obj
 0001:000381f0       ReclaimTextureMemFRM       100391f0 f   texmgmt.obj
 0001:000382c4       DestroyTextureGhostFRM     100392c4 f   texmgmt.obj
 0001:0003831c       CreateTextureMemory        1003931c f   texmgmt.obj
 0001:000384b0       TexMgrGhostTexture         100394b0 f   texmgmt.obj
 0001:00038598       TextureRemoveResident      10039598 f   texmgmt.obj
 0001:000385b0       TextureMakeResident        100395b0 f   texmgmt.obj
 0001:0003893c       IsTextureConsistent        1003993c f   texmgmt.obj
 0001:00038c58       TextureCreatePBufferLevel  10039c58 f   texmgmt.obj
 0001:00038e24       TextureCreateImageLevel    10039e24 f   texmgmt.obj
 0001:00039034       TextureCreateLevel         1003a034 f   texmgmt.obj
 0001:000391c8       CreateTexture              1003a1c8 f   texmgmt.obj
 0001:0003944c       CreateTextureState         1003a44c f   texmgmt.obj
 0001:000394e4       SetupTexNameArray          1003a4e4 f   texmgmt.obj
 0001:000394f4       ReleaseTextureManager      1003a4f4 f   texmgmt.obj
 0001:00039534       FreeTextureState           1003a534 f   texmgmt.obj
 0001:000395bc       SetupTextureState          1003a5bc f   texmgmt.obj
 0001:00039974       SetupTextureRenderTargetControlWords 1003a974 f   texmgmt.obj
 0001:00039a94       CreateTextureManager       1003aa94 f   texmgmt.obj
 0001:00039b6c       ReleasePbufferFromTexture  1003ab6c f   texrender.obj
 0001:00039b9c       GLESBindTexImage           1003ab9c f   texrender.obj
 0001:00039c34       GLESReleaseTexImage        1003ac34 f   texrender.obj
 0001:00039ddc       SetupYUVCoefficients       1003addc f   texstream.obj
 0001:0003a0dc       GetNumStreamDevices        1003b0dc f   texstream.obj
 0001:0003a110       FreeTexStreamState         1003b110 f   texstream.obj
 0001:0003a33c       FindBufferDevice           1003b33c f   texstream.obj
 0001:0003a374       AddBufferDevice            1003b374 f   texstream.obj
 0001:0003a62c       glGetTexStreamDeviceAttributeivIMG 1003b62c f   texstream.obj
 0001:0003a728       glTexBindStreamIMG         1003b728 f   texstream.obj
 0001:0003a858       glGetTexStreamDeviceNameIMG 1003b858 f   texstream.obj
 0001:0003a8d0       InitLightingState          1003b8d0 f   tnlapi.obj
 0001:0003aa3c       FreeLightingState          1003ba3c f   tnlapi.obj
 0001:0003aa7c       SetupTransformLightingProcs 1003ba7c f   tnlapi.obj
 0001:0003acb4       glLightModelfv             1003bcb4 f   tnlapi.obj
 0001:0003ad74       glLightModelf              1003bd74 f   tnlapi.obj
 0001:0003adbc       glLightModelxv             1003bdbc f   tnlapi.obj
 0001:0003aefc       glLightModelx              1003befc f   tnlapi.obj
 0001:0003b204       glLightf                   1003c204 f   tnlapi.obj
 0001:0003b264       glLightfv                  1003c264 f   tnlapi.obj
 0001:0003b290       glLightx                   1003c290 f   tnlapi.obj
 0001:0003b328       glLightxv                  1003c328 f   tnlapi.obj
 0001:0003b43c       Materialfv                 1003c43c f   tnlapi.obj
 0001:0003b650       glMaterialf                1003c650 f   tnlapi.obj
 0001:0003b69c       glMaterialfv               1003c69c f   tnlapi.obj
 0001:0003b6c8       glMaterialx                1003c6c8 f   tnlapi.obj
 0001:0003b74c       glMaterialxv               1003c74c f   tnlapi.obj
 0001:0003b878       ApplyViewport              1003c878 f   tnlapi.obj
 0001:0003ba18       glViewport                 1003ca18 f   tnlapi.obj
 0001:0003bb24       ApplyDepthRange            1003cb24 f   tnlapi.obj
 0001:0003bc24       glDepthRangef              1003cc24 f   tnlapi.obj
 0001:0003bc48       glDepthRangex              1003cc48 f   tnlapi.obj
 0001:0003bcd0       glMatrixMode               1003ccd0 f   tnlapi.obj
 0001:0003c0bc       glFrustumf                 1003d0bc f   tnlapi.obj
 0001:0003c10c       glFrustumx                 1003d10c f   tnlapi.obj
 0001:0003c5bc       glOrthof                   1003d5bc f   tnlapi.obj
 0001:0003c60c       glOrthox                   1003d60c f   tnlapi.obj
 0001:0003c764       glLoadIdentity             1003d764 f   tnlapi.obj
 0001:0003c780       glLoadMatrixf              1003d780 f   tnlapi.obj
 0001:0003c8ac       glLoadMatrixx              1003d8ac f   tnlapi.obj
 0001:0003cc28       glMultMatrixf              1003dc28 f   tnlapi.obj
 0001:0003ccf4       glMultMatrixx              1003dcf4 f   tnlapi.obj
 0001:0003d484       glRotatef                  1003e484 f   tnlapi.obj
 0001:0003d4c0       glRotatex                  1003e4c0 f   tnlapi.obj
 0001:0003d5b8       glScalef                   1003e5b8 f   tnlapi.obj
 0001:0003d5f8       glScalex                   1003e5f8 f   tnlapi.obj
 0001:0003d6cc       glTranslatef               1003e6cc f   tnlapi.obj
 0001:0003d70c       glTranslatex               1003e70c f   tnlapi.obj
 0001:0003d7e0       glPushMatrix               1003e7e0 f   tnlapi.obj
 0001:0003d7fc       glPopMatrix                1003e7fc f   tnlapi.obj
 0001:0003d818       glClipPlanef               1003e818 f   tnlapi.obj
 0001:0003d8a0       glClipPlanex               1003e8a0 f   tnlapi.obj
 0001:0003d9f8       GetFBBlendType             1003e9f8 f   usegles.obj
 0001:0003f1a4       WriteEOTUSSECode           100401a4 f   usegles.obj
 0001:0003f2a8       GetStateCopyUSEAddress     100402a8 f   usegles.obj
 0001:0003f3b4       InitSpecialUSECodeBlocks   100403b4 f   usegles.obj
 0001:0003f46c       FreeSpecialUSECodeBlocks   1004046c f   usegles.obj
 0001:0003fa38       SetupUSEVertexShader       10040a38 f   usegles.obj
 0001:0003fe68       SetupUSEFragmentShader     10040e68 f   usegles.obj
 0001:00040afc       WriteUSEVertexShaderMemConsts 10041afc f   usegles.obj
 0001:00040b98       AddInstruction             10041b98 f   useasmgles.obj
 0001:00040c9c       FreeUSEASMInstructionList  10041c9c f   useasmgles.obj
 0001:00040cf0       DuplicateUSEASMInstructionList 10041cf0 f   useasmgles.obj
 0001:00040e2c       AssembleUSEASMInstructions 10041e2c f   useasmgles.obj
 0001:0004103c       EncodeDmaBurst             1004203c f   validate.obj
 0001:000410e0       OutputTerminateState       100420e0 f   validate.obj
 0001:00041290       SetupPixelEventProgram     10042290 f   validate.obj
 0001:000432c4       DestroyHashedPDSFragSA     100442c4 f   validate.obj
 0001:000439f0       PatchPregenMTEStateCopyPrograms 100449f0 f   validate.obj
 0001:00043b40       WriteMTEStateCopyPrograms  10044b40 f   validate.obj
 0001:00043c94       SetupStateUpdate           10044c94 f   validate.obj
 0001:00043e9c       SetupMTEPregenBuffer       10044e9c f   validate.obj
 0001:00043ee8       SetupPDSVertexPregenBuffer 10044ee8 f   validate.obj
 0001:00044818       ValidateState              10045818 f   validate.obj
 0001:00044b38       GLES1EmitState             10045b38 f   validate.obj
 0001:00045368       glClientActiveTexture      10046368 f   vertex.obj
 0001:000453a0       glEnableClientState        100463a0 f   vertex.obj
 0001:00045484       glDisableClientState       10046484 f   vertex.obj
 0001:00045568       glColor4f                  10046568 f   vertex.obj
 0001:000455bc       glColor4x                  100465bc f   vertex.obj
 0001:000456c8       glColor4ub                 100466c8 f   vertex.obj
 0001:000457d8       glMultiTexCoord4f          100467d8 f   vertex.obj
 0001:0004582c       glMultiTexCoord4x          1004682c f   vertex.obj
 0001:00045934       glNormal3f                 10046934 f   vertex.obj
 0001:0004595c       glNormal3x                 1004695c f   vertex.obj
 0001:00045a10       glColorPointer             10046a10 f   vertex.obj
 0001:00045b2c       glNormalPointer            10046b2c f   vertex.obj
 0001:00045c44       glTexCoordPointer          10046c44 f   vertex.obj
 0001:00045d8c       glVertexPointer            10046d8c f   vertex.obj
 0001:00045ebc       glPointSizePointerOES      10046ebc f   vertex.obj
 0001:00045fa8       glMatrixIndexPointerOES    10046fa8 f   vertex.obj
 0001:00046098       glWeightPointerOES         10047098 f   vertex.obj
 0001:000461a0       glVertexAttribPointerARB   100471a0 f   vertex.obj
 0001:00046320       InitVertexArrayState       10047320 f   vertex.obj
 0001:000463cc       glVertexAttrib4fARB        100473cc f   vprogram.obj
 0001:0004641c       glProgramEnvParameter4fARB 1004741c f   vprogram.obj
 0001:00046498       glProgramEnvParameter4fvARB 10047498 f   vprogram.obj
 0001:00046518       glProgramLocalParameter4fARB 10047518 f   vprogram.obj
 0001:000465bc       glProgramLocalParameter4fvARB 100475bc f   vprogram.obj
 0001:00046660       glVertexAttrib4xIMG        10047660 f   vprogram.obj
 0001:00046764       glProgramLocalParameter4xIMG 10047764 f   vprogram.obj
 0001:000468b4       glProgramLocalParameter4xvIMG 100478b4 f   vprogram.obj
 0001:000469f4       glProgramEnvParameter4xIMG 100479f4 f   vprogram.obj
 0001:00046b20       glProgramEnvParameter4xvIMG 10047b20 f   vprogram.obj
 0001:00046c3c       glEnableVertexAttribArrayARB 10047c3c f   vprogram.obj
 0001:00046c80       glDisableVertexAttribArrayARB 10047c80 f   vprogram.obj
 0001:00046cc4       glProgramStringARB         10047cc4 f   vprogram.obj
 0001:00047fc4       glBindProgramARB           10048fc4 f   vprogram.obj
 0001:00048018       glDeleteProgramsARB        10049018 f   vprogram.obj
 0001:000480dc       glGenProgramsARB           100490dc f   vprogram.obj
 0001:00048128       CreateIMGVertexProgramState 10049128 f   vprogram.obj
 0001:00048170       FreeIMGVertexProgramState  10049170 f   vprogram.obj
 0001:00048230       SetupIMGVertexProgramNameArray 10049230 f   vprogram.obj
 0001:00048240       GetConstantFromBinding     10049240 f   vprogram.obj
 0001:00048988       OGL_GetTLSValue            10049988 f   wince6_tls.obj
 0001:000489b8       OGL_SetTLSValue            100499b8 f   wince6_tls.obj
 0001:000489fc       PDSGeneratePixelEventProgram 100499fc f   pds.obj
 0001:00048b18       PDSPatchVertexShaderProgram 10049b18 f   pds.obj
 0001:00048c44       PDSGeneratePixelShaderSAProgram 10049c44 f   pds.obj
 0001:00048eec       PDSGenerateStaticPixelShaderSAProgram 10049eec f   pds.obj
 0001:00049104       PDSGeneratePixelShaderProgram 1004a104 f   pds.obj
 0001:00049354       PDSGenerateStateCopyProgram 1004a354 f   pds.obj
 0001:000494c4       PDSGenerateStaticVertexShaderProgram 1004a4c4 f   pds.obj
 0001:00049908       PDSGenerateVertexShaderProgram 1004a908 f   pds.obj
 0001:00049fd4       PDSGenerateTerminateStateProgram 1004afd4 f   pds.obj
 0001:0004a07c       PDSPatchTerminateStateProgram 1004b07c f   pds.obj
 0001:0004a088       WriteEndOfPassUSSECode     1004b088 f   pixevent.obj
 0001:0004a0a0       WriteEndOfRenderUSSECode   1004b0a0 f   pixevent.obj
 0001:0004a0d0       WriteEndOfTileUSSECode     1004b0d0 f   pixevent.obj
 0001:0004a190       VPAssemblerError           1004b190 f   vpuscfns.obj
 0001:0004a1a0       VPUseAssemblerSetLabelAddress 1004b1a0 f   vpuscfns.obj
 0001:0004a1ac       VPUseAssemblerGetLabelName 1004b1ac f   vpuscfns.obj
 0001:0004a1b4       VPUseAssemblerGetLabelAddress 1004b1b4 f   vpuscfns.obj
 0001:0004a1c0       VPUseasmRealloc            1004b1c0 f   vpuscfns.obj
 0001:0004a1cc       VPAddRegToList             1004b1cc f   vpreg.obj
 0001:0004a22c       VPGetTemp                  1004b22c f   vpreg.obj
 0001:0004a338       VPReleaseReg               1004b338 f   vpreg.obj
 0001:0004a3c0       VPLoadConstant             1004b3c0 f   vpreg.obj
 0001:0004a984       VPGetRegfn                 1004b984 f   vpreg.obj
 0001:0004ab08       VPDestroyRegList           1004bb08 f   vpreg.obj
 0001:0004ab40       VP_COMMENT                 1004bb40 f   vpinst.obj
 0001:0004abac       VPCheckRegUsage            1004bbac f   vpinst.obj
 0001:0004ad08       VPGetUseInst               1004bd08 f   vpinst.obj
 0001:0004ad5c       VPEncodeReg                1004bd5c f   vpinst.obj
 0001:0004adfc       VPEncodeInstructionfn      1004bdfc f   vpinst.obj
 0001:0004af78       VPGenFreeProgram           1004bf78 f   vpcodegen.obj
 0001:0004affc       VPGenDestroyContext        1004bffc f   vpcodegen.obj
 0001:0004b020       VPGenCreateContext         1004c020 f   vpcodegen.obj
 0001:0004b040       VPAssignInputRegisters     1004c040 f   vpcodegen.obj
 0001:0004b1cc       VPAssignOutputRegisters    1004c1cc f   vpcodegen.obj
 0001:0004b444       VPAssignConstantRegisters  1004c444 f   vpcodegen.obj
 0001:0004b734       VPSelectRegister           1004c734 f   vpcodegen.obj
 0001:0004b908       VPConvert                  1004c908 f   vpcodegen.obj
 0001:0004b948       VP_PRINT_VGPBINARY         1004c948 f   vpcodegen.obj
 0001:0004b9b0       VPDisassembleVGPBinary     1004c9b0 f   vpcodegen.obj
 0001:0004d750       VPGenEmitVertexEnd         1004e750 f   vpcodegen.obj
 0001:0004d7a4       VPDestroyCode              1004e7a4 f   vpcodegen.obj
 0001:0004d7f4       VPGenerateCode             1004e7f4 f   vpcodegen.obj
 0001:0004db3c       InitVPState                1004eb3c f   vpgles.obj
 0001:0004db78       FreeVPState                1004eb78 f   vpgles.obj
 0001:0004db90       SetupVPShaderInputs        1004eb90 f   vpgles.obj
 0001:0004dc14       SetupVPShaderOutputs       1004ec14 f   vpgles.obj
 0001:0004dd00       UpdateVPShaderConstantsSize 1004ed00 f   vpgles.obj
 0001:0004dd50       SetupBuildVPShaderConstants 1004ed50 f   vpgles.obj
 0001:0004e088       SetupVPShader              1004f088 f   vpgles.obj
 0001:0004e160       eglGetError                1004f160 f   eglentrypoints.obj
 0001:0004e164       eglGetDisplay              1004f164 f   eglentrypoints.obj
 0001:0004e168       eglInitialize              1004f168 f   eglentrypoints.obj
 0001:0004e16c       eglTerminate               1004f16c f   eglentrypoints.obj
 0001:0004e170       eglQueryString             1004f170 f   eglentrypoints.obj
 0001:0004e174       eglGetProcAddress          1004f174 f   eglentrypoints.obj
 0001:0004e178       eglGetConfigs              1004f178 f   eglentrypoints.obj
 0001:0004e17c       eglChooseConfig            1004f17c f   eglentrypoints.obj
 0001:0004e198       eglGetConfigAttrib         1004f198 f   eglentrypoints.obj
 0001:0004e19c       eglCreateWindowSurface     1004f19c f   eglentrypoints.obj
 0001:0004e1a0       eglCreatePixmapSurface     1004f1a0 f   eglentrypoints.obj
 0001:0004e1a4       eglCreatePbufferSurface    1004f1a4 f   eglentrypoints.obj
 0001:0004e1a8       eglDestroySurface          1004f1a8 f   eglentrypoints.obj
 0001:0004e1ac       eglQuerySurface            1004f1ac f   eglentrypoints.obj
 0001:0004e1b0       eglCreateContext           1004f1b0 f   eglentrypoints.obj
 0001:0004e1b4       eglDestroyContext          1004f1b4 f   eglentrypoints.obj
 0001:0004e1b8       eglMakeCurrent             1004f1b8 f   eglentrypoints.obj
 0001:0004e1bc       eglGetCurrentContext       1004f1bc f   eglentrypoints.obj
 0001:0004e1c0       eglGetCurrentSurface       1004f1c0 f   eglentrypoints.obj
 0001:0004e1c4       eglGetCurrentDisplay       1004f1c4 f   eglentrypoints.obj
 0001:0004e1c8       eglQueryContext            1004f1c8 f   eglentrypoints.obj
 0001:0004e1cc       eglWaitGL                  1004f1cc f   eglentrypoints.obj
 0001:0004e1d0       eglWaitNative              1004f1d0 f   eglentrypoints.obj
 0001:0004e1d4       eglSwapBuffers             1004f1d4 f   eglentrypoints.obj
 0001:0004e1d8       eglCopyBuffers             1004f1d8 f   eglentrypoints.obj
 0001:0004e1dc       eglSwapInterval            1004f1dc f   eglentrypoints.obj
 0001:0004e1e0       eglSurfaceAttrib           1004f1e0 f   eglentrypoints.obj
 0001:0004e1e4       eglBindTexImage            1004f1e4 f   eglentrypoints.obj
 0001:0004e1e8       eglReleaseTexImage         1004f1e8 f   eglentrypoints.obj
 0001:0004e1ec       UCH_CodeHeapCreate         1004f1ec f   eurasiaconcmn:codeheap.obj
 0001:0004e2c4       UCH_CodeHeapDestroy        1004f2c4 f   eurasiaconcmn:codeheap.obj
 0001:0004e3f8       UCH_CodeHeapFreeFunc       1004f3f8 f   eurasiaconcmn:codeheap.obj
 0001:0004e44c       UCH_CodeHeapAllocateFunc   1004f44c f   eurasiaconcmn:codeheap.obj
 0001:0004e93c       CBUF_GetBufferSpace        1004f93c f   eurasiaconcmn:buffers.obj
 0001:0004eb7c       CBUF_UpdateBufferPos       1004fb7c f   eurasiaconcmn:buffers.obj
 0001:0004ebb8       CBUF_GetBufferDeviceAddress 1004fbb8 f   eurasiaconcmn:buffers.obj
 0001:0004ebdc       CBUF_UpdateBufferCommittedPrimOffsets 1004fbdc f   eurasiaconcmn:buffers.obj
 0001:0004ec64       CBUF_UpdateBufferCommittedHWOffsets 1004fc64 f   eurasiaconcmn:buffers.obj
 0001:0004eca8       CBUF_UpdateTACtrlKickBase  1004fca8 f   eurasiaconcmn:buffers.obj
 0001:0004ecf8       CBUF_CreateBuffer          1004fcf8 f   eurasiaconcmn:buffers.obj
 0001:0004ee38       CBUF_DestroyBuffer         1004fe38 f   eurasiaconcmn:buffers.obj
 0001:0004ee54       FRM_Initialize             1004fe54 f   eurasiaconcmn:frameresource.obj
 0001:0004f024       FRM_Attach                 10050024 f   eurasiaconcmn:frameresource.obj
 0001:0004f130       FRM_IsResourceNeeded       10050130 f   eurasiaconcmn:frameresource.obj
 0001:0004f21c       FRM_WaitForAllResources    1005021c f   eurasiaconcmn:frameresource.obj
 0001:0004f2a4       FRM_GhostResource          100502a4 f   eurasiaconcmn:frameresource.obj
 0001:0004f3b4       FRM_RemoveResourceFromAllLists 100503b4 f   eurasiaconcmn:frameresource.obj
 0001:0004f48c       FRM_RemoveSurfaceReferences 1005048c f   eurasiaconcmn:frameresource.obj
 0001:0004f4cc       FRM_Destroy                100504cc f   eurasiaconcmn:frameresource.obj
 0001:0004f634       FRM_ReclaimUnneededResources 10050634 f   eurasiaconcmn:frameresource.obj
 0001:0004f644       FRM_DestroyUnneededGhosts  10050644 f   eurasiaconcmn:frameresource.obj
 0001:000501ac       DeTwiddleAddress16bpp      100511ac f   eurasiaconcmn:twiddle.obj
 0001:00050324       ReadBackTwiddle16bpp       10051324 f   eurasiaconcmn:twiddle.obj
 0001:00050ef4       DeTwiddleAddress32bpp      10051ef4 f   eurasiaconcmn:twiddle.obj
 0001:00051068       ReadBackTwiddle32bpp       10052068 f   eurasiaconcmn:twiddle.obj
 0001:000511a0       ReadBackTwiddle8bpp        100521a0 f   eurasiaconcmn:twiddle.obj
 0001:00051284       ReadBackTwiddleETC1        10052284 f   eurasiaconcmn:twiddle.obj
 0001:00051418       DeTwiddleAddress8bpp       10052418 f   eurasiaconcmn:twiddle.obj
 0001:00051578       DeTwiddleAddressETC1       10052578 f   eurasiaconcmn:twiddle.obj
 0001:00061da0       UseAssembleInstruction     10062da0 f   useasm:useasm.obj
 0001:00062948       CheckUndefinedLabels       10063948 f   useasm:useasm.obj
 0001:000629bc       UseAssembler               100639bc f   useasm:useasm.obj
 0001:00062a3c       UseoptSetBit               10063a3c f   useasm:useopt.obj
 0001:00062f9c       InitSopSpec                10063f9c f   useasm:useopt.obj
 0001:00066208       UseoptProgram              10067208 f   useasm:useopt.obj
 0001:00066334       OpcodeArgumentCount        10067334 f   useasm:usetab.obj
 0001:0006634c       OpcodeName                 1006734c f   useasm:usetab.obj
 0001:00066360       OpcodeAcceptsSkipInv       10067360 f   useasm:usetab.obj
 0001:00066384       OpcodeAcceptsNoSched       10067384 f   useasm:usetab.obj
 0001:000663a8       GetFeatureEntry            100673a8 f   useasm:utils.obj
 0001:00066410       GetBugEntry                10067410 f   useasm:utils.obj
 0001:00066478       FixBRN21697                10067478 f   useasm:utils.obj
 0001:00066494       FixBRN21713                10067494 f   useasm:utils.obj
 0001:000664b0       FixBRN23062                100674b0 f   useasm:utils.obj
 0001:000664cc       FixBRN23164                100674cc f   useasm:utils.obj
 0001:000664e8       FixBRN23461                100674e8 f   useasm:utils.obj
 0001:00066504       FixBRN23960                10067504 f   useasm:utils.obj
 0001:00066520       FixBRN24895                10067520 f   useasm:utils.obj
 0001:0006653c       FixBRN25355                1006753c f   useasm:utils.obj
 0001:00066558       FixBRN25060                10067558 f   useasm:utils.obj
 0001:00066574       FixBRN25580                10067574 f   useasm:utils.obj
 0001:00066590       FixBRN25582                10067590 f   useasm:utils.obj
 0001:000665ac       FixBRN26570                100675ac f   useasm:utils.obj
 0001:000665c8       FixBRN26681                100675c8 f   useasm:utils.obj
 0001:000665e4       IsEnhancedNoSched          100675e4 f   useasm:utils.obj
 0001:00066600       IsHighPrecisionFIR         10067600 f   useasm:utils.obj
 0001:0006661c       IsLoadMOEStateFromRegisters 1006761c f   useasm:utils.obj
 0001:00066638       IsPerInstMoeIncrements     10067638 f   useasm:utils.obj
 0001:00066654       IsFClampInstruction        10067654 f   useasm:utils.obj
 0001:00066670       HasNewEfoOptions           10067670 f   useasm:utils.obj
 0001:0006668c       HasPackMultipleRoundModes  1006768c f   useasm:utils.obj
 0001:000666a8       HasNoInstructionPairing    100676a8 f   useasm:utils.obj
 0001:000666c4       NumberOfMutexesSupported   100676c4 f   useasm:utils.obj
 0001:000666d4       NumberOfMonitorsSupported  100676d4 f   useasm:utils.obj
 0001:000666e4       NumberOfProgramCounterBits 100676e4 f   useasm:utils.obj
 0001:000666f4       SupportsFmad16Swizzles     100676f4 f   useasm:utils.obj
 0001:00066710       SupportsFnormalise         10067710 f   useasm:utils.obj
 0001:0006672c       SupportsIndexTwoBanks      1006772c f   useasm:utils.obj
 0001:00066748       UseAsmInitInst             10067748 f   useasm:utils.obj
 0001:00066770       UseAsmInitReg              10067770 f   useasm:utils.obj
 0001:0006679c       PVRSRVCallocUserModeMem    1006779c f   srvclum:SRVCLUM.dll
 0001:000667ac       PVRSRVPollForValue         100677ac f   srvclum:SRVCLUM.dll
 0001:000667bc       PVRSRVFreeUserModeMem      100677bc f   srvclum:SRVCLUM.dll
 0001:000667cc       PVRSRVFreeDeviceMem        100677cc f   srvclum:SRVCLUM.dll
 0001:000667dc       PVRSRVMemCopy              100677dc f   srvclum:SRVCLUM.dll
 0001:000667ec       PVRSRVAllocDeviceMem       100677ec f   srvclum:SRVCLUM.dll
 0001:000667fc       PVRSRVAllocUserModeMem     100677fc f   srvclum:SRVCLUM.dll
 0001:0006680c       PVRSRVUnlockMutex          1006780c f   srvclum:SRVCLUM.dll
 0001:0006681c       PVRSRVLockMutex            1006781c f   srvclum:SRVCLUM.dll
 0001:0006682c       PVRSRVMemSet               1006782c f   srvclum:SRVCLUM.dll
 0001:0006683c       PVRSRVDestroyMutex         1006783c f   srvclum:SRVCLUM.dll
 0001:0006684c       PVRSRVCreateMutex          1006784c f   srvclum:SRVCLUM.dll
 0001:0006685c       PVRSRVReallocUserModeMem   1006785c f   srvclum:SRVCLUM.dll
 0001:0006686c       SGXQueueTransfer           1006786c f   srvclum:SRVCLUM.dll
 0001:0006687c       PVRSRVFreeAppHintState     1006787c f   srvclum:SRVCLUM.dll
 0001:0006688c       PVRSRVGetAppHint           1006788c f   srvclum:SRVCLUM.dll
 0001:0006689c       PVRSRVCreateAppHintState   1006789c f   srvclum:SRVCLUM.dll
 0001:000668ac       PVRSRVEventObjectWait      100678ac f   srvclum:SRVCLUM.dll
 0001:000668bc       SGXKickTA                  100678bc f   srvclum:SRVCLUM.dll
 0001:000668cc       PVRSRVEnumerateDeviceClass 100678cc f   srvclum:SRVCLUM.dll
 0001:000668dc       PVRSRVCloseBCDevice        100678dc f   srvclum:SRVCLUM.dll
 0001:000668ec       PVRSRVUnmapDeviceClassMemory 100678ec f   srvclum:SRVCLUM.dll
 0001:000668fc       PVRSRVMapDeviceClassMemory 100678fc f   srvclum:SRVCLUM.dll
 0001:0006690c       PVRSRVGetBCBuffer          1006790c f   srvclum:SRVCLUM.dll
 0001:0006691c       PVRSRVGetBCBufferInfo      1006791c f   srvclum:SRVCLUM.dll
 0001:0006692c       PVRSRVOpenBCDevice         1006792c f   srvclum:SRVCLUM.dll
 0001:0006693c       KEGLGetDrawableParameters  1006793c f   libimgegl:libIMGEGL.dll
 0001:0006694c       KEGLUnbindImage            1006794c f   libimgegl:libIMGEGL.dll
 0001:0006695c       KEGLBindImage              1006795c f   libimgegl:libIMGEGL.dll
 0001:0006696c       KEGLGetImageSource         1006796c f   libimgegl:libIMGEGL.dll
 0001:0006697c       KEGLDestroyRenderSurface   1006797c f   libimgegl:libIMGEGL.dll
 0001:0006698c       KEGLCreateRenderSurface    1006798c f   libimgegl:libIMGEGL.dll
 0001:0006699c       KEGLResizeRenderSurface    1006799c f   libimgegl:libIMGEGL.dll
 0001:000669ac       KEGLSurfaceUnbind          100679ac f   libimgegl:libIMGEGL.dll
 0001:000669bc       KEGLSurfaceBind            100679bc f   libimgegl:libIMGEGL.dll
 0001:000669cc       IMGeglGetError             100679cc f   libimgegl:libIMGEGL.dll
 0001:000669dc       IMGeglGetDisplay           100679dc f   libimgegl:libIMGEGL.dll
 0001:000669ec       IMGeglInitialize           100679ec f   libimgegl:libIMGEGL.dll
 0001:000669fc       IMGeglTerminate            100679fc f   libimgegl:libIMGEGL.dll
 0001:00066a0c       IMGeglQueryString          10067a0c f   libimgegl:libIMGEGL.dll
 0001:00066a1c       IMGeglGetProcAddress       10067a1c f   libimgegl:libIMGEGL.dll
 0001:00066a2c       IMGeglGetConfigs           10067a2c f   libimgegl:libIMGEGL.dll
 0001:00066a3c       IMGeglChooseConfig         10067a3c f   libimgegl:libIMGEGL.dll
 0001:00066a4c       IMGeglGetConfigAttrib      10067a4c f   libimgegl:libIMGEGL.dll
 0001:00066a5c       IMGeglCreateWindowSurface  10067a5c f   libimgegl:libIMGEGL.dll
 0001:00066a6c       IMGeglCreatePixmapSurface  10067a6c f   libimgegl:libIMGEGL.dll
 0001:00066a7c       IMGeglCreatePbufferSurface 10067a7c f   libimgegl:libIMGEGL.dll
 0001:00066a8c       IMGeglDestroySurface       10067a8c f   libimgegl:libIMGEGL.dll
 0001:00066a9c       IMGeglQuerySurface         10067a9c f   libimgegl:libIMGEGL.dll
 0001:00066aac       IMGeglCreateContext        10067aac f   libimgegl:libIMGEGL.dll
 0001:00066abc       IMGeglDestroyContext       10067abc f   libimgegl:libIMGEGL.dll
 0001:00066acc       IMGeglMakeCurrent          10067acc f   libimgegl:libIMGEGL.dll
 0001:00066adc       IMGeglGetCurrentContext    10067adc f   libimgegl:libIMGEGL.dll
 0001:00066aec       IMGeglGetCurrentSurface    10067aec f   libimgegl:libIMGEGL.dll
 0001:00066afc       IMGeglGetCurrentDisplay    10067afc f   libimgegl:libIMGEGL.dll
 0001:00066b0c       IMGeglQueryContext         10067b0c f   libimgegl:libIMGEGL.dll
 0001:00066b1c       IMGeglWaitGL               10067b1c f   libimgegl:libIMGEGL.dll
 0001:00066b2c       IMGeglWaitNative           10067b2c f   libimgegl:libIMGEGL.dll
 0001:00066b3c       IMGeglSwapBuffers          10067b3c f   libimgegl:libIMGEGL.dll
 0001:00066b4c       IMGeglCopyBuffers          10067b4c f   libimgegl:libIMGEGL.dll
 0001:00066b5c       IMGeglSwapInterval         10067b5c f   libimgegl:libIMGEGL.dll
 0001:00066b6c       IMGeglSurfaceAttrib        10067b6c f   libimgegl:libIMGEGL.dll
 0001:00066b7c       IMGeglBindTexImage         10067b7c f   libimgegl:libIMGEGL.dll
 0001:00066b8c       IMGeglReleaseTexImage      10067b8c f   libimgegl:libIMGEGL.dll
 0001:00066b9c       FFGenGenerateTNLProgram    10067b9c f   libffgen:ffgen.obj
 0001:00066ce4       FFGenFreeProgram           10067ce4 f   libffgen:ffgen.obj
 0001:00066d6c       FFTNLDestroyEntry          10067d6c f   libffgen:ffgen.obj
 0001:00066da0       FFGenCreateContext         10067da0 f   libffgen:ffgen.obj
 0001:00066e80       FFGenDestroyContext        10067e80 f   libffgen:ffgen.obj
 0001:00066edc       FFTNLCalculateTexCoordDimensions 10067edc f   libffgen:codegen.obj
 0001:00067068       FFTNLCalculateClipPlaneRequirements 10068068 f   libffgen:codegen.obj
 0001:000670fc       FFTNLAssignOutputRegisters 100680fc f   libffgen:codegen.obj
 0001:00067494       FFTNLRedirectOutputRegisterWrites 10068494 f   libffgen:codegen.obj
 0001:00067634       FFTNLGenTransformation     10068634 f   libffgen:codegen.obj
 0001:00068690       FFTNLGenClipping           10069690 f   libffgen:codegen.obj
 0001:00068820       FFTNLGenColours            10069820 f   libffgen:codegen.obj
 0001:000689e4       FFTNLGenFog                100699e4 f   libffgen:codegen.obj
 0001:00068e34       FFTNLGenVertexToEyeVector  10069e34 f   libffgen:codegen.obj
 0001:00069108       FFTNLGenPoints             1006a108 f   libffgen:codegen.obj
 0001:00069950       FFTNLGenLinearTexGenCode   1006a950 f   libffgen:codegen.obj
 0001:00069a78       FFTNLGenTexPassthroughCode 1006aa78 f   libffgen:codegen.obj
 0001:00069bc8       FFTNLGenTexturing          1006abc8 f   libffgen:codegen.obj
 0001:0006ab9c       FFTNLGenEmitVertexEnd      1006bb9c f   libffgen:codegen.obj
 0001:0006ac0c       FFTNLGenerateCode          1006bc0c f   libffgen:codegen.obj
 0001:0006af80       FFGENDestroyCode           1006bf80 f   libffgen:codegen.obj
 0001:0006b0b0       CompressFreeList           1006c0b0 f   libffgen:reg.obj
 0001:0006b224       ReleaseReg                 1006c224 f   libffgen:reg.obj
 0001:0006b3fc       LoadStoreConstant          1006c3fc f   libffgen:reg.obj
 0001:0006bf78       GetRegfn                   1006cf78 f   libffgen:reg.obj
 0001:0006c5f0       DestroyRegList             1006d5f0 f   libffgen:reg.obj
 0001:0006c644       DestroyInstructionList     1006d644 f   libffgen:inst.obj
 0001:0006c814       GetLabel                   1006d814 f   libffgen:inst.obj
 0001:0006c904       DestroyLabelList           1006d904 f   libffgen:inst.obj
 0001:0006c968       COMMENT                    1006d968 f   libffgen:inst.obj
 0001:0006c978       NEW_BLOCK                  1006d978 f   libffgen:inst.obj
 0001:0006cc68       EncodeInstructionfn        1006dc68 f   libffgen:inst.obj
 0001:0006d018       EncodeInstructionList      1006e018 f   libffgen:inst.obj
 0001:0006d094       GetDRC                     1006e094 f   libffgen:inst.obj
 0001:0006de74       M4x4                       1006ee74 f   libffgen:inst.obj
 0001:0006dfc0       M4x3                       1006efc0 f   libffgen:inst.obj
 0001:0006e1e4       IF_PRED                    1006f1e4 f   libffgen:inst.obj
 0001:0006e29c       ELSE_PRED                  1006f29c f   libffgen:inst.obj
 0001:0006e34c       END_PRED                   1006f34c f   libffgen:inst.obj
 0001:0006e3cc       AssemblerError             1006f3cc f   libffgen:uscfns.obj
 0001:0006e3dc       UseAssemblerSetLabelAddress 1006f3dc f   libffgen:uscfns.obj
 0001:0006e3e8       UseAssemblerGetLabelName   1006f3e8 f   libffgen:uscfns.obj
 0001:0006e3f0       UseAssemblerGetLabelAddress 1006f3f0 f   libffgen:uscfns.obj
 0001:0006e3fc       UseasmRealloc              1006f3fc f   libffgen:uscfns.obj
 0001:0006e418       FFTNLAddAmbientLight       1006f418 f   libffgen:lighting.obj
 0001:0006e6e0       FFTNLAddDiffuseLight       1006f6e0 f   libffgen:lighting.obj
 0001:0006e9b0       FFTNLAddSpecularLight      1006f9b0 f   libffgen:lighting.obj
 0001:0006ec84       FFTNLGenPointInfiniteLighting 1006fc84 f   libffgen:lighting.obj
 0001:0006f51c       FFTNLGenPointLocalLighting 1007051c f   libffgen:lighting.obj
 0001:000703b0       FFTNLGenSpotInfiniteLighting 100713b0 f   libffgen:lighting.obj
 0001:00071154       FFTNLGenSpotLocalLighting  10072154 f   libffgen:lighting.obj
 0001:000722bc       FFTNLGenOptimisedLighting  100732bc f   libffgen:lighting.obj
 0001:00072e58       TlsCall                    10073e58 f   coredll:COREDLL.dll
 0001:00072e68       TlsGetValue                10073e68 f   coredll:COREDLL.dll
 0001:00072e78       TlsSetValue                10073e78 f   coredll:COREDLL.dll
 0001:00072e88       DllMain                    10073e88 f   corelib0:dllmain.obj
 0001:00072fa4       _DllMainCRTStartup         10073fa4 f   corelib0:pegdmain.obj
 0001:00072fd4       __GSHandlerCheckCommon     10073fd4 f   corelib0:gshandler.obj
 0001:00073010       __GSHandlerCheck           10074010 f   corelib0:gshandler.obj
 0001:00073034       __security_init_cookie     10074034 f   corelib0:seccinit.obj
 0001:00073090       __security_check_cookie    10074090 f   corelib0:armsecgs.obj
 0001:000730a4       __gsfailure                100740a4 f   corelib0:armsecgs.obj
 0001:000731b0       _cexit                     100741b0 f   corelib0:cexit.obj
 0001:000731cc       _initterm                  100741cc f   corelib0:crt0dat.obj
 0001:00073200       _cinit                     10074200 f   corelib0:crt0dat.obj
 0001:00073234       memset                     10074234 f   corelib1:COREDLL.dll
 0001:00073244       memcpy                     10074244 f   corelib1:COREDLL.dll
 0001:00073254       strcmp                     10074254 f   corelib1:COREDLL.dll
 0001:00073264       vsprintf                   10074264 f   corelib1:COREDLL.dll
 0001:00073274       frexp                      10074274 f   corelib1:COREDLL.dll
 0001:00073284       sprintf                    10074284 f   corelib1:COREDLL.dll
 0001:00073294       printf                     10074294 f   corelib1:COREDLL.dll
 0001:000732a4       longjmp                    100742a4 f   corelib1:COREDLL.dll
 0001:000732b4       setjmp                     100742b4 f   corelib1:COREDLL.dll
 0001:000732c4       fclose                     100742c4 f   corelib1:COREDLL.dll
 0001:000732d4       fprintf                    100742d4 f   corelib1:COREDLL.dll
 0001:000732e4       fopen                      100742e4 f   corelib1:COREDLL.dll
 0001:000732f4       strcpy                     100742f4 f   corelib1:COREDLL.dll
 0001:00073304       strlen                     10074304 f   corelib1:COREDLL.dll
 0001:00073314       _XcptFilter                10074314 f   corelib1:COREDLL.dll
 0001:00073324       __C_specific_handler       10074324 f   corelib1:COREDLL.dll
 0001:00073334       __security_gen_cookie2     10074334 f   corelib1:COREDLL.dll
 0001:00073344       __report_gsfailure         10074344 f   corelib1:COREDLL.dll
 0001:00073354       free                       10074354 f   corelib1:COREDLL.dll
 0001:00073364       DisableThreadLibraryCalls  10074364 f   coredll:COREDLL.dll
 0001:00073374       TerminateProcess           10074374 f   coredll:COREDLL.dll
 0001:000733a8       __IMPORT_DESCRIPTOR_SRVCLUM 100743a8     srvclum:SRVCLUM.dll
 0001:000733bc       __IMPORT_DESCRIPTOR_libIMGEGL 100743bc     libimgegl:libIMGEGL.dll
 0001:000733d0       __IMPORT_DESCRIPTOR_COREDLL 100743d0     coredll:COREDLL.dll
 0001:000733e4       __NULL_IMPORT_DESCRIPTOR   100743e4     srvclum:SRVCLUM.dll
 0002:00000000       __imp_TerminateProcess     10076000     coredll:COREDLL.dll
 0002:00000004       __imp_memcpy               10076004     corelib1:COREDLL.dll
 0002:00000008       __imp___rt_udiv            10076008     corelib1:COREDLL.dll
 0002:0000000c       __imp___divs               1007600c     corelib1:COREDLL.dll
 0002:00000010       __imp___adds               10076010     corelib1:COREDLL.dll
 0002:00000014       __imp___subs               10076014     corelib1:COREDLL.dll
 0002:00000018       __imp___gts                10076018     corelib1:COREDLL.dll
 0002:0000001c       __imp___les                1007601c     corelib1:COREDLL.dll
 0002:00000020       __imp___ges                10076020     corelib1:COREDLL.dll
 0002:00000024       __imp___lts                10076024     corelib1:COREDLL.dll
 0002:00000028       __imp___itos               10076028     corelib1:COREDLL.dll
 0002:0000002c       __imp___utos               1007602c     corelib1:COREDLL.dll
 0002:00000030       __imp___muls               10076030     corelib1:COREDLL.dll
 0002:00000034       __imp_memset               10076034     corelib1:COREDLL.dll
 0002:00000038       __imp_TlsSetValue          10076038     coredll:COREDLL.dll
 0002:0000003c       __imp_TlsGetValue          1007603c     coredll:COREDLL.dll
 0002:00000040       __imp_TlsCall              10076040     coredll:COREDLL.dll
 0002:00000044       __imp___stou               10076044     corelib1:COREDLL.dll
 0002:00000048       __imp___eqs                10076048     corelib1:COREDLL.dll
 0002:0000004c       __imp_vsprintf             1007604c     corelib1:COREDLL.dll
 0002:00000050       __imp___nes                10076050     corelib1:COREDLL.dll
 0002:00000054       __imp_sqrt                 10076054     corelib1:COREDLL.dll
 0002:00000058       __imp___stod               10076058     corelib1:COREDLL.dll
 0002:0000005c       __imp_cos                  1007605c     corelib1:COREDLL.dll
 0002:00000060       __imp___dtos               10076060     corelib1:COREDLL.dll
 0002:00000064       __imp_DisableThreadLibraryCalls 10076064     coredll:COREDLL.dll
 0002:00000068       __imp_free                 10076068     corelib1:COREDLL.dll
 0002:0000006c       __imp___report_gsfailure   1007606c     corelib1:COREDLL.dll
 0002:00000070       __imp___security_gen_cookie2 10076070     corelib1:COREDLL.dll
 0002:00000074       __imp___C_specific_handler 10076074     corelib1:COREDLL.dll
 0002:00000078       __imp__XcptFilter          10076078     corelib1:COREDLL.dll
 0002:0000007c       __imp_strlen               1007607c     corelib1:COREDLL.dll
 0002:00000080       __imp_strcpy               10076080     corelib1:COREDLL.dll
 0002:00000084       __imp_fopen                10076084     corelib1:COREDLL.dll
 0002:00000088       __imp_fprintf              10076088     corelib1:COREDLL.dll
 0002:0000008c       __imp_fclose               1007608c     corelib1:COREDLL.dll
 0002:00000090       __imp_setjmp               10076090     corelib1:COREDLL.dll
 0002:00000094       __imp_longjmp              10076094     corelib1:COREDLL.dll
 0002:00000098       __imp___dtou               10076098     corelib1:COREDLL.dll
 0002:0000009c       __imp___addd               1007609c     corelib1:COREDLL.dll
 0002:000000a0       __imp___divd               100760a0     corelib1:COREDLL.dll
 0002:000000a4       __imp_log                  100760a4     corelib1:COREDLL.dll
 0002:000000a8       __imp___utod               100760a8     corelib1:COREDLL.dll
 0002:000000ac       __imp_printf               100760ac     corelib1:COREDLL.dll
 0002:000000b0       __imp_sin                  100760b0     corelib1:COREDLL.dll
 0002:000000b4       __imp_sprintf              100760b4     corelib1:COREDLL.dll
 0002:000000b8       __imp_frexp                100760b8     corelib1:COREDLL.dll
 0002:000000bc       __imp_sqrtf                100760bc     corelib1:COREDLL.dll
 0002:000000c0       __imp___stoi               100760c0     corelib1:COREDLL.dll
 0002:000000c4       __imp_floorf               100760c4     corelib1:COREDLL.dll
 0002:000000c8       __imp___muld               100760c8     corelib1:COREDLL.dll
 0002:000000cc       __imp___negs               100760cc     corelib1:COREDLL.dll
 0002:000000d0       __imp_strcmp               100760d0     corelib1:COREDLL.dll
 0002:000000d4       \177COREDLL_NULL_THUNK_DATA 100760d4     coredll:COREDLL.dll
 0002:000000d8       __imp_PVRSRVOpenBCDevice   100760d8     srvclum:SRVCLUM.dll
 0002:000000dc       __imp_PVRSRVGetBCBufferInfo 100760dc     srvclum:SRVCLUM.dll
 0002:000000e0       __imp_PVRSRVGetBCBuffer    100760e0     srvclum:SRVCLUM.dll
 0002:000000e4       __imp_PVRSRVMapDeviceClassMemory 100760e4     srvclum:SRVCLUM.dll
 0002:000000e8       __imp_PVRSRVCallocUserModeMem 100760e8     srvclum:SRVCLUM.dll
 0002:000000ec       __imp_PVRSRVUnmapDeviceClassMemory 100760ec     srvclum:SRVCLUM.dll
 0002:000000f0       __imp_PVRSRVCloseBCDevice  100760f0     srvclum:SRVCLUM.dll
 0002:000000f4       __imp_PVRSRVEnumerateDeviceClass 100760f4     srvclum:SRVCLUM.dll
 0002:000000f8       __imp_SGXKickTA            100760f8     srvclum:SRVCLUM.dll
 0002:000000fc       __imp_PVRSRVEventObjectWait 100760fc     srvclum:SRVCLUM.dll
 0002:00000100       __imp_PVRSRVCreateAppHintState 10076100     srvclum:SRVCLUM.dll
 0002:00000104       __imp_PVRSRVGetAppHint     10076104     srvclum:SRVCLUM.dll
 0002:00000108       __imp_PVRSRVFreeAppHintState 10076108     srvclum:SRVCLUM.dll
 0002:0000010c       __imp_SGXQueueTransfer     1007610c     srvclum:SRVCLUM.dll
 0002:00000110       __imp_PVRSRVReallocUserModeMem 10076110     srvclum:SRVCLUM.dll
 0002:00000114       __imp_PVRSRVCreateMutex    10076114     srvclum:SRVCLUM.dll
 0002:00000118       __imp_PVRSRVDestroyMutex   10076118     srvclum:SRVCLUM.dll
 0002:0000011c       __imp_PVRSRVMemSet         1007611c     srvclum:SRVCLUM.dll
 0002:00000120       __imp_PVRSRVLockMutex      10076120     srvclum:SRVCLUM.dll
 0002:00000124       __imp_PVRSRVUnlockMutex    10076124     srvclum:SRVCLUM.dll
 0002:00000128       __imp_PVRSRVAllocUserModeMem 10076128     srvclum:SRVCLUM.dll
 0002:0000012c       __imp_PVRSRVAllocDeviceMem 1007612c     srvclum:SRVCLUM.dll
 0002:00000130       __imp_PVRSRVMemCopy        10076130     srvclum:SRVCLUM.dll
 0002:00000134       __imp_PVRSRVFreeDeviceMem  10076134     srvclum:SRVCLUM.dll
 0002:00000138       __imp_PVRSRVFreeUserModeMem 10076138     srvclum:SRVCLUM.dll
 0002:0000013c       __imp_PVRSRVPollForValue   1007613c     srvclum:SRVCLUM.dll
 0002:00000140       \177SRVCLUM_NULL_THUNK_DATA 10076140     srvclum:SRVCLUM.dll
 0002:00000144       __imp_IMGeglReleaseTexImage 10076144     libimgegl:libIMGEGL.dll
 0002:00000148       __imp_IMGeglBindTexImage   10076148     libimgegl:libIMGEGL.dll
 0002:0000014c       __imp_IMGeglSwapInterval   1007614c     libimgegl:libIMGEGL.dll
 0002:00000150       __imp_IMGeglCopyBuffers    10076150     libimgegl:libIMGEGL.dll
 0002:00000154       __imp_IMGeglSwapBuffers    10076154     libimgegl:libIMGEGL.dll
 0002:00000158       __imp_IMGeglWaitNative     10076158     libimgegl:libIMGEGL.dll
 0002:0000015c       __imp_IMGeglWaitGL         1007615c     libimgegl:libIMGEGL.dll
 0002:00000160       __imp_IMGeglQueryContext   10076160     libimgegl:libIMGEGL.dll
 0002:00000164       __imp_IMGeglGetCurrentDisplay 10076164     libimgegl:libIMGEGL.dll
 0002:00000168       __imp_IMGeglGetCurrentSurface 10076168     libimgegl:libIMGEGL.dll
 0002:0000016c       __imp_IMGeglGetCurrentContext 1007616c     libimgegl:libIMGEGL.dll
 0002:00000170       __imp_IMGeglMakeCurrent    10076170     libimgegl:libIMGEGL.dll
 0002:00000174       __imp_IMGeglDestroyContext 10076174     libimgegl:libIMGEGL.dll
 0002:00000178       __imp_IMGeglCreateContext  10076178     libimgegl:libIMGEGL.dll
 0002:0000017c       __imp_IMGeglQuerySurface   1007617c     libimgegl:libIMGEGL.dll
 0002:00000180       __imp_IMGeglDestroySurface 10076180     libimgegl:libIMGEGL.dll
 0002:00000184       __imp_IMGeglCreatePbufferSurface 10076184     libimgegl:libIMGEGL.dll
 0002:00000188       __imp_IMGeglCreatePixmapSurface 10076188     libimgegl:libIMGEGL.dll
 0002:0000018c       __imp_IMGeglCreateWindowSurface 1007618c     libimgegl:libIMGEGL.dll
 0002:00000190       __imp_IMGeglGetConfigAttrib 10076190     libimgegl:libIMGEGL.dll
 0002:00000194       __imp_IMGeglChooseConfig   10076194     libimgegl:libIMGEGL.dll
 0002:00000198       __imp_IMGeglGetConfigs     10076198     libimgegl:libIMGEGL.dll
 0002:0000019c       __imp_IMGeglGetProcAddress 1007619c     libimgegl:libIMGEGL.dll
 0002:000001a0       __imp_IMGeglQueryString    100761a0     libimgegl:libIMGEGL.dll
 0002:000001a4       __imp_IMGeglTerminate      100761a4     libimgegl:libIMGEGL.dll
 0002:000001a8       __imp_IMGeglInitialize     100761a8     libimgegl:libIMGEGL.dll
 0002:000001ac       __imp_IMGeglGetDisplay     100761ac     libimgegl:libIMGEGL.dll
 0002:000001b0       __imp_IMGeglGetError       100761b0     libimgegl:libIMGEGL.dll
 0002:000001b4       __imp_KEGLSurfaceBind      100761b4     libimgegl:libIMGEGL.dll
 0002:000001b8       __imp_KEGLSurfaceUnbind    100761b8     libimgegl:libIMGEGL.dll
 0002:000001bc       __imp_KEGLResizeRenderSurface 100761bc     libimgegl:libIMGEGL.dll
 0002:000001c0       __imp_KEGLCreateRenderSurface 100761c0     libimgegl:libIMGEGL.dll
 0002:000001c4       __imp_KEGLDestroyRenderSurface 100761c4     libimgegl:libIMGEGL.dll
 0002:000001c8       __imp_KEGLGetImageSource   100761c8     libimgegl:libIMGEGL.dll
 0002:000001cc       __imp_KEGLBindImage        100761cc     libimgegl:libIMGEGL.dll
 0002:000001d0       __imp_KEGLUnbindImage      100761d0     libimgegl:libIMGEGL.dll
 0002:000001d4       __imp_KEGLGetDrawableParameters 100761d4     libimgegl:libIMGEGL.dll
 0002:000001d8       __imp_IMGeglSurfaceAttrib  100761d8     libimgegl:libIMGEGL.dll
 0002:000001dc       \177libIMGEGL_NULL_THUNK_DATA 100761dc     libimgegl:libIMGEGL.dll
 0002:000001e4       __security_cookie          100761e4     corelib0:seccinit.obj
 0002:000001e8       __security_cookie_complement 100761e8     corelib0:seccinit.obj
 0002:000001ec       _exitflag                  100761ec     corelib0:cexit.obj
 0002:000001f0       __onexitend                100761f0     <common>
 0002:000001f4       __onexitbegin              100761f4     <common>
 0002:000001f8       _pRawDllMain               100761f8     <common>

 entry point at        0001:00072fa4

 Static symbols

 0001:00012f70       SetupVerticesForAccum      10013f70 f   accum.obj
 0001:000132ec       SetupVerticesAndShaderForAccum 100142ec f   accum.obj
 0001:000139ac       WaitUntilBufObjNotUsed     100149ac f   bufobj.obj
 0001:00013a68       DisposeBufObject           10014a68 f   bufobj.obj
 0001:000142b0       SetupVerticesForClear      100152b0 f   clear.obj
 0001:00014600       SetupVerticesAndShaderForClear 10015600 f   clear.obj
 0001:00014858       SetupFragmentShaderForClear 10015858 f   clear.obj
 0001:00014f78       DrawTexture                10015f78 f   drawtex.obj
 0001:00015ca8       WriteDirect16Indices       10016ca8 f   drawvarray.obj
 0001:00015dc0       WriteLineStripOrLoop16Indices 10016dc0 f   drawvarray.obj
 0001:00015f0c       GetNumIndices              10016f0c f   drawvarray.obj
 0001:00015fa8       SetupStreamPointers        10016fa8 f   drawvarray.obj
 0001:000160a8       CopyVArrayData             100170a8 f   drawvarray.obj
 0001:00016170       CopyVArrayDataDeindex      10017170 f   drawvarray.obj
 0001:000162d8       GetVertexIndexBufferSpace  100172d8 f   drawvarray.obj
 0001:000163c8       CreateSequentialStaticIndices 100173c8 f   drawvarray.obj
 0001:0001646c       CreateLineStripStaticIndices 1001746c f   drawvarray.obj
 0001:00016514       GetVArrayBatchRewindCount  10017514 f   drawvarray.obj
 0001:0001658c       DrawVertexArray            1001758c f   drawvarray.obj
 0001:00016698       DrawArraysBatchedStaticIndices 10017698 f   drawvarray.obj
 0001:0001674c       DrawArraysAutoIndices      1001774c f   drawvarray.obj
 0001:00016850       DrawElementsDeindex        10017850 f   drawvarray.obj
 0001:000168bc       DrawElementsIndexBO        100178bc f   drawvarray.obj
 0001:0001699c       DrawBatchOnVBuffer         1001799c f   drawvarray.obj
 0001:00016ec0       PickDrawArraysProc         10017ec0 f   drawvarray.obj
 0001:00016fe4       PickDrawElementsProc       10017fe4 f   drawvarray.obj
 0001:0001711c       DetermineMinAndMaxIndices  1001811c f   drawvarray.obj
 0001:000171d4       TransformIndicesTo16Bits   100181d4 f   drawvarray.obj
 0001:00017310       AttachAllUsedVBOToCurrentKick 10018310 f   drawvarray.obj
 0001:000174d0       HandlePrimitiveTypeChange  100184d0 f   drawvarray.obj
 0001:00017ad0       MultiDrawArraysAutoIndices 10018ad0 f   drawvarray.obj
 0001:00017c58       MultiDrawBatchOnVBuffer    10018c58 f   drawvarray.obj
 0001:000181b0       MultiDrawVertexArray       100191b0 f   drawvarray.obj
 0001:000183a0       MultiDrawElementsDeindex   100193a0 f   drawvarray.obj
 0001:00018510       MultiDrawElementsIndexBO   10019510 f   drawvarray.obj
 0001:0001867c       PickMultiDrawElementsProc  1001967c f   drawvarray.obj
 0001:00019084       FreeContextSharedState     1001a084 f   eglglue.obj
 0001:000191ec       CreateSharedState          1001a1ec f   eglglue.obj
 0001:000193f8       InitContext                1001a3f8 f   eglglue.obj
 0001:00019a2c       DeInitContext              1001aa2c f   eglglue.obj
 0001:00019b28       GLESCreateGC               1001ab28 f   eglglue.obj
 0001:00019b9c       GLESDestroyGC              1001ab9c f   eglglue.obj
 0001:00019bcc       GLESMakeCurrentGC          1001abcc f   eglglue.obj
 0001:00019d2c       GLESMakeUnCurrentGC        1001ad2c f   eglglue.obj
 0001:00019d88       GLESFlushBuffersGC         1001ad88 f   eglglue.obj
 0001:00019dfc       GLESMarkRenderSurfaceAsInvalid 1001adfc f   eglglue.obj
 0001:00019e00       GLESGetProcAddress         1001ae00 f   eglglue.obj
 0001:0001ae40       FreeFrameBuffer            1001be40 f   fbo.obj
 0001:0001af48       DisposeFrameBufferObject   1001bf48 f   fbo.obj
 0001:0001af4c       DisposeRenderBuffer        1001bf4c f   fbo.obj
 0001:0001b314       ComputeFrameBufferCompleteness 1001c314 f   fbo.obj
 0001:0001b80c       NotifyFrameBuffer          1001c80c f   fbo.obj
 0001:0001caa8       Fogfv                      1001daa8 f   fog.obj
 0001:0001cfac       SetupBlendingOPs           1001dfac f   fftex.obj
 0001:0001d414       ReuseHashedBlendState      1001e414 f   fftex.obj
 0001:0001d8c4       AllocateTempReg            1001e8c4 f   fftexhw.obj
 0001:0001d920       SetupColourSourceRegTypeNum 1001e920 f   fftexhw.obj
 0001:0001d9d8       SetupAlphaSourceRegTypeNum 1001e9d8 f   fftexhw.obj
 0001:0001da90       EncodeFPMA                 1001ea90 f   fftexhw.obj
 0001:0001ddd0       SetupSourcesForSOP2        1001edd0 f   fftexhw.obj
 0001:0001e140       EncodeRestrictedBlend      1001f140 f   fftexhw.obj
 0001:0001e758       IntegerCopy                1001f758 f   fftexhw.obj
 0001:0001e7f0       SetupTwoSidedColour        1001f7f0 f   fftexhw.obj
 0001:0001e98c       IntegerCombineColorAndAlpha 1001f98c f   fftexhw.obj
 0001:0001ebf4       IntegerADDSIGNEDSOP2       1001fbf4 f   fftexhw.obj
 0001:0001ee64       IntegerConvertTextureFormat 1001fe64 f   fftexhw.obj
 0001:0001f128       CalculateSourceInformation 10020128 f   fftexhw.obj
 0001:0001f58c       EncodeYUVColourSpaceConversion 1002058c f   fftexhw.obj
 0001:0001fa98       EncodeYUV420ColourSpaceConversion 10020a98 f   fftexhw.obj
 0001:0001ffa8       LoadFPMASpecialConstant    10020fa8 f   fftexhw.obj
 0001:00020010       EncodeFPMAReplace          10021010 f   fftexhw.obj
 0001:000200d8       EncodeGeneralAlphaBlend    100210d8 f   fftexhw.obj
 0001:0002047c       IntegerScaleColorAndAlpha  1002147c f   fftexhw.obj
 0001:000206f0       EncodeDOT3                 100216f0 f   fftexhw.obj
 0001:0002090c       EncodeGeneralColorBlend    1002190c f   fftexhw.obj
 0001:00020d44       EncodeGeneralADDSIGNEDBlend 10021d44 f   fftexhw.obj
 0001:0002103c       IntegerSetupTextureBlend   1002203c f   fftexhw.obj
 0001:0002181c       GetFFTNLGenDesc            1002281c f   fftnlgles.obj
 0001:00021e7c       SetupFFTNLShaderInputs     10022e7c f   fftnlgles.obj
 0001:00022f74       ConvertResult              10023f74 f   get.obj
 0001:00023478       GetBlendFactor             10024478 f   get.obj
 0001:00023518       GetStencilOp               10024518 f   get.obj
 0001:000235a8       GetTexParameter            100245a8 f   get.obj
 0001:000237b4       GetTexEnvCombine           100247b4 f   get.obj
 0001:00023ad8       GetTexEnvfv                10024ad8 f   get.obj
 0001:00023d44       GetLightfv                 10024d44 f   get.obj
 0001:00023e7c       GetMaterialfv              10024e7c f   get.obj
 0001:00023f8c       IsEnabled                  10024f8c f   get.obj
 0001:00024fe4       DoGet                      10025fe4 f   get.obj
 0001:000266b0       HardwareMipTextureTransfer 100276b0 f   makemips.obj
 0001:000268a8       HardwareMipGen             100278a8 f   makemips.obj
 0001:00026a54       MakeMapLevel8bpp           10027a54 f   makemips.obj
 0001:00026b48       MakeMapLevel16bpp          10027b48 f   makemips.obj
 0001:00026e6c       MakeMapLevel32bpp          10027e6c f   makemips.obj
 0001:00027044       SetupMipmapTextureControlWords 10028044 f   makemips.obj
 0001:000279c8       XForm2                     100289c8 f   matrix.obj
 0001:00027b7c       XForm3                     10028b7c f   matrix.obj
 0001:00027e04       XForm4                     10028e04 f   matrix.obj
 0001:0002c324       CheckReadPixelArgs         1002d324 f   pixop.obj
 0001:0002cc80       DestroyUSEShaderVariant    1002dc80 f   shader.obj
 0001:0002cf08       CalcRegionClip             1002df08 f   scissor.obj
 0001:0002cfc8       SetupVerticesForDrawmask   1002dfc8 f   scissor.obj
 0001:0002d274       SetupVerticesAndShaderForDrawmask 1002e274 f   scissor.obj
 0001:0002d4c0       SendDrawMaskRect           1002e4c0 f   scissor.obj
 0001:0002dba4       SetupZLSRegs               1002eba4 f   sgxif.obj
 0001:0002dd74       GLESInitRegs               1002ed74 f   sgxif.obj
 0001:0002de38       StartFrame                 1002ee38 f   sgxif.obj
 0001:0002e250       DoKickTA                   1002f250 f   sgxif.obj
 0001:0002fe38       SetUpAlphaTestParams       10030e38 f   state.obj
 0001:00030084       BlendFuncSeparate          10031084 f   state.obj
 0001:0003052c       PointSize                  1003152c f   state.obj
 0001:000306e0       PointParameterfv           100316e0 f   state.obj
 0001:00031490       ConvertFactorColor         10032490 f   tex.obj
 0001:00031ff0       Copy888Palette4Span        10032ff0 f   tex.obj
 0001:0003205c       Copy888Palette4Level1xN    1003305c f   tex.obj
 0001:0003210c       Copy888Palette8Span        1003310c f   tex.obj
 0001:00032144       Copy8888Palette4Span       10033144 f   tex.obj
 0001:00032170       Copy8888Palette4Level1xN   10033170 f   tex.obj
 0001:000321bc       Copy8888Palette8Span       100331bc f   tex.obj
 0001:000321d8       Copy565Palette4Span        100331d8 f   tex.obj
 0001:0003220c       Copy565Palette4Level1xN    1003320c f   tex.obj
 0001:00032268       Copy565Palette8Span        10033268 f   tex.obj
 0001:00032288       Copy4444Palette4Span       10033288 f   tex.obj
 0001:000322cc       Copy4444Palette4Level1xN   100332cc f   tex.obj
 0001:00032340       Copy4444Palette8Span       10033340 f   tex.obj
 0001:00032368       Copy5551Palette4Span       10033368 f   tex.obj
 0001:000323ac       Copy5551Palette4Level1xN   100333ac f   tex.obj
 0001:00032420       Copy5551Palette8Span       10033420 f   tex.obj
 0001:00032874       CheckTexImageArgs          10033874 f   tex.obj
 0001:00032970       CheckTexSubImageArgs       10033970 f   tex.obj
 0001:00032afc       UpdateEGLImage             10033afc f   tex.obj
 0001:000354d0       TexEnvfv                   100364d0 f   tex.obj
 0001:00035878       TexEnvxv                   10036878 f   tex.obj
 0001:00035cb8       TexEnviv                   10036cb8 f   tex.obj
 0001:00036188       TexParameterfv             10037188 f   tex.obj
 0001:000367b4       TexGenfv                   100377b4 f   tex.obj
 0001:00036f14       HardwareTextureTransfer    10037f14 f   texdata.obj
 0001:0003880c       UnloadInconsistentTexture  1003980c f   texmgmt.obj
 0001:000392b8       FreeTexture                1003a2b8 f   texmgmt.obj
 0001:00039448       DisposeTexObj              1003a448 f   texmgmt.obj
 0001:00039c7c       InitialiseYUVCoefficients  1003ac7c f   texstream.obj
 0001:0003a1a8       CreateTextureStreamState   1003b1a8 f   texstream.obj
 0001:0003aaf4       TransformLightDirection    1003baf4 f   tnlapi.obj
 0001:0003af44       Lightfv                    1003bf44 f   tnlapi.obj
 0001:0003bdec       Frustumf                   1003cdec f   tnlapi.obj
 0001:0003c264       Orthof                     1003d264 f   tnlapi.obj
 0001:0003d038       Rotatef                    1003e038 f   tnlapi.obj
 0001:0003db08       CreateFBBlendUSEASMCode    1003eb08 f   usegles.obj
 0001:0003e030       CreateLogicalOpsUSEASMCode 1003f030 f   usegles.obj
 0001:0003ecc4       CreateColorMaskUSEASMCode  1003fcc4 f   usegles.obj
 0001:0003ee74       CreateFogUSEASMCode        1003fe74 f   usegles.obj
 0001:0003f2d8       InitStateCopyUSECodeBlocks 100402d8 f   usegles.obj
 0001:0003f4a8       CreateVertexUnpackUSECode  100404a8 f   usegles.obj
 0001:0003fc20       SetupIteratorsAndTextureLookups 10040c20 f   usegles.obj
 0001:00040da8       UseAssemblerError          10041da8 f   useasmgles.obj
 0001:00040dfc       UseAssemblerSetLabelAddress 10041dfc f   useasmgles.obj
 0001:00040e00       UseAssemblerGetLabelName   10041e00 f   useasmgles.obj
 0001:00040e08       UseAssemblerGetLabelAddress 10041e08 f   useasmgles.obj
 0001:00040e10       UseasmRealloc              10041e10 f   useasmgles.obj
 0001:00040e1c       UseasmAlloc                10041e1c f   useasmgles.obj
 0001:00040e24       UseasmFree                 10041e24 f   useasmgles.obj
 0001:000415dc       WritePDSPixelShaderProgram 100425dc f   validate.obj
 0001:00041ccc       PatchAuxiliaryPDSVertexShaderProgram 10042ccc f   validate.obj
 0001:00041ec4       WritePDSStaticVertexShaderProgram 10042ec4 f   validate.obj
 0001:000425a0       WritePDSVertexShaderProgram 100435a0 f   validate.obj
 0001:00042de8       LoadSecondaryAttributes    10043de8 f   validate.obj
 0001:00042fc0       WritePDSUSEShaderSAProgram 10043fc0 f   validate.obj
 0001:000432e8       WriteStaticPDSPixelSAProgram 100442e8 f   validate.obj
 0001:00043790       WriteMTEState              10044790 f   validate.obj
 0001:00043d88       GenerateVertexCompileMask  10044d88 f   validate.obj
 0001:00043fc0       SetupAttribStreams         10044fc0 f   validate.obj
 0001:000441ac       SetupRenderState           100451ac f   validate.obj
 0001:00044684       WriteVDMControlStream      10045684 f   validate.obj
 0001:00044e94       Copy1Byte                  10045e94 f   vertex.obj
 0001:00044eb4       Copy3Bytes                 10045eb4 f   vertex.obj
 0001:00044eec       Copy1Short                 10045eec f   vertex.obj
 0001:00044f14       Copy3Shorts                10045f14 f   vertex.obj
 0001:00044f50       Copy1Long                  10045f50 f   vertex.obj
 0001:00044f74       Copy2Longs                 10045f74 f   vertex.obj
 0001:00044fa8       Copy3Longs                 10045fa8 f   vertex.obj
 0001:00044fe4       Copy4Longs                 10045fe4 f   vertex.obj
 0001:00045028       MemCopy1Byte               10046028 f   vertex.obj
 0001:00045044       MemCopy3Bytes              10046044 f   vertex.obj
 0001:00045060       MemCopy1Short              10046060 f   vertex.obj
 0001:0004507c       MemCopy3Shorts             1004607c f   vertex.obj
 0001:0004509c       MemCopy1Long               1004609c f   vertex.obj
 0001:000450b8       MemCopy2Longs              100460b8 f   vertex.obj
 0001:000450d4       MemCopy3Longs              100460d4 f   vertex.obj
 0001:000450f4       MemCopy4Longs              100460f4 f   vertex.obj
 0001:00045110       Copy2Bytes                 10046110 f   vertex.obj
 0001:00045140       Copy4Bytes                 10046140 f   vertex.obj
 0001:00045180       Copy6Bytes                 10046180 f   vertex.obj
 0001:000451bc       Copy8Bytes                 100461bc f   vertex.obj
 0001:000451f8       Copy12Bytes                100461f8 f   vertex.obj
 0001:00045234       Copy16Bytes                10046234 f   vertex.obj
 0001:00045270       Copy2Shorts                10046270 f   vertex.obj
 0001:000452a4       Copy4Shorts                100462a4 f   vertex.obj
 0001:000452e8       Copy6Shorts                100462e8 f   vertex.obj
 0001:00045328       Copy8Shorts                10046328 f   vertex.obj
 0001:00047ed8       BindProgram                10048ed8 f   vprogram.obj
 0001:000481ec       DisposeProgram             100491ec f   vprogram.obj
 0001:00048a9c       PDSEncodeSimpleMOVS        10049a9c f   pds.obj
 0001:00048bbc       PDSGetNextConstant         10049bbc f   pds.obj
 0001:00048c00       PDSGetNumConstants         10049c00 f   pds.obj
 0001:0004e330       CodeHeapInsertBlockInFreeList 1004f330 f   eurasiaconcmn:codeheap.obj
 0001:0004e76c       GetBufferSpaceLeftInBytes  1004f76c f   eurasiaconcmn:buffers.obj
 0001:0004e7d4       CheckUSSEBufferSpace       1004f7d4 f   eurasiaconcmn:buffers.obj
 0001:0004e8a8       CheckTACtrlBufferSpace     1004f8a8 f   eurasiaconcmn:buffers.obj
 0001:0004ef6c       AllocAttachment            1004ff6c f   eurasiaconcmn:frameresource.obj
 0001:0004f190       WaitUntilResourceIsNotNeeded 10050190 f   eurasiaconcmn:frameresource.obj
 0001:0004f2f8       RemoveResourceFromAllLists 100502f8 f   eurasiaconcmn:frameresource.obj
 0001:0004f3e0       RemoveSurfaceReferencesInList 100503e0 f   eurasiaconcmn:frameresource.obj
 0001:0004f540       ReclaimUnneededResourcesInList 10050540 f   eurasiaconcmn:frameresource.obj
 0001:0004f654       InitLookupTable32          10050654 f   eurasiaconcmn:twiddle.obj
 0001:0004f79c       Write8x8Pixels16bpp        1005079c f   eurasiaconcmn:twiddle.obj
 0001:0004fa70       TwiddleSmallTexture16bpp   10050a70 f   eurasiaconcmn:twiddle.obj
 0001:0004fbf4       Twiddle32x3216bpp          10050bf4 f   eurasiaconcmn:twiddle.obj
 0001:0004fddc       RecursiveTwid16bpp         10050ddc f   eurasiaconcmn:twiddle.obj
 0001:0004fea8       TwiddleRectangularTexture16bpp 10050ea8 f   eurasiaconcmn:twiddle.obj
 0001:0005024c       Untwiddle16Bpp             1005124c f   eurasiaconcmn:twiddle.obj
 0001:0005045c       Write8x8Pixels32bpp        1005145c f   eurasiaconcmn:twiddle.obj
 0001:000507a4       TwiddleSmallTexture32bpp   100517a4 f   eurasiaconcmn:twiddle.obj
 0001:00050928       Twiddle32x3232bpp          10051928 f   eurasiaconcmn:twiddle.obj
 0001:00050b00       RecursiveTwid32bpp         10051b00 f   eurasiaconcmn:twiddle.obj
 0001:00050bcc       TwiddleRectangularTexture32bpp 10051bcc f   eurasiaconcmn:twiddle.obj
 0001:00050f94       Untwiddle32bpp             10051f94 f   eurasiaconcmn:twiddle.obj
 0001:00051390       getUV                      10052390 f   eurasiaconcmn:twiddle.obj
 0001:000516f4       SetLabelAddress            100526f4 f   useasm:useasm.obj
 0001:000518c0       FixupLabelAddresses        100528c0 f   useasm:useasm.obj
 0001:00051a14       GetLabelAddress            10052a14 f   useasm:useasm.obj
 0001:00051b38       CheckArgFlags              10052b38 f   useasm:useasm.obj
 0001:00051dc4       CheckFlags                 10052dc4 f   useasm:useasm.obj
 0001:00052508       EncodeIndex                10053508 f   useasm:useasm.obj
 0001:000526b8       EncodeDestBankAndNum       100536b8 f   useasm:useasm.obj
 0001:00052a34       EncodeDest                 10053a34 f   useasm:useasm.obj
 0001:00052a88       GetSrc0EncodedBankAndNumber 10053a88 f   useasm:useasm.obj
 0001:00052cf0       EncodeSrc0                 10053cf0 f   useasm:useasm.obj
 0001:00052d48       GetSrc1EncodedBankAndNumber 10053d48 f   useasm:useasm.obj
 0001:00053240       EncodeSrc1                 10054240 f   useasm:useasm.obj
 0001:000532b4       GetSrc2EncodedBankAndNumber 100542b4 f   useasm:useasm.obj
 0001:00053770       EncodeSrc2                 10054770 f   useasm:useasm.obj
 0001:000537e4       EncodePredicate            100547e4 f   useasm:useasm.obj
 0001:000538cc       AssembleDot34              100548cc f   useasm:useasm.obj
 0001:000543a8       EncodeTestInstruction_AluOp 100553a8 f   useasm:useasm.obj
 0001:000546f8       EncodeTestInstruction_Repeat 100556f8 f   useasm:useasm.obj
 0001:000548e4       EncodeTestInstruction      100558e4 f   useasm:useasm.obj
 0001:00054f78       EncodeFloatInstruction     10055f78 f   useasm:useasm.obj
 0001:00055600       EncodeNormaliseInstruction 10056600 f   useasm:useasm.obj
 0001:00055c1c       EncodeSOP2Instruction      10056c1c f   useasm:useasm.obj
 0001:00056648       EncodePackInstruction      10057648 f   useasm:useasm.obj
 0001:00056dac       EncodeBitwiseInstruction   10057dac f   useasm:useasm.obj
 0001:00057298       ExpandMacros               10058298 f   useasm:useasm.obj
 0001:00057ccc       EncodeFDPCInstruction      10058ccc f   useasm:useasm.obj
 0001:00057fa4       EncodeFDDPInstruction      10058fa4 f   useasm:useasm.obj
 0001:000582ec       EncodeFDDPCInstruction     100592ec f   useasm:useasm.obj
 0001:000586dc       EncodeMovcInstruction      100596dc f   useasm:useasm.obj
 0001:00058a3c       EncodeEfoInstruction       10059a3c f   useasm:useasm.obj
 0001:00058d64       EncodeSOPWMInstruction     10059d64 f   useasm:useasm.obj
 0001:00059398       EncodeLRP1Instruction      1005a398 f   useasm:useasm.obj
 0001:00059ba4       EncodeLRP2Instruction      1005aba4 f   useasm:useasm.obj
 0001:0005a448       EncodeSOP3Instruction      1005b448 f   useasm:useasm.obj
 0001:0005afe4       EncodeFPMAInstruction      1005bfe4 f   useasm:useasm.obj
 0001:0005b688       EncodeIMA16Instruction     1005c688 f   useasm:useasm.obj
 0001:0005bbe0       EncodeIMAEInstruction      1005cbe0 f   useasm:useasm.obj
 0001:0005c228       EncodeADIFInstruction      1005d228 f   useasm:useasm.obj
 0001:0005c510       EncodeSSUM16Instruction    1005d510 f   useasm:useasm.obj
 0001:0005cab0       EncodeFIRVInstruction      1005dab0 f   useasm:useasm.obj
 0001:0005cfc0       EncodeFIRVHInstruction     1005dfc0 f   useasm:useasm.obj
 0001:0005d380       EncodeBILINInstruction     1005e380 f   useasm:useasm.obj
 0001:0005d8e8       EncodeFIRHInstruction      1005e8e8 f   useasm:useasm.obj
 0001:0005de98       EncodeFIRHHInstruction     1005ee98 f   useasm:useasm.obj
 0001:0005e498       EncodeSMPInstruction       1005f498 f   useasm:useasm.obj
 0001:0005ea04       EncodeLDSTCacheFlags       1005fa04 f   useasm:useasm.obj
 0001:0005eacc       EncodeLDSTInstruction      1005facc f   useasm:useasm.obj
 0001:0005f17c       EncodeBAInstruction        1006017c f   useasm:useasm.obj
 0001:0005f308       EncodeLAPCInstruction      10060308 f   useasm:useasm.obj
 0001:0005f3c4       EncodeBRInstruction        100603c4 f   useasm:useasm.obj
 0001:0005f554       EncodeIDFInstruction       10060554 f   useasm:useasm.obj
 0001:0005f738       EncodeWDFInstruction       10060738 f   useasm:useasm.obj
 0001:0005f840       EncodeEmitInstruction      10060840 f   useasm:useasm.obj
 0001:0005fce8       EncodeSMOAInstruction      10060ce8 f   useasm:useasm.obj
 0001:00060008       EncodeSMLSIInstruction     10061008 f   useasm:useasm.obj
 0001:00060500       EncodeMOEInstruction       10061500 f   useasm:useasm.obj
 0001:0006081c       EncodeSETFCInstruction     1006181c f   useasm:useasm.obj
 0001:00060968       EncodeMOVInstruction       10061968 f   useasm:useasm.obj
 0001:00060e50       EncodeMutexInstruction     10061e50 f   useasm:useasm.obj
 0001:00060fa8       EncodeLDRSTRInstruction    10061fa8 f   useasm:useasm.obj
 0001:00061394       EncodePTOFFPCOEFFInstruction 10062394 f   useasm:useasm.obj
 0001:00061510       EncodeATST8Instruction     10062510 f   useasm:useasm.obj
 0001:000618b0       EncodeDEPTHFInstruction    100628b0 f   useasm:useasm.obj
 0001:00061b34       EncodeSETMInstruction      10062b34 f   useasm:useasm.obj
 0001:00061c90       EncodeWOPInstruction       10062c90 f   useasm:useasm.obj
 0001:00062a64       UseoptAlloc                10063a64 f   useasm:useopt.obj
 0001:00062aa0       IsNode                     10063aa0 f   useasm:useopt.obj
 0001:00062b3c       RegToNode                  10063b3c f   useasm:useopt.obj
 0001:00062b90       FixUseoptData              10063b90 f   useasm:useopt.obj
 0001:00062c4c       InitOptState               10063c4c f   useasm:useopt.obj
 0001:00062e58       SetInstFlags               10063e58 f   useasm:useopt.obj
 0001:00062ed4       UsesSrc0                   10063ed4 f   useasm:useopt.obj
 0001:00063030       ExtractSop2Spec            10064030 f   useasm:useopt.obj
 0001:000633ac       EncodeSop2Spec             100643ac f   useasm:useopt.obj
 0001:00063650       EncodeSop3Spec             10064650 f   useasm:useopt.obj
 0001:00063888       IsMove                     10064888 f   useasm:useopt.obj
 0001:00063a48       RemoveInst                 10064a48 f   useasm:useopt.obj
 0001:00063ad8       GetNextInst                10064ad8 f   useasm:useopt.obj
 0001:00063b18       DeleteInst                 10064b18 f   useasm:useopt.obj
 0001:00063bc8       InsertBefore               10064bc8 f   useasm:useopt.obj
 0001:00063c3c       EmitMove                   10064c3c f   useasm:useopt.obj
 0001:00063ce4       CanUseSrc                  10064ce4 f   useasm:useopt.obj
 0001:00063ec8       SubstInstSrc               10064ec8 f   useasm:useopt.obj
 0001:00064078       UpdateNodeRepl             10065078 f   useasm:useopt.obj
 0001:00064158       GetNodeRepl                10065158 f   useasm:useopt.obj
 0001:000642a8       MunchMovs                  100652a8 f   useasm:useopt.obj
 0001:00064558       SetRegValues               10065558 f   useasm:useopt.obj
 0001:0006466c       Sop2AddMult                1006566c f   useasm:useopt.obj
 0001:00064aa0       Sop2MultAdd                10065aa0 f   useasm:useopt.obj
 0001:00064ef0       ElimUnusedAlpha            10065ef0 f   useasm:useopt.obj
 0001:00065358       IsScalingSop               10066358 f   useasm:useopt.obj
 0001:00065474       Sop2Scaling                10066474 f   useasm:useopt.obj
 0001:0006558c       PeepHoleSop2               1006658c f   useasm:useopt.obj
 0001:0006581c       EliminateMoves             1006681c f   useasm:useopt.obj
 0001:00065b50       SplitBlock                 10066b50 f   useasm:useopt.obj
 0001:00065be0       FormRepeatsBlock           10066be0 f   useasm:useopt.obj
 0001:00065dcc       OptimiseBlock              10066dcc f   useasm:useopt.obj
 0001:0006b008       AddRegToList               1006c008 f   libffgen:reg.obj
 0001:0006b2c4       GetTemp                    1006c2c4 f   libffgen:reg.obj
 0001:0006bcd0       LoadConstant               1006ccd0 f   libffgen:reg.obj
 0001:0006bd78       RelativeAddressingSA       1006cd78 f   libffgen:reg.obj
 0001:0006c678       StoreInstruction           1006d678 f   libffgen:inst.obj
 0001:0006c988       CheckRegUsage              1006d988 f   libffgen:inst.obj
 0001:0006d110       SetupNoSchedBeforeEFOs     1006e110 f   libffgen:inst.obj
 0001:0006d21c       M4x4_efos                  1006e21c f   libffgen:inst.obj
 0001:0006da6c       M4x4_dp4                   1006ea6c f   libffgen:inst.obj
 0001:00072ea8       _DllMainCRTStartupHelper   10073ea8 f   corelib0:pegdmain.obj
 0001:000730e8       doexit                     100740e8 f   corelib0:cexit.obj
